 opencl_support

 Timestamp is 5c7622d3 (Wed Feb 27 12:40:35 2019)

 Preferred load address is 10000000

 Start         Length     Name                   Class
 0001:00000000 00000a1bH .text$di                CODE
 0001:00000a20 0000583eH .text$mn                CODE
 0001:00006260 00000b73H .text$x                 CODE
 0001:00006de0 000001ebH .text$yd                CODE
 0002:00000000 0000041cH .idata$5                DATA
 0002:0000041c 00000004H .CRT$XCA                DATA
 0002:00000420 00000068H .CRT$XCU                DATA
 0002:00000488 00000004H .CRT$XCZ                DATA
 0002:0000048c 00000004H .CRT$XIA                DATA
 0002:00000490 00000004H .CRT$XIAA               DATA
 0002:00000494 00000004H .CRT$XIC                DATA
 0002:00000498 00000004H .CRT$XIZ                DATA
 0002:000004a0 00000d18H .rdata                  DATA
 0002:000011b8 00000074H .rdata$debug            DATA
 0002:0000122c 000007fcH .rdata$r                DATA
 0002:00001a30 000000c8H .rdata$sxdata           DATA
 0002:00001af8 00000004H .rtc$IAA                DATA
 0002:00001afc 00000004H .rtc$IZZ                DATA
 0002:00001b00 00000004H .rtc$TAA                DATA
 0002:00001b04 00000004H .rtc$TZZ                DATA
 0002:00001b08 00000e24H .xdata$x                DATA
 0002:00002930 00000099H .edata                  DATA
 0002:000029cc 000000a0H .idata$2                DATA
 0002:00002a6c 00000014H .idata$3                DATA
 0002:00002a80 0000041cH .idata$4                DATA
 0002:00002e9c 00002a36H .idata$6                DATA
 0003:00000000 00000084H .data                   DATA
 0003:00000084 000003a8H .data$r                 DATA
 0003:00000430 000003ecH .bss                    DATA
 0004:00000000 00000058H .rsrc$01                DATA
 0004:00000060 00000180H .rsrc$02                DATA

  Address         Publics by Value              Rva+Base       Lib:Object

 0000:00000000       ___guard_fids_table        00000000     <absolute>
 0000:00000000       __except_list              00000000     <absolute>
 0000:00000000       ___guard_flags             00000000     <absolute>
 0000:00000000       ___guard_fids_count        00000000     <absolute>
 0000:00000032       ___safe_se_handler_count   00000032     <absolute>
 0000:00009876       __ldused                   00009876     <absolute>
 0000:00009876       __fltused                  00009876     <absolute>
 0000:00000000       ___ImageBase               10000000     <linker-defined>
 0001:00000a20       ??$_Allocate@D@std@@YAPADIPAD@Z 10001a20 f i OpenCLSupportPlugin.obj
 0001:00000a50       ??$addressof@D@std@@YAPADAAD@Z 10001a50 f i OpenCLSupportPlugin.obj
 0001:00000a60       ??$atomic@H@?$QAtomicOpsBySize@$03@@CAPAJPAH@Z 10001a60 f i OpenCLSupportPlugin.obj
 0001:00000a70       ??$construct@PADAAPAD@?$_Wrap_alloc@V?$allocator@D@std@@@std@@QAEXPAPADAAPAD@Z 10001a70 f i OpenCLSupportPlugin.obj
 0001:00000a90       ??$construct@PADAAPAD@?$allocator@D@std@@QAEXPAPADAAPAD@Z 10001a90 f i OpenCLSupportPlugin.obj
 0001:00000ab0       ??$construct@PADAAPAD@?$allocator_traits@V?$allocator@D@std@@@std@@SAXAAV?$allocator@D@1@PAPADAAPAD@Z 10001ab0 f i OpenCLSupportPlugin.obj
 0001:00000ad0       ??$deref@H@?$QAtomicOpsBySize@$03@@SA_NAAH@Z 10001ad0 f i OpenCLSupportPlugin.obj
 0001:00000af0       ??$destroy@PAD@?$_Wrap_alloc@V?$allocator@D@std@@@std@@QAEXPAPAD@Z 10001af0 f i OpenCLSupportPlugin.obj
 0001:00000b00       ??$destroy@PAD@?$allocator@D@std@@QAEXPAPAD@Z 10001b00 f i OpenCLSupportPlugin.obj
 0001:00000b10       ??$destroy@PAD@?$allocator_traits@V?$allocator@D@std@@@std@@SAXAAV?$allocator@D@1@PAPAD@Z 10001b10 f i OpenCLSupportPlugin.obj
 0001:00000b20       ??$forward@AAPAD@std@@YAAAPADAAPAD@Z 10001b20 f i OpenCLSupportPlugin.obj
 0001:00000b30       ??$load@H@?$QGenericAtomicOps@U?$QAtomicOpsBySize@$03@@@@SAHABH@Z 10001b30 f i OpenCLSupportPlugin.obj
 0001:00000b40       ??$ref@H@?$QAtomicOpsBySize@$03@@SA_NAAH@Z 10001b40 f i OpenCLSupportPlugin.obj
 0001:00000b60       ??0?$QForeachContainer@V?$QList@PAVOpenCLGpuModel@U2@@@@@@QAE@ABV?$QList@PAVOpenCLGpuModel@U2@@@@@Z 10001b60 f i OpenCLSupportPlugin.obj
 0001:00000ba0       ??0?$QList@PAVOpenCLGpuModel@U2@@@@QAE@ABV0@@Z 10001ba0 f i OpenCLSupportPlugin.obj
 0001:00000c60       ??0?$QList@PAVOpenCLGpuModel@U2@@@@QAE@XZ 10001c60 f i OpenCLSupportPlugin.obj
 0001:00000c70       ??0?$QScopedPointer@VOpenCLSupportPlugin@U2@@U?$QScopedPointerDeleter@VOpenCLSupportPlugin@U2@@@@@@QAE@PAVOpenCLSupportPlugin@U2@@@Z 10001c70 f i OpenCLSupportPlugin.obj
 0001:00000c80       ??0?$_String_alloc@$0A@U?$_String_base_types@DV?$allocator@D@std@@@std@@@std@@QAE@ABV?$allocator@D@1@@Z 10001c80 f i OpenCLSupportPlugin.obj
 0001:00000ca0       ??0?$_String_val@U?$_Simple_types@D@std@@@std@@QAE@XZ 10001ca0 f i OpenCLSupportPlugin.obj
 0001:00000cc0       ??0?$_Wrap_alloc@V?$allocator@D@std@@@std@@QAE@XZ 10001cc0 f i OpenCLSupportPlugin.obj
 0001:00000cd0       ??0?$allocator@D@std@@QAE@XZ 10001cd0 f i OpenCLSupportPlugin.obj
 0001:00000ce0       ??0?$basic_string@DU?$char_traits@D@std@@V?$allocator@D@2@@std@@QAE@PBD@Z 10001ce0 f i OpenCLSupportPlugin.obj
 0001:00000d40       ??0?$gauto_array@D@U2@@QAE@PAD@Z 10001d40 f i OpenCLSupportPlugin.obj
 0001:00000d50       ??0?$gauto_array@PAU_cl_device_id@@@U2@@QAE@PAPAU_cl_device_id@@@Z 10001d50 f i OpenCLSupportPlugin.obj
 0001:00000d60       ??0?$gauto_array@PAU_cl_platform_id@@@U2@@QAE@PAPAU_cl_platform_id@@@Z 10001d60 f i OpenCLSupportPlugin.obj
 0001:00000d70       ??0OpenCLSupportPlugin@U2@@QAE@XZ 10001d70 f   OpenCLSupportPlugin.obj
 0001:00001010       ??0QLatin1Char@@QAE@D@Z    10002010 f i OpenCLSupportPlugin.obj
 0001:00001020       ??0_Generic_error_category@std@@QAE@XZ 10002020 f i OpenCLSupportPlugin.obj
 0001:00001030       ??0_Ignore@std@@QAE@XZ     10002030 f i OpenCLSupportPlugin.obj
 0001:00001040       ??0_Iostream_error_category@std@@QAE@XZ 10002040 f i OpenCLSupportPlugin.obj
 0001:00001050       ??0_System_error_category@std@@QAE@XZ 10002050 f i OpenCLSupportPlugin.obj
 0001:00001060       ??0const_iterator@?$QList@PAVOpenCLGpuModel@U2@@@@QAE@PAUNode@1@@Z 10002060 f i OpenCLSupportPlugin.obj
 0001:00001070       ??0error_category@std@@QAE@XZ 10002070 f i OpenCLSupportPlugin.obj
 0001:00001080       ??0error_condition@std@@QAE@HABVerror_category@1@@Z 10002080 f i OpenCLSupportPlugin.obj
 0001:000010a0       ??1?$QForeachContainer@V?$QList@PAVOpenCLGpuModel@U2@@@@@@QAE@XZ 100020a0 f i OpenCLSupportPlugin.obj
 0001:000010d0       ??1?$QList@PAVOpenCLGpuModel@U2@@@@QAE@XZ 100020d0 f i OpenCLSupportPlugin.obj
 0001:00001100       ??1?$QScopedPointer@VOpenCLSupportPlugin@U2@@U?$QScopedPointerDeleter@VOpenCLSupportPlugin@U2@@@@@@QAE@XZ 10002100 f i OpenCLSupportPlugin.obj
 0001:00001110       ??1?$basic_string@DU?$char_traits@D@std@@V?$allocator@D@2@@std@@QAE@XZ 10002110 f i OpenCLSupportPlugin.obj
 0001:00001140       ??1?$gauto_array@D@U2@@QAE@XZ 10002140 f i OpenCLSupportPlugin.obj
 0001:00001150       ??1?$gauto_array@PAU_cl_device_id@@@U2@@QAE@XZ 10002150 f i OpenCLSupportPlugin.obj
 0001:00001160       ??1?$gauto_array@PAU_cl_platform_id@@@U2@@QAE@XZ 10002160 f i OpenCLSupportPlugin.obj
 0001:00001170       ??1OpenCLSupportPlugin@U2@@UAE@XZ 10002170 f   OpenCLSupportPlugin.obj
 0001:00001230       ??1_Generic_error_category@std@@UAE@XZ 10002230 f i OpenCLSupportPlugin.obj
 0001:00001240       ??1_Iostream_error_category@std@@UAE@XZ 10002240 f i OpenCLSupportPlugin.obj
 0001:00001250       ??1_System_error_category@std@@UAE@XZ 10002250 f i OpenCLSupportPlugin.obj
 0001:00001260       ??1error_category@std@@UAE@XZ 10002260 f i OpenCLSupportPlugin.obj
 0001:00001270       ??2@YAPAXIPAX@Z            10002270 f i OpenCLSupportPlugin.obj
 0001:00001280       ??3@YAXPAX0@Z              10002280 f i OpenCLSupportPlugin.obj
 0001:00001290       ??8error_category@std@@QBE_NABV01@@Z 10002290 f i OpenCLSupportPlugin.obj
 0001:000012a0       ??8error_condition@std@@QBE_NABV01@@Z 100022a0 f i OpenCLSupportPlugin.obj
 0001:000012c0       ??9const_iterator@?$QList@PAVOpenCLGpuModel@U2@@@@QBE_NABV01@@Z 100022c0 f i OpenCLSupportPlugin.obj
 0001:000012e0       ??Dconst_iterator@?$QList@PAVOpenCLGpuModel@U2@@@@QBEABQAVOpenCLGpuModel@U2@@XZ 100022e0 f i OpenCLSupportPlugin.obj
 0001:000012f0       ??Econst_iterator@?$QList@PAVOpenCLGpuModel@U2@@@@QAEAAV01@XZ 100022f0 f i OpenCLSupportPlugin.obj
 0001:00001300       ??H@YA?BVQString@@ABV0@0@Z 10002300 f i OpenCLSupportPlugin.obj
 0001:00001370       ??H@YA?BVQString@@ABV0@PBD@Z 10002370 f i OpenCLSupportPlugin.obj
 0001:00001410       ??H@YA?BVQString@@PBDABV0@@Z 10002410 f i OpenCLSupportPlugin.obj
 0001:00001480       ??_GAppResourceSemaphore@U2@@UAEPAXI@Z 10002480 f i OpenCLSupportPlugin.obj
 0001:00001480       ??_EAppResourceSemaphore@U2@@UAEPAXI@Z 10002480 f i OpenCLSupportPlugin.obj
 0001:000014b0       ??_EOpenCLSupportPlugin@U2@@UAEPAXI@Z 100024b0 f i OpenCLSupportPlugin.obj
 0001:000014b0       ??_GOpenCLSupportPlugin@U2@@UAEPAXI@Z 100024b0 f i OpenCLSupportPlugin.obj
 0001:000014e0       ??_E_Generic_error_category@std@@UAEPAXI@Z 100024e0 f i OpenCLSupportPlugin.obj
 0001:000014e0       ??_G_Generic_error_category@std@@UAEPAXI@Z 100024e0 f i OpenCLSupportPlugin.obj
 0001:00001510       ??_E_Iostream_error_category@std@@UAEPAXI@Z 10002510 f i OpenCLSupportPlugin.obj
 0001:00001510       ??_G_Iostream_error_category@std@@UAEPAXI@Z 10002510 f i OpenCLSupportPlugin.obj
 0001:00001540       ??_E_System_error_category@std@@UAEPAXI@Z 10002540 f i OpenCLSupportPlugin.obj
 0001:00001540       ??_G_System_error_category@std@@UAEPAXI@Z 10002540 f i OpenCLSupportPlugin.obj
 0001:00001570       ??_Eerror_category@std@@UAEPAXI@Z 10002570 f i OpenCLSupportPlugin.obj
 0001:00001570       ??_Gerror_category@std@@UAEPAXI@Z 10002570 f i OpenCLSupportPlugin.obj
 0001:000015a0       ?_Copy@?$basic_string@DU?$char_traits@D@std@@V?$allocator@D@2@@std@@QAEXII@Z 100025a0 f i OpenCLSupportPlugin.obj
 0001:000016f0       ?_Eos@?$basic_string@DU?$char_traits@D@std@@V?$allocator@D@2@@std@@QAEXI@Z 100026f0 f i OpenCLSupportPlugin.obj
 0001:00001720       ?_Getal@?$_String_alloc@$0A@U?$_String_base_types@DV?$allocator@D@std@@@std@@@std@@QBE?AU?$_Wrap_alloc@V?$allocator@D@std@@@2@XZ 10002720 f i OpenCLSupportPlugin.obj
 0001:00001730       ?_Grow@?$basic_string@DU?$char_traits@D@std@@V?$allocator@D@2@@std@@QAE_NI_N@Z 10002730 f i OpenCLSupportPlugin.obj
 0001:000017e0       ?_Inside@?$basic_string@DU?$char_traits@D@std@@V?$allocator@D@2@@std@@QAE_NPBD@Z 100027e0 f i OpenCLSupportPlugin.obj
 0001:00001820       ?_Myptr@?$_String_val@U?$_Simple_types@D@std@@@std@@QAEPADXZ 10002820 f i OpenCLSupportPlugin.obj
 0001:00001830       ?_Myptr@?$_String_val@U?$_Simple_types@D@std@@@std@@QBEPBDXZ 10002830 f i OpenCLSupportPlugin.obj
 0001:00001840       ?_Tidy@?$basic_string@DU?$char_traits@D@std@@V?$allocator@D@2@@std@@QAEX_NI@Z 10002840 f i OpenCLSupportPlugin.obj
 0001:00001890       ?_Xlen@?$basic_string@DU?$char_traits@D@std@@V?$allocator@D@2@@std@@QBEXXZ 10002890 f i OpenCLSupportPlugin.obj
 0001:000018a0       ?_Xran@?$basic_string@DU?$char_traits@D@std@@V?$allocator@D@2@@std@@QBEXXZ 100028a0 f i OpenCLSupportPlugin.obj
 0001:000018b0       ?allocate@?$_Wrap_alloc@V?$allocator@D@std@@@std@@QAEPADI@Z 100028b0 f i OpenCLSupportPlugin.obj
 0001:000018e0       ?allocate@?$allocator@D@std@@QAEPADI@Z 100028e0 f i OpenCLSupportPlugin.obj
 0001:00001910       ?append@?$QList@PAVOpenCLGpuModel@U2@@@@QAEXABQAVOpenCLGpuModel@U2@@@Z 10002910 f i OpenCLSupportPlugin.obj
 0001:000019a0       ?assign@?$basic_string@DU?$char_traits@D@std@@V?$allocator@D@2@@std@@QAEAAV12@ABV12@II@Z 100029a0 f i OpenCLSupportPlugin.obj
 0001:00001ac0       ?assign@?$basic_string@DU?$char_traits@D@std@@V?$allocator@D@2@@std@@QAEAAV12@PBD@Z 10002ac0 f i OpenCLSupportPlugin.obj
 0001:00001b00       ?assign@?$basic_string@DU?$char_traits@D@std@@V?$allocator@D@2@@std@@QAEAAV12@PBDI@Z 10002b00 f i OpenCLSupportPlugin.obj
 0001:00001c00       ?assign@?$char_traits@D@std@@SAXAADABD@Z 10002c00 f i OpenCLSupportPlugin.obj
 0001:00001c10       ?begin@?$QList@PAVOpenCLGpuModel@U2@@@@QBE?AVconst_iterator@1@XZ 10002c10 f i OpenCLSupportPlugin.obj
 0001:00001c30       ?category@error_code@std@@QBEABVerror_category@2@XZ 10002c30 f i OpenCLSupportPlugin.obj
 0001:00001c40       ?category@error_condition@std@@QBEABVerror_category@2@XZ 10002c40 f i OpenCLSupportPlugin.obj
 0001:00001c50       ?cleanup@?$QScopedPointerDeleter@VOpenCLSupportPlugin@U2@@@@SAXPAVOpenCLSupportPlugin@U2@@@Z 10002c50 f i OpenCLSupportPlugin.obj
 0001:00001c70       ?copy@?$char_traits@D@std@@SAPADPADPBDI@Z 10002c70 f i OpenCLSupportPlugin.obj
 0001:00001c90       ?dealloc@?$QList@PAVOpenCLGpuModel@U2@@@@AAEXPAUData@QListData@@@Z 10002c90 f i OpenCLSupportPlugin.obj
 0001:00001cb0       ?deallocate@?$_Wrap_alloc@V?$allocator@D@std@@@std@@QAEXPADI@Z 10002cb0 f i OpenCLSupportPlugin.obj
 0001:00001cd0       ?deallocate@?$allocator@D@std@@QAEXPADI@Z 10002cd0 f i OpenCLSupportPlugin.obj
 0001:00001cf0       ?default_error_condition@_System_error_category@std@@UBE?AVerror_condition@2@H@Z 10002cf0 f i OpenCLSupportPlugin.obj
 0001:00001d30       ?default_error_condition@error_category@std@@UBE?AVerror_condition@2@H@Z 10002d30 f i OpenCLSupportPlugin.obj
 0001:00001d50       ?deref@?$QBasicAtomicInteger@H@@QAE_NXZ 10002d50 f i OpenCLSupportPlugin.obj
 0001:00001d60       ?deref@RefCount@QtPrivate@@QAE_NXZ 10002d60 f i OpenCLSupportPlugin.obj
 0001:00001d80       ?detach_helper_grow@?$QList@PAVOpenCLGpuModel@U2@@@@AAEPAUNode@1@HH@Z 10002d80 f i OpenCLSupportPlugin.obj
 0001:00001e90       ?empty@?$QList@PAVOpenCLGpuModel@U2@@@@QBE_NXZ 10002e90 f i OpenCLSupportPlugin.obj
 0001:00001ea0       ?end@?$QList@PAVOpenCLGpuModel@U2@@@@QBE?AVconst_iterator@1@XZ 10002ea0 f i OpenCLSupportPlugin.obj
 0001:00001ec0       ?equivalent@error_category@std@@UBE_NABVerror_code@2@H@Z 10002ec0 f i OpenCLSupportPlugin.obj
 0001:00001ee0       ?equivalent@error_category@std@@UBE_NHABVerror_condition@2@@Z 10002ee0 f i OpenCLSupportPlugin.obj
 0001:00001f20       ?erase@?$basic_string@DU?$char_traits@D@std@@V?$allocator@D@2@@std@@QAEAAV12@I@Z 10002f20 f i OpenCLSupportPlugin.obj
 0001:00001f60       ?erase@?$basic_string@DU?$char_traits@D@std@@V?$allocator@D@2@@std@@QAEAAV12@II@Z 10002f60 f i OpenCLSupportPlugin.obj
 0001:00002000       ?generic_category@std@@YAABVerror_category@1@XZ 10003000 f i OpenCLSupportPlugin.obj
 0001:00002010       ?get@?$gauto_array@D@U2@@QBEPADXZ 10003010 f i OpenCLSupportPlugin.obj
 0001:00002020       ?get@?$gauto_array@PAU_cl_device_id@@@U2@@QBEPAPAU_cl_device_id@@XZ 10003020 f i OpenCLSupportPlugin.obj
 0001:00002030       ?get@?$gauto_array@PAU_cl_platform_id@@@U2@@QBEPAPAU_cl_platform_id@@XZ 10003030 f i OpenCLSupportPlugin.obj
 0001:00002040       ?getError@OpenCLSupportPlugin@U2@@QBE?AW4OpenCLSupportError@12@XZ 10003040 f   OpenCLSupportPlugin.obj
 0001:00002050       ?getSettingsErrorString@OpenCLSupportPlugin@U2@@CA?AVQString@@W4OpenCLSupportError@12@@Z 10003050 f   OpenCLSupportPlugin.obj
 0001:000020d0       ?hasOPENCLError@OpenCLSupportPlugin@U2@@AAE_NHAAVQString@@@Z 100030d0 f   OpenCLSupportPlugin.obj
 0001:00002190       ?isEmpty@?$QList@PAVOpenCLGpuModel@U2@@@@QBE_NXZ 10003190 f i OpenCLSupportPlugin.obj
 0001:000021a0       ?isShared@RefCount@QtPrivate@@QBE_NXZ 100031a0 f i OpenCLSupportPlugin.obj
 0001:000021c0       ?length@?$char_traits@D@std@@SAIPBD@Z 100031c0 f i OpenCLSupportPlugin.obj
 0001:000021e0       ?load@?$QBasicAtomicInteger@H@@QBEHXZ 100031e0 f i OpenCLSupportPlugin.obj
 0001:000021f0       ?loadGpusSettings@OpenCLSupportPlugin@U2@@AAEXXZ 100031f0 f   OpenCLSupportPlugin.obj
 0001:00002380       ?max_size@?$_Wrap_alloc@V?$allocator@D@std@@@std@@QBEIXZ 10003380 f i OpenCLSupportPlugin.obj
 0001:00002390       ?max_size@?$allocator@D@std@@QBEIXZ 10003390 f i OpenCLSupportPlugin.obj
 0001:000023a0       ?max_size@?$allocator_traits@V?$allocator@D@std@@@std@@SAIABV?$allocator@D@2@@Z 100033a0 f i OpenCLSupportPlugin.obj
 0001:000023b0       ?max_size@?$basic_string@DU?$char_traits@D@std@@V?$allocator@D@2@@std@@QBEIXZ 100033b0 f i OpenCLSupportPlugin.obj
 0001:000023c0       ?message@_Generic_error_category@std@@UBE?AV?$basic_string@DU?$char_traits@D@std@@V?$allocator@D@2@@2@H@Z 100033c0 f i OpenCLSupportPlugin.obj
 0001:00002440       ?message@_Iostream_error_category@std@@UBE?AV?$basic_string@DU?$char_traits@D@std@@V?$allocator@D@2@@2@H@Z 10003440 f i OpenCLSupportPlugin.obj
 0001:00002490       ?message@_System_error_category@std@@UBE?AV?$basic_string@DU?$char_traits@D@std@@V?$allocator@D@2@@2@H@Z 10003490 f i OpenCLSupportPlugin.obj
 0001:00002510       ?move@?$char_traits@D@std@@SAPADPADPBDI@Z 10003510 f i OpenCLSupportPlugin.obj
 0001:00002530       ?name@_Generic_error_category@std@@UBEPBDXZ 10003530 f i OpenCLSupportPlugin.obj
 0001:00002540       ?name@_Iostream_error_category@std@@UBEPBDXZ 10003540 f i OpenCLSupportPlugin.obj
 0001:00002550       ?name@_System_error_category@std@@UBEPBDXZ 10003550 f i OpenCLSupportPlugin.obj
 0001:00002560       ?node_construct@?$QList@PAVOpenCLGpuModel@U2@@@@AAEXPAUNode@1@ABQAVOpenCLGpuModel@U2@@@Z 10003560 f i OpenCLSupportPlugin.obj
 0001:00002580       ?node_copy@?$QList@PAVOpenCLGpuModel@U2@@@@AAEXPAUNode@1@00@Z 10003580 f i OpenCLSupportPlugin.obj
 0001:000025b0       ?node_destruct@?$QList@PAVOpenCLGpuModel@U2@@@@AAEXPAUNode@1@0@Z 100035b0 f i OpenCLSupportPlugin.obj
 0001:000025c0       ?node_destruct@?$QList@PAVOpenCLGpuModel@U2@@@@AAEXPAUNode@1@@Z 100035c0 f i OpenCLSupportPlugin.obj
 0001:000025d0       ?obtainGpusInfo@OpenCLSupportPlugin@U2@@AAE?AW4OpenCLSupportError@12@AAVQString@@@Z 100035d0 f   OpenCLSupportPlugin.obj
 0001:00002f70       ?push_back@?$QList@PAVOpenCLGpuModel@U2@@@@QAEXABQAVOpenCLGpuModel@U2@@@Z 10003f70 f i OpenCLSupportPlugin.obj
 0001:00002f80       ?ref@?$QBasicAtomicInteger@H@@QAE_NXZ 10003f80 f i OpenCLSupportPlugin.obj
 0001:00002fa0       ?ref@RefCount@QtPrivate@@QAE_NXZ 10003fa0 f i OpenCLSupportPlugin.obj
 0001:00002fc0       ?registerAvailableGpus@OpenCLSupportPlugin@U2@@AAEXXZ 10003fc0 f   OpenCLSupportPlugin.obj
 0001:00003090       ?size@?$QList@PAVOpenCLGpuModel@U2@@@@QBEHXZ 10004090 f i OpenCLSupportPlugin.obj
 0001:000030a0       ?size@?$basic_string@DU?$char_traits@D@std@@V?$allocator@D@2@@std@@QBEIXZ 100040a0 f i OpenCLSupportPlugin.obj
 0001:000030b0       ?system_category@std@@YAABVerror_category@1@XZ 100040b0 f i OpenCLSupportPlugin.obj
 0001:000030c0       ?t@Node@?$QList@PAVOpenCLGpuModel@U2@@@@QAEAAPAVOpenCLGpuModel@U2@@XZ 100040c0 f i OpenCLSupportPlugin.obj
 0001:000030d0       ?tr@OpenCLSupportPlugin@U2@@SA?AVQString@@PBD0H@Z 100040d0 f i OpenCLSupportPlugin.obj
 0001:00003100       ?unregisterAvailableGpus@OpenCLSupportPlugin@U2@@AAEXXZ 10004100 f   OpenCLSupportPlugin.obj
 0001:000031d0       ?value@error_code@std@@QBEHXZ 100041d0 f i OpenCLSupportPlugin.obj
 0001:000031e0       ?value@error_condition@std@@QBEHXZ 100041e0 f i OpenCLSupportPlugin.obj
 0001:000031f0       _hypot                     100041f0 f i OpenCLSupportPlugin.obj
 0001:00003220       _ugene_plugin_fail_message 10004220 f   OpenCLSupportPlugin.obj
 0001:000032c0       _ugene_plugin_init         100042c0 f   OpenCLSupportPlugin.obj
 0001:000032e0       _ugene_plugin_verify       100042e0 f   OpenCLSupportPlugin.obj
 0001:00003320       ??$_Count_np@PB_N_N@std@@YAHPB_N0AB_N@Z 10004320 f i OpenCLSupportSettingsController.obj
 0001:00003360       ??$_Unchecked@PB_N@std@@YAPB_NPB_N@Z 10004360 f i OpenCLSupportSettingsController.obj
 0001:00003370       ??$count@PB_N_N@std@@YAHPB_N0AB_N@Z 10004370 f i OpenCLSupportSettingsController.obj
 0001:000033b0       ??$qobject_cast@PAVOpenCLSupportSettingsPageState@U2@@@@YAPAVOpenCLSupportSettingsPageState@U2@@PAVQObject@@@Z 100043b0 f i OpenCLSupportSettingsController.obj
 0001:000033d0       ??0?$QFlags@W4AlignmentFlag@Qt@@@@QAE@PQPrivate@0@H@Z 100043d0 f i OpenCLSupportSettingsController.obj
 0001:000033e0       ??0?$QFlags@W4AlignmentFlag@Qt@@@@QAE@VQFlag@@@Z 100043e0 f i OpenCLSupportSettingsController.obj
 0001:000033f0       ??0?$QFlags@W4AlignmentFlag@Qt@@@@QAE@W4AlignmentFlag@Qt@@@Z 100043f0 f i OpenCLSupportSettingsController.obj
 0001:00003400       ??0?$QFlags@W4AllocationOption@QArrayData@@@@QAE@PQPrivate@0@H@Z 10004400 f i OpenCLSupportSettingsController.obj
 0001:00003410       ??0?$QFlags@W4AllocationOption@QArrayData@@@@QAE@W4AllocationOption@QArrayData@@@Z 10004410 f i OpenCLSupportSettingsController.obj
 0001:00003420       ??0?$QFlags@W4WindowType@Qt@@@@QAE@PQPrivate@0@H@Z 10004420 f i OpenCLSupportSettingsController.obj
 0001:00003430       ??0?$QList@PAVQCheckBox@@@@QAE@XZ 10004430 f i OpenCLSupportSettingsController.obj
 0001:00003440       ??0?$QVector@_N@@QAE@XZ    10004440 f i OpenCLSupportSettingsController.obj
 0001:00003450       ??0OpenCLSupportSettingsPageController@U2@@QAE@ABVQString@@PAVQObject@@@Z 10004450 f   OpenCLSupportSettingsController.obj
 0001:00003500       ??0OpenCLSupportSettingsPageState@U2@@QAE@H@Z 10004500 f   OpenCLSupportSettingsController.obj
 0001:000035a0       ??0OpenCLSupportSettingsPageWidget@U2@@QAE@ABVQString@@PAVOpenCLSupportSettingsPageController@1@@Z 100045a0 f   OpenCLSupportSettingsController.obj
 0001:00003a70       ??0QFlag@@QAE@H@Z          10004a70 f i OpenCLSupportSettingsController.obj
 0001:00003a80       ??1?$QList@PAVQCheckBox@@@@QAE@XZ 10004a80 f i OpenCLSupportSettingsController.obj
 0001:00003ab0       ??1?$QVector@_N@@QAE@XZ    10004ab0 f i OpenCLSupportSettingsController.obj
 0001:00003af0       ??1OpenCLSupportSettingsPageController@U2@@UAE@XZ 10004af0 f i OpenCLSupportSettingsController.obj
 0001:00003b50       ??1OpenCLSupportSettingsPageState@U2@@UAE@XZ 10004b50 f i OpenCLSupportSettingsController.obj
 0001:00003be0       ??1OpenCLSupportSettingsPageWidget@U2@@UAE@XZ 10004be0 f i OpenCLSupportSettingsController.obj
 0001:00003c70       ??A?$QList@PAVOpenCLGpuModel@U2@@@@QAEAAPAVOpenCLGpuModel@U2@@H@Z 10004c70 f i OpenCLSupportSettingsController.obj
 0001:00003ca0       ??A?$QVector@_N@@QAEAA_NH@Z 10004ca0 f i OpenCLSupportSettingsController.obj
 0001:00003d10       ??BQFlag@@QBEHXZ           10004d10 f i OpenCLSupportSettingsController.obj
 0001:00003d20       ??U?$QFlags@W4AlignmentFlag@Qt@@@@QBE?AV0@W4AlignmentFlag@Qt@@@Z 10004d20 f i OpenCLSupportSettingsController.obj
 0001:00003d40       ??U@YA?AV?$QFlags@W4AlignmentFlag@Qt@@@@W4AlignmentFlag@Qt@@0@Z 10004d40 f i OpenCLSupportSettingsController.obj
 0001:00003d50       ??_EOpenCLSupportSettingsPageWidget@U2@@W7AEPAXI@Z 10004d50 f i OpenCLSupportSettingsController.obj
 0001:00003d58       ??_EQCheckBox@@W7AEPAXI@Z  10004d58 f i OpenCLSupportSettingsController.obj
 0001:00003d60       ??_EQHBoxLayout@@W7AEPAXI@Z 10004d60 f i OpenCLSupportSettingsController.obj
 0001:00003d68       ??_EQLabel@@W7AEPAXI@Z     10004d68 f i OpenCLSupportSettingsController.obj
 0001:00003d70       ??_EQVBoxLayout@@W7AEPAXI@Z 10004d70 f i OpenCLSupportSettingsController.obj
 0001:00003d80       ??_GOpenCLSupportSettingsPageController@U2@@UAEPAXI@Z 10004d80 f i OpenCLSupportSettingsController.obj
 0001:00003d80       ??_EOpenCLSupportSettingsPageController@U2@@UAEPAXI@Z 10004d80 f i OpenCLSupportSettingsController.obj
 0001:00003df0       ??_EOpenCLSupportSettingsPageState@U2@@UAEPAXI@Z 10004df0 f i OpenCLSupportSettingsController.obj
 0001:00003df0       ??_GOpenCLSupportSettingsPageState@U2@@UAEPAXI@Z 10004df0 f i OpenCLSupportSettingsController.obj
 0001:00003ea0       ??_GOpenCLSupportSettingsPageWidget@U2@@UAEPAXI@Z 10004ea0 f i OpenCLSupportSettingsController.obj
 0001:00003ea0       ??_EOpenCLSupportSettingsPageWidget@U2@@UAEPAXI@Z 10004ea0 f i OpenCLSupportSettingsController.obj
 0001:00003f40       ??_GQCheckBox@@UAEPAXI@Z   10004f40 f i OpenCLSupportSettingsController.obj
 0001:00003f40       ??_EQCheckBox@@UAEPAXI@Z   10004f40 f i OpenCLSupportSettingsController.obj
 0001:00003f70       ??_GQHBoxLayout@@UAEPAXI@Z 10004f70 f i OpenCLSupportSettingsController.obj
 0001:00003f70       ??_EQHBoxLayout@@UAEPAXI@Z 10004f70 f i OpenCLSupportSettingsController.obj
 0001:00003fa0       ??_GQLabel@@UAEPAXI@Z      10004fa0 f i OpenCLSupportSettingsController.obj
 0001:00003fa0       ??_EQLabel@@UAEPAXI@Z      10004fa0 f i OpenCLSupportSettingsController.obj
 0001:00003fd0       ??_GQVBoxLayout@@UAEPAXI@Z 10004fd0 f i OpenCLSupportSettingsController.obj
 0001:00003fd0       ??_EQVBoxLayout@@UAEPAXI@Z 10004fd0 f i OpenCLSupportSettingsController.obj
 0001:00004000       ?allocate@?$QTypedArrayData@_N@@SAPAU1@IV?$QFlags@W4AllocationOption@QArrayData@@@@@Z 10005000 f i OpenCLSupportSettingsController.obj
 0001:00004020       ?append@?$QList@PAVQCheckBox@@@@QAEXABQAVQCheckBox@@@Z 10005020 f i OpenCLSupportSettingsController.obj
 0001:000040b0       ?at@?$QList@PAVOpenCLGpuModel@U2@@@@QBEABQAVOpenCLGpuModel@U2@@H@Z 100050b0 f i OpenCLSupportSettingsController.obj
 0001:000040d0       ?at@?$QList@PAVQCheckBox@@@@QBEABQAVQCheckBox@@H@Z 100050d0 f i OpenCLSupportSettingsController.obj
 0001:000040f0       ?at@?$QVector@_N@@QBEAB_NH@Z 100050f0 f i OpenCLSupportSettingsController.obj
 0001:00004110       ?begin@?$QTypedArrayData@_N@@QAEPA_NPA_N@Z 10005110 f i OpenCLSupportSettingsController.obj
 0001:00004120       ?count@?$QVector@_N@@QBEHAB_N@Z 10005120 f i OpenCLSupportSettingsController.obj
 0001:00004180       ?createWidget@OpenCLSupportSettingsPageController@U2@@UAEPAVAppSettingsGUIPageWidget@2@PAVAppSettingsGUIPageState@2@@Z 10005180 f   OpenCLSupportSettingsController.obj
 0001:00004200       ?data@?$QTypedArrayData@_N@@QAEPA_NXZ 10005200 f i OpenCLSupportSettingsController.obj
 0001:00004210       ?data@?$QVector@_N@@QAEPA_NXZ 10005210 f i OpenCLSupportSettingsController.obj
 0001:00004270       ?dealloc@?$QList@PAVQCheckBox@@@@AAEXPAUData@QListData@@@Z 10005270 f i OpenCLSupportSettingsController.obj
 0001:00004290       ?deallocate@?$QTypedArrayData@_N@@SAXPAUQArrayData@@@Z 10005290 f i OpenCLSupportSettingsController.obj
 0001:000042b0       ?defaultConstruct@?$QVector@_N@@AAEXPA_N0@Z 100052b0 f i OpenCLSupportSettingsController.obj
 0001:000042d0       ?destruct@?$QVector@_N@@AAEXPA_N0@Z 100052d0 f i OpenCLSupportSettingsController.obj
 0001:000042e0       ?detach@?$QList@PAVOpenCLGpuModel@U2@@@@QAEXXZ 100052e0 f i OpenCLSupportSettingsController.obj
 0001:00004300       ?detach@?$QVector@_N@@QAEXXZ 10005300 f i OpenCLSupportSettingsController.obj
 0001:00004350       ?detach_helper@?$QList@PAVOpenCLGpuModel@U2@@@@AAEXH@Z 10005350 f i OpenCLSupportSettingsController.obj
 0001:00004420       ?detach_helper@?$QList@PAVOpenCLGpuModel@U2@@@@AAEXXZ 10005420 f i OpenCLSupportSettingsController.obj
 0001:00004430       ?detach_helper_grow@?$QList@PAVQCheckBox@@@@AAEPAUNode@1@HH@Z 10005430 f i OpenCLSupportSettingsController.obj
 0001:00004540       ?end@?$QTypedArrayData@_N@@QAEPA_NPA_N@Z 10005540 f i OpenCLSupportSettingsController.obj
 0001:00004550       ?freeData@?$QVector@_N@@AAEXPAU?$QTypedArrayData@_N@@@Z 10005550 f i OpenCLSupportSettingsController.obj
 0001:00004580       ?getHelpPageId@OpenCLSupportSettingsPageController@U2@@UBEABVQString@@XZ 10005580 f i OpenCLSupportSettingsController.obj
 0001:00004590       ?getSavedState@OpenCLSupportSettingsPageController@U2@@UAEPAVAppSettingsGUIPageState@2@XZ 10005590 f   OpenCLSupportSettingsController.obj
 0001:000046e0       ?getState@OpenCLSupportSettingsPageWidget@U2@@UBEPAVAppSettingsGUIPageState@2@AAVQString@@@Z 100056e0 f   OpenCLSupportSettingsController.obj
 0001:00004810       ?isDetached@?$QVector@_N@@QBE_NXZ 10005810 f i OpenCLSupportSettingsController.obj
 0001:00004840       ?node_construct@?$QList@PAVQCheckBox@@@@AAEXPAUNode@1@ABQAVQCheckBox@@@Z 10005840 f i OpenCLSupportSettingsController.obj
 0001:00004860       ?node_copy@?$QList@PAVQCheckBox@@@@AAEXPAUNode@1@00@Z 10005860 f i OpenCLSupportSettingsController.obj
 0001:00004890       ?node_destruct@?$QList@PAVQCheckBox@@@@AAEXPAUNode@1@0@Z 10005890 f i OpenCLSupportSettingsController.obj
 0001:000048a0       ?node_destruct@?$QList@PAVQCheckBox@@@@AAEXPAUNode@1@@Z 100058a0 f i OpenCLSupportSettingsController.obj
 0001:000048b0       ?push_back@?$QList@PAVQCheckBox@@@@QAEXABQAVQCheckBox@@@Z 100058b0 f i OpenCLSupportSettingsController.obj
 0001:000048c0       ?qt_noop@@YAXXZ            100058c0 f i OpenCLSupportSettingsController.obj
 0001:000048d0       ?reallocData@?$QVector@_N@@AAEXHHV?$QFlags@W4AllocationOption@QArrayData@@@@@Z 100058d0 f i OpenCLSupportSettingsController.obj
 0001:00004b00       ?resize@?$QVector@_N@@QAEXH@Z 10005b00 f i OpenCLSupportSettingsController.obj
 0001:00004b50       ?saveState@OpenCLSupportSettingsPageController@U2@@UAEXPAVAppSettingsGUIPageState@2@@Z 10005b50 f   OpenCLSupportSettingsController.obj
 0001:00004cf0       ?setState@OpenCLSupportSettingsPageWidget@U2@@UAEXPAVAppSettingsGUIPageState@2@@Z 10005cf0 f   OpenCLSupportSettingsController.obj
 0001:00004d50       ?sharedNull@?$QTypedArrayData@_N@@SAPAU1@XZ 10005d50 f i OpenCLSupportSettingsController.obj
 0001:00004d60       ?size@?$QList@PAVQCheckBox@@@@QBEHXZ 10005d60 f i OpenCLSupportSettingsController.obj
 0001:00004d70       ?size@?$QVector@_N@@QBEHXZ 10005d70 f i OpenCLSupportSettingsController.obj
 0001:00004d80       ?t@Node@?$QList@PAVQCheckBox@@@@QAEAAPAVQCheckBox@@XZ 10005d80 f i OpenCLSupportSettingsController.obj
 0001:00004d90       ?tr@OpenCLSupportSettingsPageController@U2@@SA?AVQString@@PBD0H@Z 10005d90 f i OpenCLSupportSettingsController.obj
 0001:00004dc0       ?tr@OpenCLSupportSettingsPageWidget@U2@@SA?AVQString@@PBD0H@Z 10005dc0 f i OpenCLSupportSettingsController.obj
 0001:00004df0       ?unsharableEmpty@?$QTypedArrayData@_N@@SAPAU1@XZ 10005df0 f i OpenCLSupportSettingsController.obj
 0001:00004e10       ??C?$QScopedPointer@VQObjectData@@U?$QScopedPointerDeleter@VQObjectData@@@@@@QBEPAVQObjectData@@XZ 10005e10 f i moc_OpenCLSupportPlugin.obj
 0001:00004e20       ?metaObject@OpenCLSupportPlugin@U2@@UBEPBUQMetaObject@@XZ 10005e20 f   moc_OpenCLSupportPlugin.obj
 0001:00004e40       ?qt_metacall@OpenCLSupportPlugin@U2@@UAEHW4Call@QMetaObject@@HPAPAX@Z 10005e40 f   moc_OpenCLSupportPlugin.obj
 0001:00004e50       ?qt_metacast@OpenCLSupportPlugin@U2@@UAEPAXPBD@Z 10005e50 f   moc_OpenCLSupportPlugin.obj
 0001:00004eb0       ?qt_static_metacall@OpenCLSupportPlugin@U2@@CAXPAVQObject@@W4Call@QMetaObject@@HPAPAX@Z 10005eb0 f   moc_OpenCLSupportPlugin.obj
 0001:00004ec0       ?metaObject@OpenCLSupportSettingsPageController@U2@@UBEPBUQMetaObject@@XZ 10005ec0 f   moc_OpenCLSupportSettingsController.obj
 0001:00004ee0       ?metaObject@OpenCLSupportSettingsPageState@U2@@UBEPBUQMetaObject@@XZ 10005ee0 f   moc_OpenCLSupportSettingsController.obj
 0001:00004f00       ?metaObject@OpenCLSupportSettingsPageWidget@U2@@UBEPBUQMetaObject@@XZ 10005f00 f   moc_OpenCLSupportSettingsController.obj
 0001:00004f20       ?qt_metacall@OpenCLSupportSettingsPageController@U2@@UAEHW4Call@QMetaObject@@HPAPAX@Z 10005f20 f   moc_OpenCLSupportSettingsController.obj
 0001:00004f30       ?qt_metacall@OpenCLSupportSettingsPageState@U2@@UAEHW4Call@QMetaObject@@HPAPAX@Z 10005f30 f   moc_OpenCLSupportSettingsController.obj
 0001:00004f40       ?qt_metacall@OpenCLSupportSettingsPageWidget@U2@@UAEHW4Call@QMetaObject@@HPAPAX@Z 10005f40 f   moc_OpenCLSupportSettingsController.obj
 0001:00004f50       ?qt_metacast@OpenCLSupportSettingsPageController@U2@@UAEPAXPBD@Z 10005f50 f   moc_OpenCLSupportSettingsController.obj
 0001:00004fb0       ?qt_metacast@OpenCLSupportSettingsPageState@U2@@UAEPAXPBD@Z 10005fb0 f   moc_OpenCLSupportSettingsController.obj
 0001:00005010       ?qt_metacast@OpenCLSupportSettingsPageWidget@U2@@UAEPAXPBD@Z 10006010 f   moc_OpenCLSupportSettingsController.obj
 0001:00005070       ?qt_static_metacall@OpenCLSupportSettingsPageController@U2@@CAXPAVQObject@@W4Call@QMetaObject@@HPAPAX@Z 10006070 f   moc_OpenCLSupportSettingsController.obj
 0001:00005080       ?qt_static_metacall@OpenCLSupportSettingsPageState@U2@@CAXPAVQObject@@W4Call@QMetaObject@@HPAPAX@Z 10006080 f   moc_OpenCLSupportSettingsController.obj
 0001:00005090       ?qt_static_metacall@OpenCLSupportSettingsPageWidget@U2@@CAXPAVQObject@@W4Call@QMetaObject@@HPAPAX@Z 10006090 f   moc_OpenCLSupportSettingsController.obj
 0001:00005092       ?getSettings@AppContext@U2@@SAPAVSettings@2@XZ 10006092 f   U2Core:U2Core.dll
 0001:00005098       ?getAppSettingsGUI@AppContext@U2@@SAPAVAppSettingsGUI@2@XZ 10006098 f   U2Core:U2Core.dll
 0001:0000509e       ?getMainWindow@AppContext@U2@@SAPAVMainWindow@2@XZ 1000609e f   U2Core:U2Core.dll
 0001:000050a4       ?getOpenCLGpuRegistry@AppContext@U2@@SAPAVOpenCLGpuRegistry@2@XZ 100060a4 f   U2Core:U2Core.dll
 0001:000050aa       ??0Logger@U2@@QAE@ABVQString@@@Z 100060aa f   U2Core:U2Core.dll
 0001:000050b0       ??1Logger@U2@@UAE@XZ       100060b0 f   U2Core:U2Core.dll
 0001:000050b6       ?details@Logger@U2@@QAEXABVQString@@@Z 100060b6 f   U2Core:U2Core.dll
 0001:000050bc       ?info@Logger@U2@@QAEXABVQString@@@Z 100060bc f   U2Core:U2Core.dll
 0001:000050c2       ??0AppResourceSemaphore@U2@@QAE@HHABVQString@@0@Z 100060c2 f   U2Core:U2Core.dll
 0001:000050c8       ??1AppResourceSemaphore@U2@@UAE@XZ 100060c8 f   U2Core:U2Core.dll
 0001:000050ce       ?registerResource@AppResourcePool@U2@@QAEXPAVAppResource@2@@Z 100060ce f   U2Core:U2Core.dll
 0001:000050d4       ?unregisterResource@AppResourcePool@U2@@QAEXH@Z 100060d4 f   U2Core:U2Core.dll
 0001:000050da       ?instance@AppResourcePool@U2@@SAPAV12@XZ 100060da f   U2Core:U2Core.dll
 0001:000050e0       ??0Plugin@U2@@QAE@ABVQString@@0_NW4PluginState@1@@Z 100060e0 f   U2Core:U2Core.dll
 0001:000050e6       ??1Plugin@U2@@UAE@XZ       100060e6 f   U2Core:U2Core.dll
 0001:000050ec       ?acquire@AppResourceSemaphore@U2@@UAEXHW4MemoryLockType@AppResource@2@@Z 100060ec f   U2Core:U2Core.dll
 0001:000050f2       ?available@AppResourceSemaphore@U2@@UBEHXZ 100060f2 f   U2Core:U2Core.dll
 0001:000050f8       ?release@AppResourceSemaphore@U2@@UAEXHW4MemoryLockType@AppResource@2@@Z 100060f8 f   U2Core:U2Core.dll
 0001:000050fe       ?tryAcquire@AppResourceSemaphore@U2@@UAE_NHHW4MemoryLockType@AppResource@2@@Z 100060fe f   U2Core:U2Core.dll
 0001:00005104       ?tryAcquire@AppResourceSemaphore@U2@@UAE_NHW4MemoryLockType@AppResource@2@@Z 10006104 f   U2Core:U2Core.dll
 0001:0000510a       ?setMaxUse@AppResourceSemaphore@U2@@QAEXH@Z 1000610a f   U2Core:U2Core.dll
 0001:00005110       ?getResource@AppResourcePool@U2@@QBEPAVAppResource@2@H@Z 10006110 f   U2Core:U2Core.dll
 0001:00005116       ?qt_metacast@Plugin@U2@@UAEPAXPBD@Z 10006116 f   U2Core:U2Core.dll
 0001:0000511c       ?qt_metacall@Plugin@U2@@UAEHW4Call@QMetaObject@@HPAPAX@Z 1000611c f   U2Core:U2Core.dll
 0001:00005122       ?getErrorString@OpenCLHelper@U2@@QBE?AVQString@@XZ 10006122 f   U2Algorithm:U2Algorithm.dll
 0001:00005128       ??0OpenCLHelper@U2@@QAE@XZ 10006128 f   U2Algorithm:U2Algorithm.dll
 0001:0000512e       ??1OpenCLHelper@U2@@QAE@XZ 1000612e f   U2Algorithm:U2Algorithm.dll
 0001:00005134       ??0OpenCLGpuModel@U2@@QAE@ABVQString@@ABJ1_K222III_N@Z 10006134 f   U2Algorithm:U2Algorithm.dll
 0001:0000513a       ?getName@OpenCLGpuModel@U2@@QBE?AVQString@@XZ 1000613a f   U2Algorithm:U2Algorithm.dll
 0001:00005140       ?registerOpenCLGpu@OpenCLGpuRegistry@U2@@QAEXPAVOpenCLGpuModel@2@@Z 10006140 f   U2Algorithm:U2Algorithm.dll
 0001:00005146       ?unregisterOpenCLGpu@OpenCLGpuRegistry@U2@@QAEXPAVOpenCLGpuModel@2@@Z 10006146 f   U2Algorithm:U2Algorithm.dll
 0001:0000514c       ?getRegisteredGpus@OpenCLGpuRegistry@U2@@QBE?AV?$QList@PAVOpenCLGpuModel@U2@@@@XZ 1000614c f   U2Algorithm:U2Algorithm.dll
 0001:00005152       ??1AppSettingsGUIPageState@U2@@UAE@XZ 10006152 f   U2Gui:U2Gui.dll
 0001:00005158       ??0AppSettingsGUIPageWidget@U2@@QAE@PAVQWidget@@@Z 10006158 f   U2Gui:U2Gui.dll
 0001:0000515e       ??1AppSettingsGUIPageWidget@U2@@UAE@XZ 1000615e f   U2Gui:U2Gui.dll
 0001:00005164       ??0AppSettingsGUIPageController@U2@@QAE@ABVQString@@0PAVQObject@@@Z 10006164 f   U2Gui:U2Gui.dll
 0001:0000516a       ??1AppSettingsGUIPageController@U2@@UAE@XZ 1000616a f   U2Gui:U2Gui.dll
 0001:00005170       ?qt_metacast@AppSettingsGUIPageState@U2@@UAEPAXPBD@Z 10006170 f   U2Gui:U2Gui.dll
 0001:00005176       ?qt_metacall@AppSettingsGUIPageState@U2@@UAEHW4Call@QMetaObject@@HPAPAX@Z 10006176 f   U2Gui:U2Gui.dll
 0001:0000517c       ?qt_metacast@AppSettingsGUIPageWidget@U2@@UAEPAXPBD@Z 1000617c f   U2Gui:U2Gui.dll
 0001:00005182       ?qt_metacall@AppSettingsGUIPageWidget@U2@@UAEHW4Call@QMetaObject@@HPAPAX@Z 10006182 f   U2Gui:U2Gui.dll
 0001:00005188       ?qt_metacast@AppSettingsGUIPageController@U2@@UAEPAXPBD@Z 10006188 f   U2Gui:U2Gui.dll
 0001:0000518e       ?qt_metacall@AppSettingsGUIPageController@U2@@UAEHW4Call@QMetaObject@@HPAPAX@Z 1000618e f   U2Gui:U2Gui.dll
 0001:00005194       ??0QSizePolicy@@QAE@W4Policy@0@0W4ControlType@0@@Z 10006194 f   Qt5Widgets:Qt5Widgets.dll
 0001:0000519a       ??1QWidget@@UAE@XZ         1000619a f   Qt5Widgets:Qt5Widgets.dll
 0001:000051a0       ?setSizePolicy@QWidget@@QAEXVQSizePolicy@@@Z 100061a0 f   Qt5Widgets:Qt5Widgets.dll
 0001:000051a6       ?setLayout@QWidget@@QAEXPAVQLayout@@@Z 100061a6 f   Qt5Widgets:Qt5Widgets.dll
 0001:000051ac       ??0QLabel@@QAE@ABVQString@@PAVQWidget@@V?$QFlags@W4WindowType@Qt@@@@@Z 100061ac f   Qt5Widgets:Qt5Widgets.dll
 0001:000051b2       ??1QLabel@@UAE@XZ          100061b2 f   Qt5Widgets:Qt5Widgets.dll
 0001:000051b8       ?setAlignment@QLabel@@QAEXV?$QFlags@W4AlignmentFlag@Qt@@@@@Z 100061b8 f   Qt5Widgets:Qt5Widgets.dll
 0001:000051be       ?setAlignment@QLayoutItem@@QAEXV?$QFlags@W4AlignmentFlag@Qt@@@@@Z 100061be f   Qt5Widgets:Qt5Widgets.dll
 0001:000051c4       ?addStretch@QBoxLayout@@QAEXH@Z 100061c4 f   Qt5Widgets:Qt5Widgets.dll
 0001:000051ca       ?addWidget@QBoxLayout@@QAEXPAVQWidget@@HV?$QFlags@W4AlignmentFlag@Qt@@@@@Z 100061ca f   Qt5Widgets:Qt5Widgets.dll
 0001:000051d0       ?addLayout@QBoxLayout@@QAEXPAVQLayout@@H@Z 100061d0 f   Qt5Widgets:Qt5Widgets.dll
 0001:000051d6       ??0QHBoxLayout@@QAE@PAVQWidget@@@Z 100061d6 f   Qt5Widgets:Qt5Widgets.dll
 0001:000051dc       ??1QHBoxLayout@@UAE@XZ     100061dc f   Qt5Widgets:Qt5Widgets.dll
 0001:000051e2       ??0QVBoxLayout@@QAE@PAVQWidget@@@Z 100061e2 f   Qt5Widgets:Qt5Widgets.dll
 0001:000051e8       ??1QVBoxLayout@@UAE@XZ     100061e8 f   Qt5Widgets:Qt5Widgets.dll
 0001:000051ee       ?isChecked@QAbstractButton@@QBE_NXZ 100061ee f   Qt5Widgets:Qt5Widgets.dll
 0001:000051f4       ?setChecked@QAbstractButton@@QAEX_N@Z 100061f4 f   Qt5Widgets:Qt5Widgets.dll
 0001:000051fa       ??0QCheckBox@@QAE@ABVQString@@PAVQWidget@@@Z 100061fa f   Qt5Widgets:Qt5Widgets.dll
 0001:00005200       ??1QCheckBox@@UAE@XZ       10006200 f   Qt5Widgets:Qt5Widgets.dll
 0001:00005206       ?actionEvent@QWidget@@MAEXPAVQActionEvent@@@Z 10006206 f   Qt5Widgets:Qt5Widgets.dll
 0001:0000520c       ?addItem@QBoxLayout@@UAEXPAVQLayoutItem@@@Z 1000620c f   Qt5Widgets:Qt5Widgets.dll
 0001:00005212       ?changeEvent@QAbstractButton@@MAEXPAVQEvent@@@Z 10006212 f   Qt5Widgets:Qt5Widgets.dll
 0001:00005218       ?changeEvent@QLabel@@MAEXPAVQEvent@@@Z 10006218 f   Qt5Widgets:Qt5Widgets.dll
 0001:0000521e       ?changeEvent@QWidget@@MAEXPAVQEvent@@@Z 1000621e f   Qt5Widgets:Qt5Widgets.dll
 0001:00005224       ?checkStateSet@QCheckBox@@MAEXXZ 10006224 f   Qt5Widgets:Qt5Widgets.dll
 0001:0000522a       ?childEvent@QLayout@@MAEXPAVQChildEvent@@@Z 1000622a f   Qt5Widgets:Qt5Widgets.dll
 0001:00005230       ?closeEvent@QWidget@@MAEXPAVQCloseEvent@@@Z 10006230 f   Qt5Widgets:Qt5Widgets.dll
 0001:00005236       ?contextMenuEvent@QLabel@@MAEXPAVQContextMenuEvent@@@Z 10006236 f   Qt5Widgets:Qt5Widgets.dll
 0001:0000523c       ?contextMenuEvent@QWidget@@MAEXPAVQContextMenuEvent@@@Z 1000623c f   Qt5Widgets:Qt5Widgets.dll
 0001:00005242       ?controlTypes@QLayout@@UBE?AV?$QFlags@W4ControlType@QSizePolicy@@@@XZ 10006242 f   Qt5Widgets:Qt5Widgets.dll
 0001:00005248       ?count@QBoxLayout@@UBEHXZ  10006248 f   Qt5Widgets:Qt5Widgets.dll
 0001:0000524e       ?devType@QWidget@@UBEHXZ   1000624e f   Qt5Widgets:Qt5Widgets.dll
 0001:00005254       ?dragEnterEvent@QWidget@@MAEXPAVQDragEnterEvent@@@Z 10006254 f   Qt5Widgets:Qt5Widgets.dll
 0001:0000525a       ?dragLeaveEvent@QWidget@@MAEXPAVQDragLeaveEvent@@@Z 1000625a f   Qt5Widgets:Qt5Widgets.dll
 0001:00005260       ?dragMoveEvent@QWidget@@MAEXPAVQDragMoveEvent@@@Z 10006260 f   Qt5Widgets:Qt5Widgets.dll
 0001:00005266       ?dropEvent@QWidget@@MAEXPAVQDropEvent@@@Z 10006266 f   Qt5Widgets:Qt5Widgets.dll
 0001:0000526c       ?enterEvent@QWidget@@MAEXPAVQEvent@@@Z 1000626c f   Qt5Widgets:Qt5Widgets.dll
 0001:00005272       ?event@QCheckBox@@MAE_NPAVQEvent@@@Z 10006272 f   Qt5Widgets:Qt5Widgets.dll
 0001:00005278       ?event@QLabel@@MAE_NPAVQEvent@@@Z 10006278 f   Qt5Widgets:Qt5Widgets.dll
 0001:0000527e       ?event@QWidget@@MAE_NPAVQEvent@@@Z 1000627e f   Qt5Widgets:Qt5Widgets.dll
 0001:00005284       ?expandingDirections@QBoxLayout@@UBE?AV?$QFlags@W4Orientation@Qt@@@@XZ 10006284 f   Qt5Widgets:Qt5Widgets.dll
 0001:0000528a       ?focusInEvent@QAbstractButton@@MAEXPAVQFocusEvent@@@Z 1000628a f   Qt5Widgets:Qt5Widgets.dll
 0001:00005290       ?focusInEvent@QLabel@@MAEXPAVQFocusEvent@@@Z 10006290 f   Qt5Widgets:Qt5Widgets.dll
 0001:00005296       ?focusInEvent@QWidget@@MAEXPAVQFocusEvent@@@Z 10006296 f   Qt5Widgets:Qt5Widgets.dll
 0001:0000529c       ?focusNextPrevChild@QLabel@@MAE_N_N@Z 1000629c f   Qt5Widgets:Qt5Widgets.dll
 0001:000052a2       ?focusNextPrevChild@QWidget@@MAE_N_N@Z 100062a2 f   Qt5Widgets:Qt5Widgets.dll
 0001:000052a8       ?focusOutEvent@QAbstractButton@@MAEXPAVQFocusEvent@@@Z 100062a8 f   Qt5Widgets:Qt5Widgets.dll
 0001:000052ae       ?focusOutEvent@QLabel@@MAEXPAVQFocusEvent@@@Z 100062ae f   Qt5Widgets:Qt5Widgets.dll
 0001:000052b4       ?focusOutEvent@QWidget@@MAEXPAVQFocusEvent@@@Z 100062b4 f   Qt5Widgets:Qt5Widgets.dll
 0001:000052ba       ?geometry@QLayout@@UBE?AVQRect@@XZ 100062ba f   Qt5Widgets:Qt5Widgets.dll
 0001:000052c0       ?hasHeightForWidth@QBoxLayout@@UBE_NXZ 100062c0 f   Qt5Widgets:Qt5Widgets.dll
 0001:000052c6       ?hasHeightForWidth@QWidget@@UBE_NXZ 100062c6 f   Qt5Widgets:Qt5Widgets.dll
 0001:000052cc       ?heightForWidth@QBoxLayout@@UBEHH@Z 100062cc f   Qt5Widgets:Qt5Widgets.dll
 0001:000052d2       ?heightForWidth@QLabel@@UBEHH@Z 100062d2 f   Qt5Widgets:Qt5Widgets.dll
 0001:000052d8       ?heightForWidth@QWidget@@UBEHH@Z 100062d8 f   Qt5Widgets:Qt5Widgets.dll
 0001:000052de       ?hideEvent@QWidget@@MAEXPAVQHideEvent@@@Z 100062de f   Qt5Widgets:Qt5Widgets.dll
 0001:000052e4       ?hitButton@QCheckBox@@MBE_NABVQPoint@@@Z 100062e4 f   Qt5Widgets:Qt5Widgets.dll
 0001:000052ea       ?indexOf@QLayout@@UBEHPAVQWidget@@@Z 100062ea f   Qt5Widgets:Qt5Widgets.dll
 0001:000052f0       ?initPainter@QWidget@@MBEXPAVQPainter@@@Z 100062f0 f   Qt5Widgets:Qt5Widgets.dll
 0001:000052f6       ?inputMethodEvent@QWidget@@MAEXPAVQInputMethodEvent@@@Z 100062f6 f   Qt5Widgets:Qt5Widgets.dll
 0001:000052fc       ?inputMethodQuery@QWidget@@UBE?AVQVariant@@W4InputMethodQuery@Qt@@@Z 100062fc f   Qt5Widgets:Qt5Widgets.dll
 0001:00005302       ?invalidate@QBoxLayout@@UAEXXZ 10006302 f   Qt5Widgets:Qt5Widgets.dll
 0001:00005308       ?isEmpty@QLayout@@UBE_NXZ  10006308 f   Qt5Widgets:Qt5Widgets.dll
 0001:0000530e       ?itemAt@QBoxLayout@@UBEPAVQLayoutItem@@H@Z 1000630e f   Qt5Widgets:Qt5Widgets.dll
 0001:00005314       ?keyPressEvent@QAbstractButton@@MAEXPAVQKeyEvent@@@Z 10006314 f   Qt5Widgets:Qt5Widgets.dll
 0001:0000531a       ?keyPressEvent@QLabel@@MAEXPAVQKeyEvent@@@Z 1000631a f   Qt5Widgets:Qt5Widgets.dll
 0001:00005320       ?keyPressEvent@QWidget@@MAEXPAVQKeyEvent@@@Z 10006320 f   Qt5Widgets:Qt5Widgets.dll
 0001:00005326       ?keyReleaseEvent@QAbstractButton@@MAEXPAVQKeyEvent@@@Z 10006326 f   Qt5Widgets:Qt5Widgets.dll
 0001:0000532c       ?keyReleaseEvent@QWidget@@MAEXPAVQKeyEvent@@@Z 1000632c f   Qt5Widgets:Qt5Widgets.dll
 0001:00005332       ?layout@QLayout@@UAEPAV1@XZ 10006332 f   Qt5Widgets:Qt5Widgets.dll
 0001:00005338       ?leaveEvent@QWidget@@MAEXPAVQEvent@@@Z 10006338 f   Qt5Widgets:Qt5Widgets.dll
 0001:0000533e       ?maximumSize@QBoxLayout@@UBE?AVQSize@@XZ 1000633e f   Qt5Widgets:Qt5Widgets.dll
 0001:00005344       ?metaObject@QCheckBox@@UBEPBUQMetaObject@@XZ 10006344 f   Qt5Widgets:Qt5Widgets.dll
 0001:0000534a       ?metaObject@QHBoxLayout@@UBEPBUQMetaObject@@XZ 1000634a f   Qt5Widgets:Qt5Widgets.dll
 0001:00005350       ?metaObject@QLabel@@UBEPBUQMetaObject@@XZ 10006350 f   Qt5Widgets:Qt5Widgets.dll
 0001:00005356       ?metaObject@QVBoxLayout@@UBEPBUQMetaObject@@XZ 10006356 f   Qt5Widgets:Qt5Widgets.dll
 0001:0000535c       ?metric@QWidget@@MBEHW4PaintDeviceMetric@QPaintDevice@@@Z 1000635c f   Qt5Widgets:Qt5Widgets.dll
 0001:00005362       ?minimumHeightForWidth@QBoxLayout@@UBEHH@Z 10006362 f   Qt5Widgets:Qt5Widgets.dll
 0001:00005368       ?minimumSize@QBoxLayout@@UBE?AVQSize@@XZ 10006368 f   Qt5Widgets:Qt5Widgets.dll
 0001:0000536e       ?minimumSizeHint@QCheckBox@@UBE?AVQSize@@XZ 1000636e f   Qt5Widgets:Qt5Widgets.dll
 0001:00005374       ?minimumSizeHint@QLabel@@UBE?AVQSize@@XZ 10006374 f   Qt5Widgets:Qt5Widgets.dll
 0001:0000537a       ?minimumSizeHint@QWidget@@UBE?AVQSize@@XZ 1000637a f   Qt5Widgets:Qt5Widgets.dll
 0001:00005380       ?mouseDoubleClickEvent@QWidget@@MAEXPAVQMouseEvent@@@Z 10006380 f   Qt5Widgets:Qt5Widgets.dll
 0001:00005386       ?mouseMoveEvent@QCheckBox@@MAEXPAVQMouseEvent@@@Z 10006386 f   Qt5Widgets:Qt5Widgets.dll
 0001:0000538c       ?mouseMoveEvent@QLabel@@MAEXPAVQMouseEvent@@@Z 1000638c f   Qt5Widgets:Qt5Widgets.dll
 0001:00005392       ?mouseMoveEvent@QWidget@@MAEXPAVQMouseEvent@@@Z 10006392 f   Qt5Widgets:Qt5Widgets.dll
 0001:00005398       ?mousePressEvent@QAbstractButton@@MAEXPAVQMouseEvent@@@Z 10006398 f   Qt5Widgets:Qt5Widgets.dll
 0001:0000539e       ?mousePressEvent@QLabel@@MAEXPAVQMouseEvent@@@Z 1000639e f   Qt5Widgets:Qt5Widgets.dll
 0001:000053a4       ?mousePressEvent@QWidget@@MAEXPAVQMouseEvent@@@Z 100063a4 f   Qt5Widgets:Qt5Widgets.dll
 0001:000053aa       ?mouseReleaseEvent@QAbstractButton@@MAEXPAVQMouseEvent@@@Z 100063aa f   Qt5Widgets:Qt5Widgets.dll
 0001:000053b0       ?mouseReleaseEvent@QLabel@@MAEXPAVQMouseEvent@@@Z 100063b0 f   Qt5Widgets:Qt5Widgets.dll
 0001:000053b6       ?mouseReleaseEvent@QWidget@@MAEXPAVQMouseEvent@@@Z 100063b6 f   Qt5Widgets:Qt5Widgets.dll
 0001:000053bc       ?moveEvent@QWidget@@MAEXPAVQMoveEvent@@@Z 100063bc f   Qt5Widgets:Qt5Widgets.dll
 0001:000053c2       ?nativeEvent@QWidget@@MAE_NABVQByteArray@@PAXPAJ@Z 100063c2 f   Qt5Widgets:Qt5Widgets.dll
 0001:000053c8       ?nextCheckState@QCheckBox@@MAEXXZ 100063c8 f   Qt5Widgets:Qt5Widgets.dll
 0001:000053ce       ?paintEngine@QWidget@@UBEPAVQPaintEngine@@XZ 100063ce f   Qt5Widgets:Qt5Widgets.dll
 0001:000053d4       ?paintEvent@QCheckBox@@MAEXPAVQPaintEvent@@@Z 100063d4 f   Qt5Widgets:Qt5Widgets.dll
 0001:000053da       ?paintEvent@QLabel@@MAEXPAVQPaintEvent@@@Z 100063da f   Qt5Widgets:Qt5Widgets.dll
 0001:000053e0       ?paintEvent@QWidget@@MAEXPAVQPaintEvent@@@Z 100063e0 f   Qt5Widgets:Qt5Widgets.dll
 0001:000053e6       ?qt_metacall@QCheckBox@@UAEHW4Call@QMetaObject@@HPAPAX@Z 100063e6 f   Qt5Widgets:Qt5Widgets.dll
 0001:000053ec       ?qt_metacall@QHBoxLayout@@UAEHW4Call@QMetaObject@@HPAPAX@Z 100063ec f   Qt5Widgets:Qt5Widgets.dll
 0001:000053f2       ?qt_metacall@QLabel@@UAEHW4Call@QMetaObject@@HPAPAX@Z 100063f2 f   Qt5Widgets:Qt5Widgets.dll
 0001:000053f8       ?qt_metacall@QVBoxLayout@@UAEHW4Call@QMetaObject@@HPAPAX@Z 100063f8 f   Qt5Widgets:Qt5Widgets.dll
 0001:000053fe       ?qt_metacast@QCheckBox@@UAEPAXPBD@Z 100063fe f   Qt5Widgets:Qt5Widgets.dll
 0001:00005404       ?qt_metacast@QHBoxLayout@@UAEPAXPBD@Z 10006404 f   Qt5Widgets:Qt5Widgets.dll
 0001:0000540a       ?qt_metacast@QLabel@@UAEPAXPBD@Z 1000640a f   Qt5Widgets:Qt5Widgets.dll
 0001:00005410       ?qt_metacast@QVBoxLayout@@UAEPAXPBD@Z 10006410 f   Qt5Widgets:Qt5Widgets.dll
 0001:00005416       ?redirected@QWidget@@MBEPAVQPaintDevice@@PAVQPoint@@@Z 10006416 f   Qt5Widgets:Qt5Widgets.dll
 0001:0000541c       ?resizeEvent@QWidget@@MAEXPAVQResizeEvent@@@Z 1000641c f   Qt5Widgets:Qt5Widgets.dll
 0001:00005422       ?setGeometry@QBoxLayout@@UAEXABVQRect@@@Z 10006422 f   Qt5Widgets:Qt5Widgets.dll
 0001:00005428       ?setVisible@QWidget@@UAEX_N@Z 10006428 f   Qt5Widgets:Qt5Widgets.dll
 0001:0000542e       ?sharedPainter@QWidget@@MBEPAVQPainter@@XZ 1000642e f   Qt5Widgets:Qt5Widgets.dll
 0001:00005434       ?showEvent@QWidget@@MAEXPAVQShowEvent@@@Z 10006434 f   Qt5Widgets:Qt5Widgets.dll
 0001:0000543a       ?sizeHint@QBoxLayout@@UBE?AVQSize@@XZ 1000643a f   Qt5Widgets:Qt5Widgets.dll
 0001:00005440       ?sizeHint@QCheckBox@@UBE?AVQSize@@XZ 10006440 f   Qt5Widgets:Qt5Widgets.dll
 0001:00005446       ?sizeHint@QLabel@@UBE?AVQSize@@XZ 10006446 f   Qt5Widgets:Qt5Widgets.dll
 0001:0000544c       ?sizeHint@QWidget@@UBE?AVQSize@@XZ 1000644c f   Qt5Widgets:Qt5Widgets.dll
 0001:00005452       ?spacerItem@QLayoutItem@@UAEPAVQSpacerItem@@XZ 10006452 f   Qt5Widgets:Qt5Widgets.dll
 0001:00005458       ?tabletEvent@QWidget@@MAEXPAVQTabletEvent@@@Z 10006458 f   Qt5Widgets:Qt5Widgets.dll
 0001:0000545e       ?takeAt@QBoxLayout@@UAEPAVQLayoutItem@@H@Z 1000645e f   Qt5Widgets:Qt5Widgets.dll
 0001:00005464       ?timerEvent@QAbstractButton@@MAEXPAVQTimerEvent@@@Z 10006464 f   Qt5Widgets:Qt5Widgets.dll
 0001:0000546a       ?wheelEvent@QWidget@@MAEXPAVQWheelEvent@@@Z 1000646a f   Qt5Widgets:Qt5Widgets.dll
 0001:00005470       ?widget@QLayoutItem@@UAEPAVQWidget@@XZ 10006470 f   Qt5Widgets:Qt5Widgets.dll
 0001:00005476       ?tr@QMetaObject@@QBE?AVQString@@PBD0H@Z 10006476 f   Qt5Core:Qt5Core.dll
 0001:0000547c       ??0QChar@@QAE@UQLatin1Char@@@Z 1000647c f   Qt5Core:Qt5Core.dll
 0001:00005482       ??0QString@@QAE@XZ         10006482 f   Qt5Core:Qt5Core.dll
 0001:00005488       ??0QString@@QAE@ABV0@@Z    10006488 f   Qt5Core:Qt5Core.dll
 0001:0000548e       ??1QString@@QAE@XZ         1000648e f   Qt5Core:Qt5Core.dll
 0001:00005494       ??4QString@@QAEAAV0@$$QAV0@@Z 10006494 f   Qt5Core:Qt5Core.dll
 0001:0000549a       ?arg@QString@@QBE?AV1@_KHHVQChar@@@Z 1000649a f   Qt5Core:Qt5Core.dll
 0001:000054a0       ?arg@QString@@QBE?AV1@HHHVQChar@@@Z 100064a0 f   Qt5Core:Qt5Core.dll
 0001:000054a6       ?arg@QString@@QBE?AV1@IHHVQChar@@@Z 100064a6 f   Qt5Core:Qt5Core.dll
 0001:000054ac       ?arg@QString@@QBE?AV1@ABV1@HVQChar@@@Z 100064ac f   Qt5Core:Qt5Core.dll
 0001:000054b2       ?append@QString@@QAEAAV1@ABV1@@Z 100064b2 f   Qt5Core:Qt5Core.dll
 0001:000054b8       ?fromUtf8@QString@@SA?AV1@PBDH@Z 100064b8 f   Qt5Core:Qt5Core.dll
 0001:000054be       ?number@QString@@SA?AV1@JH@Z 100064be f   Qt5Core:Qt5Core.dll
 0001:000054c4       ??4QString@@QAEAAV0@PBD@Z  100064c4 f   Qt5Core:Qt5Core.dll
 0001:000054ca       ?fromAscii_helper@QString@@CAPAU?$QTypedArrayData@G@@PBDH@Z 100064ca f   Qt5Core:Qt5Core.dll
 0001:000054d0       ?detach@QListData@@QAEPAUData@1@H@Z 100064d0 f   Qt5Core:Qt5Core.dll
 0001:000054d6       ?detach_grow@QListData@@QAEPAUData@1@PAHH@Z 100064d6 f   Qt5Core:Qt5Core.dll
 0001:000054dc       ?dispose@QListData@@SAXPAUData@1@@Z 100064dc f   Qt5Core:Qt5Core.dll
 0001:000054e2       ?append@QListData@@QAEPAPAXXZ 100064e2 f   Qt5Core:Qt5Core.dll
 0001:000054e8       ??0QVariant@@QAE@XZ        100064e8 f   Qt5Core:Qt5Core.dll
 0001:000054ee       ??1QVariant@@QAE@XZ        100064ee f   Qt5Core:Qt5Core.dll
 0001:000054f4       ?isNull@QVariant@@QBE_NXZ  100064f4 f   Qt5Core:Qt5Core.dll
 0001:000054fa       ?toBool@QVariant@@QBE_NXZ  100064fa f   Qt5Core:Qt5Core.dll
 0001:00005500       ?childEvent@QObject@@MAEXPAVQChildEvent@@@Z 10006500 f   Qt5Core:Qt5Core.dll
 0001:00005506       ?connectNotify@QObject@@MAEXABVQMetaMethod@@@Z 10006506 f   Qt5Core:Qt5Core.dll
 0001:0000550c       ?customEvent@QObject@@MAEXPAVQEvent@@@Z 1000650c f   Qt5Core:Qt5Core.dll
 0001:00005512       ?disconnectNotify@QObject@@MAEXABVQMetaMethod@@@Z 10006512 f   Qt5Core:Qt5Core.dll
 0001:00005518       ?event@QObject@@UAE_NPAVQEvent@@@Z 10006518 f   Qt5Core:Qt5Core.dll
 0001:0000551e       ?eventFilter@QObject@@UAE_NPAV1@PAVQEvent@@@Z 1000651e f   Qt5Core:Qt5Core.dll
 0001:00005524       ?timerEvent@QObject@@MAEXPAVQTimerEvent@@@Z 10006524 f   Qt5Core:Qt5Core.dll
 0001:0000552a       ?qBadAlloc@@YAXXZ          1000652a f   Qt5Core:Qt5Core.dll
 0001:00005530       ?cast@QMetaObject@@QBEPAVQObject@@PAV2@@Z 10006530 f   Qt5Core:Qt5Core.dll
 0001:00005536       ?data@QArrayData@@QAEPAXXZ 10006536 f   Qt5Core:Qt5Core.dll
 0001:0000553c       ?allocate@QArrayData@@SAPAU1@IIIV?$QFlags@W4AllocationOption@QArrayData@@@@@Z 1000653c f   Qt5Core:Qt5Core.dll
 0001:00005542       ?deallocate@QArrayData@@SAXPAU1@II@Z 10006542 f   Qt5Core:Qt5Core.dll
 0001:00005548       ?number@QString@@SA?AV1@_KH@Z 10006548 f   Qt5Core:Qt5Core.dll
 0001:0000554e       ??0QObject@@QAE@PAV0@@Z    1000654e f   Qt5Core:Qt5Core.dll
 0001:00005554       ??1QObject@@UAE@XZ         10006554 f   Qt5Core:Qt5Core.dll
 0001:0000555a       ?dynamicMetaObject@QObjectData@@QBEPAUQMetaObject@@XZ 1000655a f   Qt5Core:Qt5Core.dll
 0001:00005560       ??_U@YAPAXI@Z              10006560 f   msvcprt:newaop_s.obj
 0001:0000556a       ?_Xbad_alloc@std@@YAXXZ    1000656a f   msvcprt:MSVCP120.dll
 0001:00005570       ?_Xlength_error@std@@YAXPBD@Z 10006570 f   msvcprt:MSVCP120.dll
 0001:00005576       ?_Xout_of_range@std@@YAXPBD@Z 10006576 f   msvcprt:MSVCP120.dll
 0001:0000557c       ?_Syserror_map@std@@YAPBDH@Z 1000657c f   msvcprt:MSVCP120.dll
 0001:00005582       ?_Winerror_map@std@@YAPBDH@Z 10006582 f   msvcprt:MSVCP120.dll
 0001:00005588       __purecall                 10006588 f   MSVCRT:MSVCR120.dll
 0001:0000558e       ??2@YAPAXI@Z               1000658e f   MSVCRT:MSVCR120.dll
 0001:00005594       ??3@YAXPAX@Z               10006594 f   MSVCRT:MSVCR120.dll
 0001:0000559a       ___atonexitinit            1000659a f   MSVCRT:atonexit.obj
 0001:000055d6       __onexit                   100065d6 f   MSVCRT:atonexit.obj
 0001:0000567f       _atexit                    1000667f f   MSVCRT:atonexit.obj
 0001:00005694       _memmove                   10006694 f   MSVCRT:MSVCR120.dll
 0001:0000569a       _strncpy                   1000669a f   MSVCRT:MSVCR120.dll
 0001:000056a0       ??_V@YAXPAX@Z              100066a0 f   MSVCRT:MSVCR120.dll
 0001:000056a6       __hypot                    100066a6 f   MSVCRT:MSVCR120.dll
 0001:000056ac       @__security_check_cookie@4 100066ac f   MSVCRT:secchk.obj
 0001:000056bc       __CxxThrowException@8      100066bc f   MSVCRT:MSVCR120.dll
 0001:000056c2       ___CxxFrameHandler3        100066c2 f   MSVCRT:MSVCR120.dll
 0001:000056c8       _memcpy                    100066c8 f   MSVCRT:MSVCR120.dll
 0001:000056ce       ??0type_info@@AAE@ABV0@@Z  100066ce f   MSVCRT:ti_inst.obj
 0001:000056d9       ??4type_info@@AAEAAV0@ABV0@@Z 100066d9 f   MSVCRT:ti_inst.obj
 0001:000056de       ??_Etype_info@@UAEPAXI@Z   100066de f i MSVCRT:ti_inst.obj
 0001:00005730       ___RTDynamicCast           10006730 f   MSVCRT:MSVCR120.dll
 0001:00005736       _memset                    10006736 f   MSVCRT:MSVCR120.dll
 0001:00005788       _NtCurrentTeb              10006788 f i MSVCRT:crtdll.obj
 0001:0000578f       __CRT_INIT@12              1000678f f   MSVCRT:crtdll.obj
 0001:00005986       __DllMainCRTStartup@12     10006986 f   MSVCRT:crtdll.obj
 0001:00005adc       __lock                     10006adc f   MSVCRT:MSVCR120.dll
 0001:00005ae2       __unlock                   10006ae2 f   MSVCRT:MSVCR120.dll
 0001:00005ae8       __calloc_crt               10006ae8 f   MSVCRT:MSVCR120.dll
 0001:00005aee       ___dllonexit               10006aee f   MSVCRT:MSVCR120.dll
 0001:00005b00       __SEH_prolog4              10006b00 f   MSVCRT:sehprolg4.obj
 0001:00005b45       __SEH_epilog4              10006b45 f   MSVCRT:sehprolg4.obj
 0001:00005b59       __except_handler4          10006b59 f   MSVCRT:chandler4gs.obj
 0001:00005b7c       ___raise_securityfailure   10006b7c f   MSVCRT:gs_report.obj
 0001:00005bb9       ___report_gsfailure        10006bb9 f   MSVCRT:gs_report.obj
 0001:00005cb4       ___report_rangecheckfailure 10006cb4 f   MSVCRT:gs_report.obj
 0001:00005cc0       ___report_securityfailure  10006cc0 f   MSVCRT:gs_report.obj
 0001:00005d90       ___report_securityfailureEx 10006d90 f   MSVCRT:gs_report.obj
 0001:00005ea6       ??_M@YGXPAXIHP6EX0@Z@Z     10006ea6 f   MSVCRT:ehvecdtr.obj
 0001:00005f2e       ?__ArrayUnwind@@YGXPAXIHP6EX0@Z@Z 10006f2e f   MSVCRT:ehvecdtr.obj
 0001:00005f8c       ??1type_info@@UAE@XZ       10006f8c f   MSVCRT:MSVCR120.dll
 0001:00005f92       ___CppXcptFilter           10006f92 f   MSVCRT:MSVCR120.dll
 0001:00005f98       __amsg_exit                10006f98 f   MSVCRT:MSVCR120.dll
 0001:00005fa0       __FindPESection            10006fa0 f   MSVCRT:pesect.obj
 0001:00005ff0       __IsNonwritableInCurrentImage 10006ff0 f   MSVCRT:pesect.obj
 0001:000060b0       __ValidateImageBase        100070b0 f   MSVCRT:pesect.obj
 0001:000060e2       _free                      100070e2 f   MSVCRT:MSVCR120.dll
 0001:000060e8       ___security_init_cookie    100070e8 f   MSVCRT:gs_support.obj
 0001:00006184       _DllMain@12                10007184 f   MSVCRT:dllmain.obj
 0001:000061a6       __malloc_crt               100071a6 f   MSVCRT:MSVCR120.dll
 0001:000061ac       __RTC_Initialize           100071ac f   MSVCRT:initsect.obj
 0001:000061cc       __RTC_Terminate            100071cc f   MSVCRT:initsect.obj
 0001:000061ec       __initterm                 100071ec f   MSVCRT:MSVCR120.dll
 0001:000061f2       __initterm_e               100071f2 f   MSVCRT:MSVCR120.dll
 0001:000061f8       ___clean_type_info_names   100071f8 f   MSVCRT:tncleanup.obj
 0001:00006204       __except_handler4_common   10007204 f   MSVCRT:MSVCR120.dll
 0001:0000620a       __crt_debugger_hook        1000720a f   MSVCRT:MSVCR120.dll
 0001:00006210       ___crtUnhandledException   10007210 f   MSVCRT:MSVCR120.dll
 0001:00006216       ___crtTerminateProcess     10007216 f   MSVCRT:MSVCR120.dll
 0001:0000621c       ?terminate@@YAXXZ          1000721c f   MSVCRT:MSVCR120.dll
 0001:00006222       ___clean_type_info_names_internal 10007222 f   MSVCRT:MSVCR120.dll
 0001:00006228       _EncodePointer@4           10007228 f   kernel32:KERNEL32.dll
 0001:0000622e       _DecodePointer@4           1000722e f   kernel32:KERNEL32.dll
 0001:00006234       _IsDebuggerPresent@0       10007234 f   kernel32:KERNEL32.dll
 0001:0000623a       _IsProcessorFeaturePresent@4 1000723a f   kernel32:KERNEL32.dll
 0001:00006240       _QueryPerformanceCounter@4 10007240 f   kernel32:KERNEL32.dll
 0001:00006246       _GetCurrentProcessId@0     10007246 f   kernel32:KERNEL32.dll
 0001:0000624c       _GetCurrentThreadId@0      1000724c f   kernel32:KERNEL32.dll
 0001:00006252       _GetSystemTimeAsFileTime@4 10007252 f   kernel32:KERNEL32.dll
 0001:00006258       _DisableThreadLibraryCalls@4 10007258 f   kernel32:KERNEL32.dll
 0002:00000000       __imp__DisableThreadLibraryCalls@4 10008000     kernel32:KERNEL32.dll
 0002:00000004       __imp__GetSystemTimeAsFileTime@4 10008004     kernel32:KERNEL32.dll
 0002:00000008       __imp__GetCurrentThreadId@0 10008008     kernel32:KERNEL32.dll
 0002:0000000c       __imp__GetCurrentProcessId@0 1000800c     kernel32:KERNEL32.dll
 0002:00000010       __imp__QueryPerformanceCounter@4 10008010     kernel32:KERNEL32.dll
 0002:00000014       __imp__IsProcessorFeaturePresent@4 10008014     kernel32:KERNEL32.dll
 0002:00000018       __imp__IsDebuggerPresent@0 10008018     kernel32:KERNEL32.dll
 0002:0000001c       __imp__DecodePointer@4     1000801c     kernel32:KERNEL32.dll
 0002:00000020       __imp__EncodePointer@4     10008020     kernel32:KERNEL32.dll
 0002:00000024       \177KERNEL32_NULL_THUNK_DATA 10008024     kernel32:KERNEL32.dll
 0002:00000028       __imp_?_Xlength_error@std@@YAXPBD@Z 10008028     msvcprt:MSVCP120.dll
 0002:0000002c       __imp_?_Xout_of_range@std@@YAXPBD@Z 1000802c     msvcprt:MSVCP120.dll
 0002:00000030       __imp_?_Syserror_map@std@@YAPBDH@Z 10008030     msvcprt:MSVCP120.dll
 0002:00000034       __imp_?_Winerror_map@std@@YAPBDH@Z 10008034     msvcprt:MSVCP120.dll
 0002:00000038       __imp_?_Xbad_alloc@std@@YAXXZ 10008038     msvcprt:MSVCP120.dll
 0002:0000003c       \177MSVCP120_NULL_THUNK_DATA 1000803c     msvcprt:MSVCP120.dll
 0002:00000040       __imp___initterm_e         10008040     MSVCRT:MSVCR120.dll
 0002:00000044       __imp___initterm           10008044     MSVCRT:MSVCR120.dll
 0002:00000048       __imp___malloc_crt         10008048     MSVCRT:MSVCR120.dll
 0002:0000004c       __imp__free                1000804c     MSVCRT:MSVCR120.dll
 0002:00000050       __imp___amsg_exit          10008050     MSVCRT:MSVCR120.dll
 0002:00000054       __imp____CppXcptFilter     10008054     MSVCRT:MSVCR120.dll
 0002:00000058       __imp___except_handler4_common 10008058     MSVCRT:MSVCR120.dll
 0002:0000005c       __imp___onexit             1000805c     MSVCRT:MSVCR120.dll
 0002:00000060       __imp____dllonexit         10008060     MSVCRT:MSVCR120.dll
 0002:00000064       __imp___calloc_crt         10008064     MSVCRT:MSVCR120.dll
 0002:00000068       __imp___unlock             10008068     MSVCRT:MSVCR120.dll
 0002:0000006c       __imp___lock               1000806c     MSVCRT:MSVCR120.dll
 0002:00000070       __imp__memset              10008070     MSVCRT:MSVCR120.dll
 0002:00000074       __imp____RTDynamicCast     10008074     MSVCRT:MSVCR120.dll
 0002:00000078       __imp__memcpy              10008078     MSVCRT:MSVCR120.dll
 0002:0000007c       __imp____CxxFrameHandler3  1000807c     MSVCRT:MSVCR120.dll
 0002:00000080       __imp___CxxThrowException@8 10008080     MSVCRT:MSVCR120.dll
 0002:00000084       __imp___hypot              10008084     MSVCRT:MSVCR120.dll
 0002:00000088       __imp_??_V@YAXPAX@Z        10008088     MSVCRT:MSVCR120.dll
 0002:0000008c       __imp__strncpy             1000808c     MSVCRT:MSVCR120.dll
 0002:00000090       __imp__memmove             10008090     MSVCRT:MSVCR120.dll
 0002:00000094       __imp_??3@YAXPAX@Z         10008094     MSVCRT:MSVCR120.dll
 0002:00000098       __imp_??2@YAPAXI@Z         10008098     MSVCRT:MSVCR120.dll
 0002:0000009c       __imp___purecall           1000809c     MSVCRT:MSVCR120.dll
 0002:000000a0       __imp___crt_debugger_hook  100080a0     MSVCRT:MSVCR120.dll
 0002:000000a4       __imp____crtUnhandledException 100080a4     MSVCRT:MSVCR120.dll
 0002:000000a8       __imp____crtTerminateProcess 100080a8     MSVCRT:MSVCR120.dll
 0002:000000ac       __imp_?terminate@@YAXXZ    100080ac     MSVCRT:MSVCR120.dll
 0002:000000b0       __imp____clean_type_info_names_internal 100080b0     MSVCRT:MSVCR120.dll
 0002:000000b4       __imp_??1type_info@@UAE@XZ 100080b4     MSVCRT:MSVCR120.dll
 0002:000000b8       \177MSVCR120_NULL_THUNK_DATA 100080b8     MSVCRT:MSVCR120.dll
 0002:000000bc       __imp_?dynamicMetaObject@QObjectData@@QBEPAUQMetaObject@@XZ 100080bc     Qt5Core:Qt5Core.dll
 0002:000000c0       __imp_?shared_null@QArrayData@@2QBU1@B 100080c0     Qt5Core:Qt5Core.dll
 0002:000000c4       __imp_??0QObject@@QAE@PAV0@@Z 100080c4     Qt5Core:Qt5Core.dll
 0002:000000c8       __imp_?number@QString@@SA?AV1@_KH@Z 100080c8     Qt5Core:Qt5Core.dll
 0002:000000cc       __imp_?deallocate@QArrayData@@SAXPAU1@II@Z 100080cc     Qt5Core:Qt5Core.dll
 0002:000000d0       __imp_?allocate@QArrayData@@SAPAU1@IIIV?$QFlags@W4AllocationOption@QArrayData@@@@@Z 100080d0     Qt5Core:Qt5Core.dll
 0002:000000d4       __imp_?data@QArrayData@@QAEPAXXZ 100080d4     Qt5Core:Qt5Core.dll
 0002:000000d8       __imp_?cast@QMetaObject@@QBEPAVQObject@@PAV2@@Z 100080d8     Qt5Core:Qt5Core.dll
 0002:000000dc       __imp_?qBadAlloc@@YAXXZ    100080dc     Qt5Core:Qt5Core.dll
 0002:000000e0       __imp_?shared_null@QListData@@2UData@1@B 100080e0     Qt5Core:Qt5Core.dll
 0002:000000e4       __imp_?timerEvent@QObject@@MAEXPAVQTimerEvent@@@Z 100080e4     Qt5Core:Qt5Core.dll
 0002:000000e8       __imp_?eventFilter@QObject@@UAE_NPAV1@PAVQEvent@@@Z 100080e8     Qt5Core:Qt5Core.dll
 0002:000000ec       __imp_?event@QObject@@UAE_NPAVQEvent@@@Z 100080ec     Qt5Core:Qt5Core.dll
 0002:000000f0       __imp_?disconnectNotify@QObject@@MAEXABVQMetaMethod@@@Z 100080f0     Qt5Core:Qt5Core.dll
 0002:000000f4       __imp_?customEvent@QObject@@MAEXPAVQEvent@@@Z 100080f4     Qt5Core:Qt5Core.dll
 0002:000000f8       __imp_?connectNotify@QObject@@MAEXABVQMetaMethod@@@Z 100080f8     Qt5Core:Qt5Core.dll
 0002:000000fc       __imp_?childEvent@QObject@@MAEXPAVQChildEvent@@@Z 100080fc     Qt5Core:Qt5Core.dll
 0002:00000100       __imp_?toBool@QVariant@@QBE_NXZ 10008100     Qt5Core:Qt5Core.dll
 0002:00000104       __imp_?isNull@QVariant@@QBE_NXZ 10008104     Qt5Core:Qt5Core.dll
 0002:00000108       __imp_??1QVariant@@QAE@XZ  10008108     Qt5Core:Qt5Core.dll
 0002:0000010c       __imp_??0QVariant@@QAE@XZ  1000810c     Qt5Core:Qt5Core.dll
 0002:00000110       __imp_?append@QListData@@QAEPAPAXXZ 10008110     Qt5Core:Qt5Core.dll
 0002:00000114       __imp_?dispose@QListData@@SAXPAUData@1@@Z 10008114     Qt5Core:Qt5Core.dll
 0002:00000118       __imp_?detach_grow@QListData@@QAEPAUData@1@PAHH@Z 10008118     Qt5Core:Qt5Core.dll
 0002:0000011c       __imp_?detach@QListData@@QAEPAUData@1@H@Z 1000811c     Qt5Core:Qt5Core.dll
 0002:00000120       __imp_?fromAscii_helper@QString@@CAPAU?$QTypedArrayData@G@@PBDH@Z 10008120     Qt5Core:Qt5Core.dll
 0002:00000124       __imp_??4QString@@QAEAAV0@PBD@Z 10008124     Qt5Core:Qt5Core.dll
 0002:00000128       __imp_?number@QString@@SA?AV1@JH@Z 10008128     Qt5Core:Qt5Core.dll
 0002:0000012c       __imp_?fromUtf8@QString@@SA?AV1@PBDH@Z 1000812c     Qt5Core:Qt5Core.dll
 0002:00000130       __imp_?append@QString@@QAEAAV1@ABV1@@Z 10008130     Qt5Core:Qt5Core.dll
 0002:00000134       __imp_?arg@QString@@QBE?AV1@ABV1@HVQChar@@@Z 10008134     Qt5Core:Qt5Core.dll
 0002:00000138       __imp_?arg@QString@@QBE?AV1@IHHVQChar@@@Z 10008138     Qt5Core:Qt5Core.dll
 0002:0000013c       __imp_?arg@QString@@QBE?AV1@HHHVQChar@@@Z 1000813c     Qt5Core:Qt5Core.dll
 0002:00000140       __imp_?arg@QString@@QBE?AV1@_KHHVQChar@@@Z 10008140     Qt5Core:Qt5Core.dll
 0002:00000144       __imp_??4QString@@QAEAAV0@$$QAV0@@Z 10008144     Qt5Core:Qt5Core.dll
 0002:00000148       __imp_??1QString@@QAE@XZ   10008148     Qt5Core:Qt5Core.dll
 0002:0000014c       __imp_??0QString@@QAE@ABV0@@Z 1000814c     Qt5Core:Qt5Core.dll
 0002:00000150       __imp_??0QString@@QAE@XZ   10008150     Qt5Core:Qt5Core.dll
 0002:00000154       __imp_??0QChar@@QAE@UQLatin1Char@@@Z 10008154     Qt5Core:Qt5Core.dll
 0002:00000158       __imp_?tr@QMetaObject@@QBE?AVQString@@PBD0H@Z 10008158     Qt5Core:Qt5Core.dll
 0002:0000015c       __imp_??1QObject@@UAE@XZ   1000815c     Qt5Core:Qt5Core.dll
 0002:00000160       \177Qt5Core_NULL_THUNK_DATA 10008160     Qt5Core:Qt5Core.dll
 0002:00000164       __imp_?event@QWidget@@MAE_NPAVQEvent@@@Z 10008164     Qt5Widgets:Qt5Widgets.dll
 0002:00000168       __imp_?expandingDirections@QBoxLayout@@UBE?AV?$QFlags@W4Orientation@Qt@@@@XZ 10008168     Qt5Widgets:Qt5Widgets.dll
 0002:0000016c       __imp_?focusInEvent@QAbstractButton@@MAEXPAVQFocusEvent@@@Z 1000816c     Qt5Widgets:Qt5Widgets.dll
 0002:00000170       __imp_?focusInEvent@QLabel@@MAEXPAVQFocusEvent@@@Z 10008170     Qt5Widgets:Qt5Widgets.dll
 0002:00000174       __imp_?focusInEvent@QWidget@@MAEXPAVQFocusEvent@@@Z 10008174     Qt5Widgets:Qt5Widgets.dll
 0002:00000178       __imp_?focusNextPrevChild@QLabel@@MAE_N_N@Z 10008178     Qt5Widgets:Qt5Widgets.dll
 0002:0000017c       __imp_?focusNextPrevChild@QWidget@@MAE_N_N@Z 1000817c     Qt5Widgets:Qt5Widgets.dll
 0002:00000180       __imp_?focusOutEvent@QAbstractButton@@MAEXPAVQFocusEvent@@@Z 10008180     Qt5Widgets:Qt5Widgets.dll
 0002:00000184       __imp_?focusOutEvent@QLabel@@MAEXPAVQFocusEvent@@@Z 10008184     Qt5Widgets:Qt5Widgets.dll
 0002:00000188       __imp_?focusOutEvent@QWidget@@MAEXPAVQFocusEvent@@@Z 10008188     Qt5Widgets:Qt5Widgets.dll
 0002:0000018c       __imp_?geometry@QLayout@@UBE?AVQRect@@XZ 1000818c     Qt5Widgets:Qt5Widgets.dll
 0002:00000190       __imp_?hasHeightForWidth@QBoxLayout@@UBE_NXZ 10008190     Qt5Widgets:Qt5Widgets.dll
 0002:00000194       __imp_?hasHeightForWidth@QWidget@@UBE_NXZ 10008194     Qt5Widgets:Qt5Widgets.dll
 0002:00000198       __imp_?heightForWidth@QBoxLayout@@UBEHH@Z 10008198     Qt5Widgets:Qt5Widgets.dll
 0002:0000019c       __imp_?heightForWidth@QLabel@@UBEHH@Z 1000819c     Qt5Widgets:Qt5Widgets.dll
 0002:000001a0       __imp_?heightForWidth@QWidget@@UBEHH@Z 100081a0     Qt5Widgets:Qt5Widgets.dll
 0002:000001a4       __imp_?hideEvent@QWidget@@MAEXPAVQHideEvent@@@Z 100081a4     Qt5Widgets:Qt5Widgets.dll
 0002:000001a8       __imp_?event@QLabel@@MAE_NPAVQEvent@@@Z 100081a8     Qt5Widgets:Qt5Widgets.dll
 0002:000001ac       __imp_?indexOf@QLayout@@UBEHPAVQWidget@@@Z 100081ac     Qt5Widgets:Qt5Widgets.dll
 0002:000001b0       __imp_?initPainter@QWidget@@MBEXPAVQPainter@@@Z 100081b0     Qt5Widgets:Qt5Widgets.dll
 0002:000001b4       __imp_?inputMethodEvent@QWidget@@MAEXPAVQInputMethodEvent@@@Z 100081b4     Qt5Widgets:Qt5Widgets.dll
 0002:000001b8       __imp_?inputMethodQuery@QWidget@@UBE?AVQVariant@@W4InputMethodQuery@Qt@@@Z 100081b8     Qt5Widgets:Qt5Widgets.dll
 0002:000001bc       __imp_?invalidate@QBoxLayout@@UAEXXZ 100081bc     Qt5Widgets:Qt5Widgets.dll
 0002:000001c0       __imp_?isEmpty@QLayout@@UBE_NXZ 100081c0     Qt5Widgets:Qt5Widgets.dll
 0002:000001c4       __imp_?itemAt@QBoxLayout@@UBEPAVQLayoutItem@@H@Z 100081c4     Qt5Widgets:Qt5Widgets.dll
 0002:000001c8       __imp_?keyPressEvent@QAbstractButton@@MAEXPAVQKeyEvent@@@Z 100081c8     Qt5Widgets:Qt5Widgets.dll
 0002:000001cc       __imp_?keyPressEvent@QLabel@@MAEXPAVQKeyEvent@@@Z 100081cc     Qt5Widgets:Qt5Widgets.dll
 0002:000001d0       __imp_?keyPressEvent@QWidget@@MAEXPAVQKeyEvent@@@Z 100081d0     Qt5Widgets:Qt5Widgets.dll
 0002:000001d4       __imp_?keyReleaseEvent@QAbstractButton@@MAEXPAVQKeyEvent@@@Z 100081d4     Qt5Widgets:Qt5Widgets.dll
 0002:000001d8       __imp_?keyReleaseEvent@QWidget@@MAEXPAVQKeyEvent@@@Z 100081d8     Qt5Widgets:Qt5Widgets.dll
 0002:000001dc       __imp_?layout@QLayout@@UAEPAV1@XZ 100081dc     Qt5Widgets:Qt5Widgets.dll
 0002:000001e0       __imp_?leaveEvent@QWidget@@MAEXPAVQEvent@@@Z 100081e0     Qt5Widgets:Qt5Widgets.dll
 0002:000001e4       __imp_?maximumSize@QBoxLayout@@UBE?AVQSize@@XZ 100081e4     Qt5Widgets:Qt5Widgets.dll
 0002:000001e8       __imp_?metaObject@QCheckBox@@UBEPBUQMetaObject@@XZ 100081e8     Qt5Widgets:Qt5Widgets.dll
 0002:000001ec       __imp_?metaObject@QHBoxLayout@@UBEPBUQMetaObject@@XZ 100081ec     Qt5Widgets:Qt5Widgets.dll
 0002:000001f0       __imp_?metaObject@QLabel@@UBEPBUQMetaObject@@XZ 100081f0     Qt5Widgets:Qt5Widgets.dll
 0002:000001f4       __imp_?metaObject@QVBoxLayout@@UBEPBUQMetaObject@@XZ 100081f4     Qt5Widgets:Qt5Widgets.dll
 0002:000001f8       __imp_?metric@QWidget@@MBEHW4PaintDeviceMetric@QPaintDevice@@@Z 100081f8     Qt5Widgets:Qt5Widgets.dll
 0002:000001fc       __imp_?minimumHeightForWidth@QBoxLayout@@UBEHH@Z 100081fc     Qt5Widgets:Qt5Widgets.dll
 0002:00000200       __imp_?minimumSize@QBoxLayout@@UBE?AVQSize@@XZ 10008200     Qt5Widgets:Qt5Widgets.dll
 0002:00000204       __imp_?minimumSizeHint@QCheckBox@@UBE?AVQSize@@XZ 10008204     Qt5Widgets:Qt5Widgets.dll
 0002:00000208       __imp_?minimumSizeHint@QLabel@@UBE?AVQSize@@XZ 10008208     Qt5Widgets:Qt5Widgets.dll
 0002:0000020c       __imp_?minimumSizeHint@QWidget@@UBE?AVQSize@@XZ 1000820c     Qt5Widgets:Qt5Widgets.dll
 0002:00000210       __imp_?mouseDoubleClickEvent@QWidget@@MAEXPAVQMouseEvent@@@Z 10008210     Qt5Widgets:Qt5Widgets.dll
 0002:00000214       __imp_?mouseMoveEvent@QCheckBox@@MAEXPAVQMouseEvent@@@Z 10008214     Qt5Widgets:Qt5Widgets.dll
 0002:00000218       __imp_?mouseMoveEvent@QLabel@@MAEXPAVQMouseEvent@@@Z 10008218     Qt5Widgets:Qt5Widgets.dll
 0002:0000021c       __imp_?mouseMoveEvent@QWidget@@MAEXPAVQMouseEvent@@@Z 1000821c     Qt5Widgets:Qt5Widgets.dll
 0002:00000220       __imp_?mousePressEvent@QAbstractButton@@MAEXPAVQMouseEvent@@@Z 10008220     Qt5Widgets:Qt5Widgets.dll
 0002:00000224       __imp_?mousePressEvent@QLabel@@MAEXPAVQMouseEvent@@@Z 10008224     Qt5Widgets:Qt5Widgets.dll
 0002:00000228       __imp_?mousePressEvent@QWidget@@MAEXPAVQMouseEvent@@@Z 10008228     Qt5Widgets:Qt5Widgets.dll
 0002:0000022c       __imp_?mouseReleaseEvent@QAbstractButton@@MAEXPAVQMouseEvent@@@Z 1000822c     Qt5Widgets:Qt5Widgets.dll
 0002:00000230       __imp_?mouseReleaseEvent@QLabel@@MAEXPAVQMouseEvent@@@Z 10008230     Qt5Widgets:Qt5Widgets.dll
 0002:00000234       __imp_?mouseReleaseEvent@QWidget@@MAEXPAVQMouseEvent@@@Z 10008234     Qt5Widgets:Qt5Widgets.dll
 0002:00000238       __imp_?moveEvent@QWidget@@MAEXPAVQMoveEvent@@@Z 10008238     Qt5Widgets:Qt5Widgets.dll
 0002:0000023c       __imp_?nativeEvent@QWidget@@MAE_NABVQByteArray@@PAXPAJ@Z 1000823c     Qt5Widgets:Qt5Widgets.dll
 0002:00000240       __imp_?nextCheckState@QCheckBox@@MAEXXZ 10008240     Qt5Widgets:Qt5Widgets.dll
 0002:00000244       __imp_?paintEngine@QWidget@@UBEPAVQPaintEngine@@XZ 10008244     Qt5Widgets:Qt5Widgets.dll
 0002:00000248       __imp_?paintEvent@QCheckBox@@MAEXPAVQPaintEvent@@@Z 10008248     Qt5Widgets:Qt5Widgets.dll
 0002:0000024c       __imp_?paintEvent@QLabel@@MAEXPAVQPaintEvent@@@Z 1000824c     Qt5Widgets:Qt5Widgets.dll
 0002:00000250       __imp_?paintEvent@QWidget@@MAEXPAVQPaintEvent@@@Z 10008250     Qt5Widgets:Qt5Widgets.dll
 0002:00000254       __imp_?qt_metacall@QCheckBox@@UAEHW4Call@QMetaObject@@HPAPAX@Z 10008254     Qt5Widgets:Qt5Widgets.dll
 0002:00000258       __imp_?qt_metacall@QHBoxLayout@@UAEHW4Call@QMetaObject@@HPAPAX@Z 10008258     Qt5Widgets:Qt5Widgets.dll
 0002:0000025c       __imp_?qt_metacall@QLabel@@UAEHW4Call@QMetaObject@@HPAPAX@Z 1000825c     Qt5Widgets:Qt5Widgets.dll
 0002:00000260       __imp_?qt_metacall@QVBoxLayout@@UAEHW4Call@QMetaObject@@HPAPAX@Z 10008260     Qt5Widgets:Qt5Widgets.dll
 0002:00000264       __imp_?qt_metacast@QCheckBox@@UAEPAXPBD@Z 10008264     Qt5Widgets:Qt5Widgets.dll
 0002:00000268       __imp_?qt_metacast@QHBoxLayout@@UAEPAXPBD@Z 10008268     Qt5Widgets:Qt5Widgets.dll
 0002:0000026c       __imp_?qt_metacast@QLabel@@UAEPAXPBD@Z 1000826c     Qt5Widgets:Qt5Widgets.dll
 0002:00000270       __imp_?qt_metacast@QVBoxLayout@@UAEPAXPBD@Z 10008270     Qt5Widgets:Qt5Widgets.dll
 0002:00000274       __imp_?redirected@QWidget@@MBEPAVQPaintDevice@@PAVQPoint@@@Z 10008274     Qt5Widgets:Qt5Widgets.dll
 0002:00000278       __imp_?resizeEvent@QWidget@@MAEXPAVQResizeEvent@@@Z 10008278     Qt5Widgets:Qt5Widgets.dll
 0002:0000027c       __imp_?setGeometry@QBoxLayout@@UAEXABVQRect@@@Z 1000827c     Qt5Widgets:Qt5Widgets.dll
 0002:00000280       __imp_?setVisible@QWidget@@UAEX_N@Z 10008280     Qt5Widgets:Qt5Widgets.dll
 0002:00000284       __imp_?sharedPainter@QWidget@@MBEPAVQPainter@@XZ 10008284     Qt5Widgets:Qt5Widgets.dll
 0002:00000288       __imp_?showEvent@QWidget@@MAEXPAVQShowEvent@@@Z 10008288     Qt5Widgets:Qt5Widgets.dll
 0002:0000028c       __imp_?sizeHint@QBoxLayout@@UBE?AVQSize@@XZ 1000828c     Qt5Widgets:Qt5Widgets.dll
 0002:00000290       __imp_?sizeHint@QCheckBox@@UBE?AVQSize@@XZ 10008290     Qt5Widgets:Qt5Widgets.dll
 0002:00000294       __imp_?sizeHint@QLabel@@UBE?AVQSize@@XZ 10008294     Qt5Widgets:Qt5Widgets.dll
 0002:00000298       __imp_?sizeHint@QWidget@@UBE?AVQSize@@XZ 10008298     Qt5Widgets:Qt5Widgets.dll
 0002:0000029c       __imp_?spacerItem@QLayoutItem@@UAEPAVQSpacerItem@@XZ 1000829c     Qt5Widgets:Qt5Widgets.dll
 0002:000002a0       __imp_?tabletEvent@QWidget@@MAEXPAVQTabletEvent@@@Z 100082a0     Qt5Widgets:Qt5Widgets.dll
 0002:000002a4       __imp_?takeAt@QBoxLayout@@UAEPAVQLayoutItem@@H@Z 100082a4     Qt5Widgets:Qt5Widgets.dll
 0002:000002a8       __imp_?timerEvent@QAbstractButton@@MAEXPAVQTimerEvent@@@Z 100082a8     Qt5Widgets:Qt5Widgets.dll
 0002:000002ac       __imp_?wheelEvent@QWidget@@MAEXPAVQWheelEvent@@@Z 100082ac     Qt5Widgets:Qt5Widgets.dll
 0002:000002b0       __imp_?widget@QLayoutItem@@UAEPAVQWidget@@XZ 100082b0     Qt5Widgets:Qt5Widgets.dll
 0002:000002b4       __imp_?event@QCheckBox@@MAE_NPAVQEvent@@@Z 100082b4     Qt5Widgets:Qt5Widgets.dll
 0002:000002b8       __imp_?enterEvent@QWidget@@MAEXPAVQEvent@@@Z 100082b8     Qt5Widgets:Qt5Widgets.dll
 0002:000002bc       __imp_?dropEvent@QWidget@@MAEXPAVQDropEvent@@@Z 100082bc     Qt5Widgets:Qt5Widgets.dll
 0002:000002c0       __imp_?dragMoveEvent@QWidget@@MAEXPAVQDragMoveEvent@@@Z 100082c0     Qt5Widgets:Qt5Widgets.dll
 0002:000002c4       __imp_?dragLeaveEvent@QWidget@@MAEXPAVQDragLeaveEvent@@@Z 100082c4     Qt5Widgets:Qt5Widgets.dll
 0002:000002c8       __imp_?dragEnterEvent@QWidget@@MAEXPAVQDragEnterEvent@@@Z 100082c8     Qt5Widgets:Qt5Widgets.dll
 0002:000002cc       __imp_?devType@QWidget@@UBEHXZ 100082cc     Qt5Widgets:Qt5Widgets.dll
 0002:000002d0       __imp_?count@QBoxLayout@@UBEHXZ 100082d0     Qt5Widgets:Qt5Widgets.dll
 0002:000002d4       __imp_?controlTypes@QLayout@@UBE?AV?$QFlags@W4ControlType@QSizePolicy@@@@XZ 100082d4     Qt5Widgets:Qt5Widgets.dll
 0002:000002d8       __imp_?contextMenuEvent@QWidget@@MAEXPAVQContextMenuEvent@@@Z 100082d8     Qt5Widgets:Qt5Widgets.dll
 0002:000002dc       __imp_?contextMenuEvent@QLabel@@MAEXPAVQContextMenuEvent@@@Z 100082dc     Qt5Widgets:Qt5Widgets.dll
 0002:000002e0       __imp_?closeEvent@QWidget@@MAEXPAVQCloseEvent@@@Z 100082e0     Qt5Widgets:Qt5Widgets.dll
 0002:000002e4       __imp_?childEvent@QLayout@@MAEXPAVQChildEvent@@@Z 100082e4     Qt5Widgets:Qt5Widgets.dll
 0002:000002e8       __imp_?checkStateSet@QCheckBox@@MAEXXZ 100082e8     Qt5Widgets:Qt5Widgets.dll
 0002:000002ec       __imp_?changeEvent@QWidget@@MAEXPAVQEvent@@@Z 100082ec     Qt5Widgets:Qt5Widgets.dll
 0002:000002f0       __imp_?changeEvent@QLabel@@MAEXPAVQEvent@@@Z 100082f0     Qt5Widgets:Qt5Widgets.dll
 0002:000002f4       __imp_?changeEvent@QAbstractButton@@MAEXPAVQEvent@@@Z 100082f4     Qt5Widgets:Qt5Widgets.dll
 0002:000002f8       __imp_?addItem@QBoxLayout@@UAEXPAVQLayoutItem@@@Z 100082f8     Qt5Widgets:Qt5Widgets.dll
 0002:000002fc       __imp_?actionEvent@QWidget@@MAEXPAVQActionEvent@@@Z 100082fc     Qt5Widgets:Qt5Widgets.dll
 0002:00000300       __imp_??1QCheckBox@@UAE@XZ 10008300     Qt5Widgets:Qt5Widgets.dll
 0002:00000304       __imp_??0QCheckBox@@QAE@ABVQString@@PAVQWidget@@@Z 10008304     Qt5Widgets:Qt5Widgets.dll
 0002:00000308       __imp_?setChecked@QAbstractButton@@QAEX_N@Z 10008308     Qt5Widgets:Qt5Widgets.dll
 0002:0000030c       __imp_?isChecked@QAbstractButton@@QBE_NXZ 1000830c     Qt5Widgets:Qt5Widgets.dll
 0002:00000310       __imp_??1QVBoxLayout@@UAE@XZ 10008310     Qt5Widgets:Qt5Widgets.dll
 0002:00000314       __imp_??0QVBoxLayout@@QAE@PAVQWidget@@@Z 10008314     Qt5Widgets:Qt5Widgets.dll
 0002:00000318       __imp_??1QHBoxLayout@@UAE@XZ 10008318     Qt5Widgets:Qt5Widgets.dll
 0002:0000031c       __imp_??0QHBoxLayout@@QAE@PAVQWidget@@@Z 1000831c     Qt5Widgets:Qt5Widgets.dll
 0002:00000320       __imp_?addLayout@QBoxLayout@@QAEXPAVQLayout@@H@Z 10008320     Qt5Widgets:Qt5Widgets.dll
 0002:00000324       __imp_?addWidget@QBoxLayout@@QAEXPAVQWidget@@HV?$QFlags@W4AlignmentFlag@Qt@@@@@Z 10008324     Qt5Widgets:Qt5Widgets.dll
 0002:00000328       __imp_?addStretch@QBoxLayout@@QAEXH@Z 10008328     Qt5Widgets:Qt5Widgets.dll
 0002:0000032c       __imp_?setAlignment@QLayoutItem@@QAEXV?$QFlags@W4AlignmentFlag@Qt@@@@@Z 1000832c     Qt5Widgets:Qt5Widgets.dll
 0002:00000330       __imp_?setAlignment@QLabel@@QAEXV?$QFlags@W4AlignmentFlag@Qt@@@@@Z 10008330     Qt5Widgets:Qt5Widgets.dll
 0002:00000334       __imp_??1QLabel@@UAE@XZ    10008334     Qt5Widgets:Qt5Widgets.dll
 0002:00000338       __imp_??0QLabel@@QAE@ABVQString@@PAVQWidget@@V?$QFlags@W4WindowType@Qt@@@@@Z 10008338     Qt5Widgets:Qt5Widgets.dll
 0002:0000033c       __imp_?setLayout@QWidget@@QAEXPAVQLayout@@@Z 1000833c     Qt5Widgets:Qt5Widgets.dll
 0002:00000340       __imp_?setSizePolicy@QWidget@@QAEXVQSizePolicy@@@Z 10008340     Qt5Widgets:Qt5Widgets.dll
 0002:00000344       __imp_??1QWidget@@UAE@XZ   10008344     Qt5Widgets:Qt5Widgets.dll
 0002:00000348       __imp_??0QSizePolicy@@QAE@W4Policy@0@0W4ControlType@0@@Z 10008348     Qt5Widgets:Qt5Widgets.dll
 0002:0000034c       __imp_?hitButton@QCheckBox@@MBE_NABVQPoint@@@Z 1000834c     Qt5Widgets:Qt5Widgets.dll
 0002:00000350       \177Qt5Widgets_NULL_THUNK_DATA 10008350     Qt5Widgets:Qt5Widgets.dll
 0002:00000354       __imp_?getErrorString@OpenCLHelper@U2@@QBE?AVQString@@XZ 10008354     U2Algorithm:U2Algorithm.dll
 0002:00000358       __imp_??1OpenCLHelper@U2@@QAE@XZ 10008358     U2Algorithm:U2Algorithm.dll
 0002:0000035c       __imp_??0OpenCLGpuModel@U2@@QAE@ABVQString@@ABJ1_K222III_N@Z 1000835c     U2Algorithm:U2Algorithm.dll
 0002:00000360       __imp_?getName@OpenCLGpuModel@U2@@QBE?AVQString@@XZ 10008360     U2Algorithm:U2Algorithm.dll
 0002:00000364       __imp_?registerOpenCLGpu@OpenCLGpuRegistry@U2@@QAEXPAVOpenCLGpuModel@2@@Z 10008364     U2Algorithm:U2Algorithm.dll
 0002:00000368       __imp_?unregisterOpenCLGpu@OpenCLGpuRegistry@U2@@QAEXPAVOpenCLGpuModel@2@@Z 10008368     U2Algorithm:U2Algorithm.dll
 0002:0000036c       __imp_?getRegisteredGpus@OpenCLGpuRegistry@U2@@QBE?AV?$QList@PAVOpenCLGpuModel@U2@@@@XZ 1000836c     U2Algorithm:U2Algorithm.dll
 0002:00000370       __imp_??0OpenCLHelper@U2@@QAE@XZ 10008370     U2Algorithm:U2Algorithm.dll
 0002:00000374       \177U2Algorithm_NULL_THUNK_DATA 10008374     U2Algorithm:U2Algorithm.dll
 0002:00000378       __imp_??1AppResourceSemaphore@U2@@UAE@XZ 10008378     U2Core:U2Core.dll
 0002:0000037c       __imp_?registerResource@AppResourcePool@U2@@QAEXPAVAppResource@2@@Z 1000837c     U2Core:U2Core.dll
 0002:00000380       __imp_??0AppResourceSemaphore@U2@@QAE@HHABVQString@@0@Z 10008380     U2Core:U2Core.dll
 0002:00000384       __imp_?instance@AppResourcePool@U2@@SAPAV12@XZ 10008384     U2Core:U2Core.dll
 0002:00000388       __imp_??0Plugin@U2@@QAE@ABVQString@@0_NW4PluginState@1@@Z 10008388     U2Core:U2Core.dll
 0002:0000038c       __imp_??1Plugin@U2@@UAE@XZ 1000838c     U2Core:U2Core.dll
 0002:00000390       __imp_?info@Logger@U2@@QAEXABVQString@@@Z 10008390     U2Core:U2Core.dll
 0002:00000394       __imp_?details@Logger@U2@@QAEXABVQString@@@Z 10008394     U2Core:U2Core.dll
 0002:00000398       __imp_??1Logger@U2@@UAE@XZ 10008398     U2Core:U2Core.dll
 0002:0000039c       __imp_??0Logger@U2@@QAE@ABVQString@@@Z 1000839c     U2Core:U2Core.dll
 0002:000003a0       __imp_?getOpenCLGpuRegistry@AppContext@U2@@SAPAVOpenCLGpuRegistry@2@XZ 100083a0     U2Core:U2Core.dll
 0002:000003a4       __imp_?getMainWindow@AppContext@U2@@SAPAVMainWindow@2@XZ 100083a4     U2Core:U2Core.dll
 0002:000003a8       __imp_?getAppSettingsGUI@AppContext@U2@@SAPAVAppSettingsGUI@2@XZ 100083a8     U2Core:U2Core.dll
 0002:000003ac       __imp_?unregisterResource@AppResourcePool@U2@@QAEXH@Z 100083ac     U2Core:U2Core.dll
 0002:000003b0       __imp_?staticMetaObject@Plugin@U2@@2UQMetaObject@@B 100083b0     U2Core:U2Core.dll
 0002:000003b4       __imp_?getSettings@AppContext@U2@@SAPAVSettings@2@XZ 100083b4     U2Core:U2Core.dll
 0002:000003b8       __imp_?qt_metacall@Plugin@U2@@UAEHW4Call@QMetaObject@@HPAPAX@Z 100083b8     U2Core:U2Core.dll
 0002:000003bc       __imp_?qt_metacast@Plugin@U2@@UAEPAXPBD@Z 100083bc     U2Core:U2Core.dll
 0002:000003c0       __imp_?getResource@AppResourcePool@U2@@QBEPAVAppResource@2@H@Z 100083c0     U2Core:U2Core.dll
 0002:000003c4       __imp_?setMaxUse@AppResourceSemaphore@U2@@QAEXH@Z 100083c4     U2Core:U2Core.dll
 0002:000003c8       __imp_?tryAcquire@AppResourceSemaphore@U2@@UAE_NHW4MemoryLockType@AppResource@2@@Z 100083c8     U2Core:U2Core.dll
 0002:000003cc       __imp_?tryAcquire@AppResourceSemaphore@U2@@UAE_NHHW4MemoryLockType@AppResource@2@@Z 100083cc     U2Core:U2Core.dll
 0002:000003d0       __imp_?release@AppResourceSemaphore@U2@@UAEXHW4MemoryLockType@AppResource@2@@Z 100083d0     U2Core:U2Core.dll
 0002:000003d4       __imp_?available@AppResourceSemaphore@U2@@UBEHXZ 100083d4     U2Core:U2Core.dll
 0002:000003d8       __imp_?acquire@AppResourceSemaphore@U2@@UAEXHW4MemoryLockType@AppResource@2@@Z 100083d8     U2Core:U2Core.dll
 0002:000003dc       \177U2Core_NULL_THUNK_DATA 100083dc     U2Core:U2Core.dll
 0002:000003e0       __imp_??1AppSettingsGUIPageState@U2@@UAE@XZ 100083e0     U2Gui:U2Gui.dll
 0002:000003e4       __imp_??0AppSettingsGUIPageWidget@U2@@QAE@PAVQWidget@@@Z 100083e4     U2Gui:U2Gui.dll
 0002:000003e8       __imp_??1AppSettingsGUIPageWidget@U2@@UAE@XZ 100083e8     U2Gui:U2Gui.dll
 0002:000003ec       __imp_??0AppSettingsGUIPageController@U2@@QAE@ABVQString@@0PAVQObject@@@Z 100083ec     U2Gui:U2Gui.dll
 0002:000003f0       __imp_??1AppSettingsGUIPageController@U2@@UAE@XZ 100083f0     U2Gui:U2Gui.dll
 0002:000003f4       __imp_?qt_metacast@AppSettingsGUIPageState@U2@@UAEPAXPBD@Z 100083f4     U2Gui:U2Gui.dll
 0002:000003f8       __imp_?qt_metacall@AppSettingsGUIPageState@U2@@UAEHW4Call@QMetaObject@@HPAPAX@Z 100083f8     U2Gui:U2Gui.dll
 0002:000003fc       __imp_?qt_metacast@AppSettingsGUIPageWidget@U2@@UAEPAXPBD@Z 100083fc     U2Gui:U2Gui.dll
 0002:00000400       __imp_?qt_metacall@AppSettingsGUIPageWidget@U2@@UAEHW4Call@QMetaObject@@HPAPAX@Z 10008400     U2Gui:U2Gui.dll
 0002:00000404       __imp_?qt_metacast@AppSettingsGUIPageController@U2@@UAEPAXPBD@Z 10008404     U2Gui:U2Gui.dll
 0002:00000408       __imp_?qt_metacall@AppSettingsGUIPageController@U2@@UAEHW4Call@QMetaObject@@HPAPAX@Z 10008408     U2Gui:U2Gui.dll
 0002:0000040c       __imp_?staticMetaObject@AppSettingsGUIPageState@U2@@2UQMetaObject@@B 1000840c     U2Gui:U2Gui.dll
 0002:00000410       __imp_?staticMetaObject@AppSettingsGUIPageWidget@U2@@2UQMetaObject@@B 10008410     U2Gui:U2Gui.dll
 0002:00000414       __imp_?staticMetaObject@AppSettingsGUIPageController@U2@@2UQMetaObject@@B 10008414     U2Gui:U2Gui.dll
 0002:00000418       \177U2Gui_NULL_THUNK_DATA  10008418     U2Gui:U2Gui.dll
 0002:0000041c       ___xc_a                    1000841c     MSVCRT:cinitexe.obj
 0002:00000488       ___xc_z                    10008488     MSVCRT:cinitexe.obj
 0002:0000048c       ___xi_a                    1000848c     MSVCRT:cinitexe.obj
 0002:00000498       ___xi_z                    10008498     MSVCRT:cinitexe.obj
 0002:000004d8       ??_C@_09NEFANJPL@OpenCLGpu?$AA@ 100084d8     OpenCLSupportPlugin.obj
 0002:000004e2       ??_C@_00CNPNBAHC@?$AA@     100084e2     OpenCLSupportPlugin.obj
 0002:000004e8       ??_7error_category@std@@6B@ 100084e8     OpenCLSupportPlugin.obj
 0002:00000504       ??_7_Generic_error_category@std@@6B@ 10008504     OpenCLSupportPlugin.obj
 0002:0000051c       ??_C@_07DCLBNMLN@generic?$AA@ 1000851c     OpenCLSupportPlugin.obj
 0002:00000524       ??_C@_0O@BFJCFAAK@unknown?5error?$AA@ 10008524     OpenCLSupportPlugin.obj
 0002:00000538       ??_7_Iostream_error_category@std@@6B@ 10008538     OpenCLSupportPlugin.obj
 0002:00000550       ??_C@_08LLGCOLLL@iostream?$AA@ 10008550     OpenCLSupportPlugin.obj
 0002:0000055c       ??_C@_0BG@PADBLCHM@iostream?5stream?5error?$AA@ 1000855c     OpenCLSupportPlugin.obj
 0002:00000578       ??_7_System_error_category@std@@6B@ 10008578     OpenCLSupportPlugin.obj
 0002:00000590       ??_C@_06FHFOAHML@system?$AA@ 10008590     OpenCLSupportPlugin.obj
 0002:00000598       ??_C@_0L@JLHNEGIN@Algorithms?$AA@ 10008598     OpenCLSupportPlugin.obj
 0002:000005a4       ??_C@_07PGLPGHFC@Console?$AA@ 100085a4     OpenCLSupportPlugin.obj
 0002:000005ac       ??_C@_0O@BOFHOPCF@Core?5Services?$AA@ 100085ac     OpenCLSupportPlugin.obj
 0002:000005bc       ??_C@_0N@PPADAKBM@Input?1Output?$AA@ 100085bc     OpenCLSupportPlugin.obj
 0002:000005cc       ??_C@_0M@KPPBKPKK@Performance?$AA@ 100085cc     OpenCLSupportPlugin.obj
 0002:000005d8       ??_C@_07BFDHHBBI@Scripts?$AA@ 100085d8     OpenCLSupportPlugin.obj
 0002:000005e0       ??_C@_05EEGKELMG@Tasks?$AA@ 100085e0     OpenCLSupportPlugin.obj
 0002:000005e8       ??_C@_0P@NIIOBHGA@User?5Interface?$AA@ 100085e8     OpenCLSupportPlugin.obj
 0002:000005f8       ??_C@_0N@JINCGGMN@User?5Actions?$AA@ 100085f8     OpenCLSupportPlugin.obj
 0002:0000060c       ??_SAppResourceSemaphore@U2@@6B@ 1000860c     OpenCLSupportPlugin.obj
 0002:00000628       ??_7OpenCLSupportPlugin@U2@@6B@ 10008628     OpenCLSupportPlugin.obj
 0002:00000658       ??_C@_0BAP@MENNKHK@Problem?5occurred?5loading?5the?5Ope@ 10008658     OpenCLSupportPlugin.obj
 0002:00000768       ??_C@_0CI@PMLJCDJK@http?3?1?1ugene?4net?1using?9video?9car@ 10008768     OpenCLSupportPlugin.obj
 0002:00000790       ??_C@_0DB@HIHBFGIO@Plugin?5provides?5support?5for?5Open@ 10008790     OpenCLSupportPlugin.obj
 0002:000007c4       ??_C@_0P@CPDIDKLL@OpenCL?5Support?$AA@ 100087c4     OpenCLSupportPlugin.obj
 0002:000007d4       ??_C@_0BO@DCHKAIHM@No?5OpenCL?9enabled?5GPUs?5found?4?$AA@ 100087d4     OpenCLSupportPlugin.obj
 0002:000007f8       ??_C@_0GK@PLEBHOBA@Cannot?5load?5OpenCL?5driver?5dynami@ 100087f8     OpenCLSupportPlugin.obj
 0002:00000868       ??_C@_0KJ@JABJLHEN@An?5error?5has?5occurred?5while?5obta@ 10008868     OpenCLSupportPlugin.obj
 0002:00000914       ??_C@_0BE@MLOHHMH@Initializing?5OpenCL?$AA@ 10008914     OpenCLSupportPlugin.obj
 0002:00000928       ??_C@_0BP@NHEDOMLH@Number?5of?5OpenCL?5platforms?3?5?$CF1?$AA@ 10008928     OpenCLSupportPlugin.obj
 0002:00000948       ??_C@_0BN@KNJEEAGA@Number?5of?5OpenCL?5devices?3?5?$CF1?$AA@ 10008948     OpenCLSupportPlugin.obj
 0002:00000968       ??_C@_01CLKCMJKC@?5?$AA@   10008968     OpenCLSupportPlugin.obj
 0002:00000970       ??_C@_0MI@FENPOFFA@Registering?5OpenCL?9enabled?5GPU?3?5@ 10008970     OpenCLSupportPlugin.obj
 0002:00000a38       ??_C@_0BH@BOFKCGAE@OpenCL?5error?5code?5?$CI?$CF1?$CJ?$AA@ 10008a38     OpenCLSupportPlugin.obj
 0002:00000a50       ??_C@_08BJBLCIEF@?1enabled?$AA@ 10008a50     OpenCLSupportPlugin.obj
 0002:00000a5c       ??_C@_0CC@DFCDCOCE@?1opencl_gpu_registry?1gpu_specifi@ 10008a5c     OpenCLSupportPlugin.obj
 0002:00000a80       ??_C@_0BA@JFNIOLAK@string?5too?5long?$AA@ 10008a80     OpenCLSupportPlugin.obj
 0002:00000a90       ??_C@_0BI@CFPLBAOH@invalid?5string?5position?$AA@ 10008a90     OpenCLSupportPlugin.obj
 0002:00000aa8       ??_C@_0HH@CPFAKEAI@The?5following?5OpenCL?9enabled?5GPU@ 10008aa8     OpenCLSupportSettingsController.obj
 0002:00000b20       ??_C@_0CA@FAGMCMIL@No?5OpenCL?9enabled?5GPU?5detected?4?$AA@ 10008b20     OpenCLSupportSettingsController.obj
 0002:00000b44       ??_SQLabel@@6BQObject@@@   10008b44     OpenCLSupportSettingsController.obj
 0002:00000bfc       ??_SQLabel@@6BQPaintDevice@@@ 10008bfc     OpenCLSupportSettingsController.obj
 0002:00000c1c       ??_SQHBoxLayout@@6BQObject@@@ 10008c1c     OpenCLSupportSettingsController.obj
 0002:00000c64       ??_SQHBoxLayout@@6BQLayoutItem@@@ 10008c64     OpenCLSupportSettingsController.obj
 0002:00000cac       ??_SQVBoxLayout@@6BQObject@@@ 10008cac     OpenCLSupportSettingsController.obj
 0002:00000cf4       ??_SQVBoxLayout@@6BQLayoutItem@@@ 10008cf4     OpenCLSupportSettingsController.obj
 0002:00000d3c       ??_SQCheckBox@@6BQObject@@@ 10008d3c     OpenCLSupportSettingsController.obj
 0002:00000e00       ??_SQCheckBox@@6BQPaintDevice@@@ 10008e00     OpenCLSupportSettingsController.obj
 0002:00000e20       ??_7OpenCLSupportSettingsPageController@U2@@6B@ 10008e20     OpenCLSupportSettingsController.obj
 0002:00000e60       ??_7OpenCLSupportSettingsPageState@U2@@6B@ 10008e60     OpenCLSupportSettingsController.obj
 0002:00000e90       ??_7OpenCLSupportSettingsPageWidget@U2@@6BQObject@@@ 10008e90     OpenCLSupportSettingsController.obj
 0002:00000f50       ??_7OpenCLSupportSettingsPageWidget@U2@@6BQPaintDevice@@@ 10008f50     OpenCLSupportSettingsController.obj
 0002:00000f6c       ??_C@_05EKFIFKMJ@oclss?$AA@ 10008f6c     OpenCLSupportSettingsController.obj
 0002:00000f74       ??_C@_06HPMJGDEN@OpenCL?$AA@ 10008f74     OpenCLSupportSettingsController.obj
 0002:00000f7c       ??_C@_08BACLAJHK@23330958?$AA@ 10008f7c     OpenCLSupportSettingsController.obj
 0002:00000f88       ??_C@_03FBAAJIGL@?5Mb?$AA@ 10008f88     OpenCLSupportSettingsController.obj
 0002:00001144       ?value@?$integral_constant@_N$0A@@std@@2_NB 10009144     msvcprt:newaop_s.obj
 0002:00001145       ?value@?$integral_constant@_N$00@std@@2_NB 10009145     msvcprt:newaop_s.obj
 0002:0000114c       ??_7type_info@@6B@         1000914c     MSVCRT:ti_inst.obj
 0002:00001150       __pDefaultRawDllMain       10009150     MSVCRT:crtdll.obj
 0002:00001150       __pRawDllMain              10009150     MSVCRT:crtdll.obj
 0002:0000115c       ?ProcessDetach@NativeDll@<CrtImplementationDetails>@@0IB 1000915c     MSVCRT:initsect.obj
 0002:00001160       ?ProcessAttach@NativeDll@<CrtImplementationDetails>@@0IB 10009160     MSVCRT:initsect.obj
 0002:00001164       ?ThreadAttach@NativeDll@<CrtImplementationDetails>@@0IB 10009164     MSVCRT:initsect.obj
 0002:00001168       ?ThreadDetach@NativeDll@<CrtImplementationDetails>@@0IB 10009168     MSVCRT:initsect.obj
 0002:0000116c       ?ProcessVerifier@NativeDll@<CrtImplementationDetails>@@0IB 1000916c     MSVCRT:initsect.obj
 0002:00001170       __load_config_used         10009170     MSVCRT:loadcfg.obj
 0002:0000122c       ??_R4error_category@std@@6B@ 1000922c     OpenCLSupportPlugin.obj
 0002:00001240       ??_R3error_category@std@@8 10009240     OpenCLSupportPlugin.obj
 0002:00001250       ??_R2error_category@std@@8 10009250     OpenCLSupportPlugin.obj
 0002:00001258       ??_R1A@?0A@EA@error_category@std@@8 10009258     OpenCLSupportPlugin.obj
 0002:00001274       ??_R4_Generic_error_category@std@@6B@ 10009274     OpenCLSupportPlugin.obj
 0002:00001288       ??_R3_Generic_error_category@std@@8 10009288     OpenCLSupportPlugin.obj
 0002:00001298       ??_R2_Generic_error_category@std@@8 10009298     OpenCLSupportPlugin.obj
 0002:000012a4       ??_R1A@?0A@EA@_Generic_error_category@std@@8 100092a4     OpenCLSupportPlugin.obj
 0002:000012c0       ??_R4_Iostream_error_category@std@@6B@ 100092c0     OpenCLSupportPlugin.obj
 0002:000012d4       ??_R3_Iostream_error_category@std@@8 100092d4     OpenCLSupportPlugin.obj
 0002:000012e4       ??_R2_Iostream_error_category@std@@8 100092e4     OpenCLSupportPlugin.obj
 0002:000012f4       ??_R1A@?0A@EA@_Iostream_error_category@std@@8 100092f4     OpenCLSupportPlugin.obj
 0002:00001310       ??_R4_System_error_category@std@@6B@ 10009310     OpenCLSupportPlugin.obj
 0002:00001324       ??_R3_System_error_category@std@@8 10009324     OpenCLSupportPlugin.obj
 0002:00001334       ??_R2_System_error_category@std@@8 10009334     OpenCLSupportPlugin.obj
 0002:00001344       ??_R1A@?0A@EA@_System_error_category@std@@8 10009344     OpenCLSupportPlugin.obj
 0002:00001360       ??_R4AppResourceSemaphore@U2@@6B@ 10009360     OpenCLSupportPlugin.obj
 0002:00001374       ??_R3AppResourceSemaphore@U2@@8 10009374     OpenCLSupportPlugin.obj
 0002:00001384       ??_R2AppResourceSemaphore@U2@@8 10009384     OpenCLSupportPlugin.obj
 0002:00001390       ??_R1A@?0A@EA@AppResourceSemaphore@U2@@8 10009390     OpenCLSupportPlugin.obj
 0002:000013ac       ??_R1A@?0A@EA@AppResource@U2@@8 100093ac     OpenCLSupportPlugin.obj
 0002:000013c8       ??_R3AppResource@U2@@8     100093c8     OpenCLSupportPlugin.obj
 0002:000013d8       ??_R2AppResource@U2@@8     100093d8     OpenCLSupportPlugin.obj
 0002:000013e0       ??_R4OpenCLSupportPlugin@U2@@6B@ 100093e0     OpenCLSupportPlugin.obj
 0002:000013f4       ??_R3OpenCLSupportPlugin@U2@@8 100093f4     OpenCLSupportPlugin.obj
 0002:00001404       ??_R2OpenCLSupportPlugin@U2@@8 10009404     OpenCLSupportPlugin.obj
 0002:00001414       ??_R1A@?0A@EA@OpenCLSupportPlugin@U2@@8 10009414     OpenCLSupportPlugin.obj
 0002:00001430       ??_R1A@?0A@EA@Plugin@U2@@8 10009430     OpenCLSupportPlugin.obj
 0002:0000144c       ??_R3Plugin@U2@@8          1000944c     OpenCLSupportPlugin.obj
 0002:0000145c       ??_R2Plugin@U2@@8          1000945c     OpenCLSupportPlugin.obj
 0002:00001468       ??_R1A@?0A@EA@QObject@@8   10009468     OpenCLSupportPlugin.obj
 0002:00001484       ??_R3QObject@@8            10009484     OpenCLSupportPlugin.obj
 0002:00001494       ??_R2QObject@@8            10009494     OpenCLSupportPlugin.obj
 0002:0000149c       ??_R4QLabel@@6BQObject@@@  1000949c     OpenCLSupportSettingsController.obj
 0002:000014b0       ??_R3QLabel@@8             100094b0     OpenCLSupportSettingsController.obj
 0002:000014c0       ??_R2QLabel@@8             100094c0     OpenCLSupportSettingsController.obj
 0002:000014d8       ??_R1A@?0A@EA@QLabel@@8    100094d8     OpenCLSupportSettingsController.obj
 0002:000014f4       ??_R1A@?0A@EA@QFrame@@8    100094f4     OpenCLSupportSettingsController.obj
 0002:00001510       ??_R3QFrame@@8             10009510     OpenCLSupportSettingsController.obj
 0002:00001520       ??_R2QFrame@@8             10009520     OpenCLSupportSettingsController.obj
 0002:00001534       ??_R1A@?0A@EA@QWidget@@8   10009534     OpenCLSupportSettingsController.obj
 0002:00001550       ??_R3QWidget@@8            10009550     OpenCLSupportSettingsController.obj
 0002:00001560       ??_R2QWidget@@8            10009560     OpenCLSupportSettingsController.obj
 0002:00001570       ??_R17?0A@EA@QPaintDevice@@8 10009570     OpenCLSupportSettingsController.obj
 0002:0000158c       ??_R3QPaintDevice@@8       1000958c     OpenCLSupportSettingsController.obj
 0002:0000159c       ??_R2QPaintDevice@@8       1000959c     OpenCLSupportSettingsController.obj
 0002:000015a4       ??_R1A@?0A@EA@QPaintDevice@@8 100095a4     OpenCLSupportSettingsController.obj
 0002:000015c0       ??_R4QLabel@@6BQPaintDevice@@@ 100095c0     OpenCLSupportSettingsController.obj
 0002:000015d4       ??_R4QHBoxLayout@@6BQObject@@@ 100095d4     OpenCLSupportSettingsController.obj
 0002:000015e8       ??_R3QHBoxLayout@@8        100095e8     OpenCLSupportSettingsController.obj
 0002:000015f8       ??_R2QHBoxLayout@@8        100095f8     OpenCLSupportSettingsController.obj
 0002:00001610       ??_R1A@?0A@EA@QHBoxLayout@@8 10009610     OpenCLSupportSettingsController.obj
 0002:0000162c       ??_R1A@?0A@EA@QBoxLayout@@8 1000962c     OpenCLSupportSettingsController.obj
 0002:00001648       ??_R3QBoxLayout@@8         10009648     OpenCLSupportSettingsController.obj
 0002:00001658       ??_R2QBoxLayout@@8         10009658     OpenCLSupportSettingsController.obj
 0002:0000166c       ??_R1A@?0A@EA@QLayout@@8   1000966c     OpenCLSupportSettingsController.obj
 0002:00001688       ??_R3QLayout@@8            10009688     OpenCLSupportSettingsController.obj
 0002:00001698       ??_R2QLayout@@8            10009698     OpenCLSupportSettingsController.obj
 0002:000016a8       ??_R17?0A@EA@QLayoutItem@@8 100096a8     OpenCLSupportSettingsController.obj
 0002:000016c4       ??_R3QLayoutItem@@8        100096c4     OpenCLSupportSettingsController.obj
 0002:000016d4       ??_R2QLayoutItem@@8        100096d4     OpenCLSupportSettingsController.obj
 0002:000016dc       ??_R1A@?0A@EA@QLayoutItem@@8 100096dc     OpenCLSupportSettingsController.obj
 0002:000016f8       ??_R4QHBoxLayout@@6BQLayoutItem@@@ 100096f8     OpenCLSupportSettingsController.obj
 0002:0000170c       ??_R4QVBoxLayout@@6BQObject@@@ 1000970c     OpenCLSupportSettingsController.obj
 0002:00001720       ??_R3QVBoxLayout@@8        10009720     OpenCLSupportSettingsController.obj
 0002:00001730       ??_R2QVBoxLayout@@8        10009730     OpenCLSupportSettingsController.obj
 0002:00001748       ??_R1A@?0A@EA@QVBoxLayout@@8 10009748     OpenCLSupportSettingsController.obj
 0002:00001764       ??_R4QVBoxLayout@@6BQLayoutItem@@@ 10009764     OpenCLSupportSettingsController.obj
 0002:00001778       ??_R4QCheckBox@@6BQObject@@@ 10009778     OpenCLSupportSettingsController.obj
 0002:0000178c       ??_R3QCheckBox@@8          1000978c     OpenCLSupportSettingsController.obj
 0002:0000179c       ??_R2QCheckBox@@8          1000979c     OpenCLSupportSettingsController.obj
 0002:000017b4       ??_R1A@?0A@EA@QCheckBox@@8 100097b4     OpenCLSupportSettingsController.obj
 0002:000017d0       ??_R1A@?0A@EA@QAbstractButton@@8 100097d0     OpenCLSupportSettingsController.obj
 0002:000017ec       ??_R3QAbstractButton@@8    100097ec     OpenCLSupportSettingsController.obj
 0002:000017fc       ??_R2QAbstractButton@@8    100097fc     OpenCLSupportSettingsController.obj
 0002:00001810       ??_R4QCheckBox@@6BQPaintDevice@@@ 10009810     OpenCLSupportSettingsController.obj
 0002:00001824       ??_R4OpenCLSupportSettingsPageController@U2@@6B@ 10009824     OpenCLSupportSettingsController.obj
 0002:00001838       ??_R3OpenCLSupportSettingsPageController@U2@@8 10009838     OpenCLSupportSettingsController.obj
 0002:00001848       ??_R2OpenCLSupportSettingsPageController@U2@@8 10009848     OpenCLSupportSettingsController.obj
 0002:00001858       ??_R1A@?0A@EA@OpenCLSupportSettingsPageController@U2@@8 10009858     OpenCLSupportSettingsController.obj
 0002:00001874       ??_R1A@?0A@EA@AppSettingsGUIPageController@U2@@8 10009874     OpenCLSupportSettingsController.obj
 0002:00001890       ??_R3AppSettingsGUIPageController@U2@@8 10009890     OpenCLSupportSettingsController.obj
 0002:000018a0       ??_R2AppSettingsGUIPageController@U2@@8 100098a0     OpenCLSupportSettingsController.obj
 0002:000018ac       ??_R4OpenCLSupportSettingsPageState@U2@@6B@ 100098ac     OpenCLSupportSettingsController.obj
 0002:000018c0       ??_R3OpenCLSupportSettingsPageState@U2@@8 100098c0     OpenCLSupportSettingsController.obj
 0002:000018d0       ??_R2OpenCLSupportSettingsPageState@U2@@8 100098d0     OpenCLSupportSettingsController.obj
 0002:000018e0       ??_R1A@?0A@EA@OpenCLSupportSettingsPageState@U2@@8 100098e0     OpenCLSupportSettingsController.obj
 0002:000018fc       ??_R1A@?0A@EA@AppSettingsGUIPageState@U2@@8 100098fc     OpenCLSupportSettingsController.obj
 0002:00001918       ??_R3AppSettingsGUIPageState@U2@@8 10009918     OpenCLSupportSettingsController.obj
 0002:00001928       ??_R2AppSettingsGUIPageState@U2@@8 10009928     OpenCLSupportSettingsController.obj
 0002:00001934       ??_R4OpenCLSupportSettingsPageWidget@U2@@6BQObject@@@ 10009934     OpenCLSupportSettingsController.obj
 0002:00001948       ??_R3OpenCLSupportSettingsPageWidget@U2@@8 10009948     OpenCLSupportSettingsController.obj
 0002:00001958       ??_R2OpenCLSupportSettingsPageWidget@U2@@8 10009958     OpenCLSupportSettingsController.obj
 0002:00001970       ??_R1A@?0A@EA@OpenCLSupportSettingsPageWidget@U2@@8 10009970     OpenCLSupportSettingsController.obj
 0002:0000198c       ??_R1A@?0A@EA@AppSettingsGUIPageWidget@U2@@8 1000998c     OpenCLSupportSettingsController.obj
 0002:000019a8       ??_R3AppSettingsGUIPageWidget@U2@@8 100099a8     OpenCLSupportSettingsController.obj
 0002:000019b8       ??_R2AppSettingsGUIPageWidget@U2@@8 100099b8     OpenCLSupportSettingsController.obj
 0002:000019cc       ??_R4OpenCLSupportSettingsPageWidget@U2@@6BQPaintDevice@@@ 100099cc     OpenCLSupportSettingsController.obj
 0002:000019e0       ??_R4type_info@@6B@        100099e0     MSVCRT:ti_inst.obj
 0002:000019f4       ??_R3type_info@@8          100099f4     MSVCRT:ti_inst.obj
 0002:00001a04       ??_R2type_info@@8          10009a04     MSVCRT:ti_inst.obj
 0002:00001a0c       ??_R1A@?0A@EA@type_info@@8 10009a0c     MSVCRT:ti_inst.obj
 0002:00001a30       ___safe_se_handler_table   10009a30     <linker-defined>
 0002:00001af8       ___rtc_iaa                 10009af8     MSVCRT:initsect.obj
 0002:00001afc       ___rtc_izz                 10009afc     MSVCRT:initsect.obj
 0002:00001b00       ___rtc_taa                 10009b00     MSVCRT:initsect.obj
 0002:00001b04       ___rtc_tzz                 10009b04     MSVCRT:initsect.obj
 0002:000029cc       __IMPORT_DESCRIPTOR_U2Core 1000a9cc     U2Core:U2Core.dll
 0002:000029e0       __IMPORT_DESCRIPTOR_U2Algorithm 1000a9e0     U2Algorithm:U2Algorithm.dll
 0002:000029f4       __IMPORT_DESCRIPTOR_U2Gui  1000a9f4     U2Gui:U2Gui.dll
 0002:00002a08       __IMPORT_DESCRIPTOR_Qt5Widgets 1000aa08     Qt5Widgets:Qt5Widgets.dll
 0002:00002a1c       __IMPORT_DESCRIPTOR_Qt5Core 1000aa1c     Qt5Core:Qt5Core.dll
 0002:00002a30       __IMPORT_DESCRIPTOR_MSVCP120 1000aa30     msvcprt:MSVCP120.dll
 0002:00002a44       __IMPORT_DESCRIPTOR_MSVCR120 1000aa44     MSVCRT:MSVCR120.dll
 0002:00002a58       __IMPORT_DESCRIPTOR_KERNEL32 1000aa58     kernel32:KERNEL32.dll
 0002:00002a6c       __NULL_IMPORT_DESCRIPTOR   1000aa6c     U2Core:U2Core.dll
 0003:00000004       ?_Generic_object@?$_Error_objects@H@std@@2V_Generic_error_category@2@A 1000e004     OpenCLSupportPlugin.obj
 0003:00000008       ?_Iostream_object@?$_Error_objects@H@std@@2V_Iostream_error_category@2@A 1000e008     OpenCLSupportPlugin.obj
 0003:0000000c       ?_System_object@?$_Error_objects@H@std@@2V_System_error_category@2@A 1000e00c     OpenCLSupportPlugin.obj
 0003:00000018       ?staticMetaObject@OpenCLSupportPlugin@U2@@2UQMetaObject@@B 1000e018     moc_OpenCLSupportPlugin.obj
 0003:00000030       ?staticMetaObject@OpenCLSupportSettingsPageController@U2@@2UQMetaObject@@B 1000e030     moc_OpenCLSupportSettingsController.obj
 0003:00000048       ?staticMetaObject@OpenCLSupportSettingsPageState@U2@@2UQMetaObject@@B 1000e048     moc_OpenCLSupportSettingsController.obj
 0003:00000060       ?staticMetaObject@OpenCLSupportSettingsPageWidget@U2@@2UQMetaObject@@B 1000e060     moc_OpenCLSupportSettingsController.obj
 0003:00000078       ___security_cookie         1000e078     MSVCRT:gs_cookie.obj
 0003:0000007c       ___security_cookie_complement 1000e07c     MSVCRT:gs_cookie.obj
 0003:00000080       ___native_dllmain_reason   1000e080     MSVCRT:natstart.obj
 0003:00000084       ??_R0?AVerror_category@std@@@8 1000e084     OpenCLSupportPlugin.obj
 0003:000000a8       ??_R0?AV_Generic_error_category@std@@@8 1000e0a8     OpenCLSupportPlugin.obj
 0003:000000d4       ??_R0?AV_Iostream_error_category@std@@@8 1000e0d4     OpenCLSupportPlugin.obj
 0003:00000100       ??_R0?AV_System_error_category@std@@@8 1000e100     OpenCLSupportPlugin.obj
 0003:0000012c       ??_R0?AVAppResourceSemaphore@U2@@@8 1000e12c     OpenCLSupportPlugin.obj
 0003:00000154       ??_R0?AVAppResource@U2@@@8 1000e154     OpenCLSupportPlugin.obj
 0003:00000174       ??_R0?AVOpenCLSupportPlugin@U2@@@8 1000e174     OpenCLSupportPlugin.obj
 0003:0000019c       ??_R0?AVPlugin@U2@@@8      1000e19c     OpenCLSupportPlugin.obj
 0003:000001b4       ??_R0?AVQObject@@@8        1000e1b4     OpenCLSupportPlugin.obj
 0003:000001cc       ??_R0?AVQLabel@@@8         1000e1cc     OpenCLSupportSettingsController.obj
 0003:000001e4       ??_R0?AVQFrame@@@8         1000e1e4     OpenCLSupportSettingsController.obj
 0003:000001fc       ??_R0?AVQWidget@@@8        1000e1fc     OpenCLSupportSettingsController.obj
 0003:00000214       ??_R0?AVQPaintDevice@@@8   1000e214     OpenCLSupportSettingsController.obj
 0003:00000230       ??_R0?AVQHBoxLayout@@@8    1000e230     OpenCLSupportSettingsController.obj
 0003:0000024c       ??_R0?AVQBoxLayout@@@8     1000e24c     OpenCLSupportSettingsController.obj
 0003:00000268       ??_R0?AVQLayout@@@8        1000e268     OpenCLSupportSettingsController.obj
 0003:00000280       ??_R0?AVQLayoutItem@@@8    1000e280     OpenCLSupportSettingsController.obj
 0003:0000029c       ??_R0?AVQVBoxLayout@@@8    1000e29c     OpenCLSupportSettingsController.obj
 0003:000002b8       ??_R0?AVQCheckBox@@@8      1000e2b8     OpenCLSupportSettingsController.obj
 0003:000002d0       ??_R0?AVQAbstractButton@@@8 1000e2d0     OpenCLSupportSettingsController.obj
 0003:000002f0       ??_R0?AVOpenCLSupportSettingsPageController@U2@@@8 1000e2f0     OpenCLSupportSettingsController.obj
 0003:00000328       ??_R0?AVAppSettingsGUIPageController@U2@@@8 1000e328     OpenCLSupportSettingsController.obj
 0003:00000358       ??_R0?AVOpenCLSupportSettingsPageState@U2@@@8 1000e358     OpenCLSupportSettingsController.obj
 0003:00000388       ??_R0?AVAppSettingsGUIPageState@U2@@@8 1000e388     OpenCLSupportSettingsController.obj
 0003:000003b4       ??_R0?AVOpenCLSupportSettingsPageWidget@U2@@@8 1000e3b4     OpenCLSupportSettingsController.obj
 0003:000003e8       ??_R0?AVAppSettingsGUIPageWidget@U2@@@8 1000e3e8     OpenCLSupportSettingsController.obj
 0003:00000414       ??_R0?AVtype_info@@@8      1000e414     MSVCRT:ti_inst.obj
 0003:0000047c       ?id@?$num_put@DV?$back_insert_iterator@V?$basic_string@DU?$char_traits@D@std@@V?$allocator@D@2@@std@@@std@@@std@@2V0locale@2@A 1000e47c     OpenCLSupportPlugin.obj
 0003:00000480       ?id@?$num_put@_WV?$back_insert_iterator@V?$basic_string@_WU?$char_traits@_W@std@@V?$allocator@_W@2@@std@@@std@@@std@@2V0locale@2@A 1000e480     OpenCLSupportPlugin.obj
 0003:000004d0       ?helpPageId@OpenCLSupportSettingsPageController@U2@@0VQString@@B 1000e4d0     OpenCLSupportSettingsController.obj
 0003:00000800       ?__type_info_root_node@@3U__type_info_node@@A 1000e800     MSVCRT:tncleanup.obj
 0003:00000808       ___native_startup_lock     1000e808     <common>
 0003:0000080c       ___native_startup_state    1000e80c     <common>
 0003:00000810       ___dyn_tls_init_callback   1000e810     <common>
 0003:00000814       ___onexitend               1000e814     <common>
 0003:00000818       ___onexitbegin             1000e818     <common>

 entry point at        0001:00005986

 Static symbols

 0000:fffee000       .debug$S                   10000000     MSVCRT:MSVCR120.dll
 0000:fffee000       .debug$S                   10000000     MSVCRT:MSVCR120.dll
 0000:fffee000       .debug$S                   10000000     MSVCRT:MSVCR120.dll
 0000:fffee000       .debug$S                   10000000     MSVCRT:MSVCR120.dll
 0000:fffee000       .debug$S                   10000000     MSVCRT:MSVCR120.dll
 0000:fffee000       .debug$S                   10000000     MSVCRT:MSVCR120.dll
 0000:fffee000       .debug$S                   10000000     MSVCRT:MSVCR120.dll
 0000:fffee000       .debug$S                   10000000     MSVCRT:MSVCR120.dll
 0000:fffee000       .debug$S                   10000000     MSVCRT:MSVCR120.dll
 0000:fffee000       .debug$S                   10000000     MSVCRT:MSVCR120.dll
 0000:fffee000       .debug$S                   10000000     MSVCRT:MSVCR120.dll
 0000:fffee000       .debug$S                   10000000     MSVCRT:MSVCR120.dll
 0000:fffee000       .debug$S                   10000000     MSVCRT:MSVCR120.dll
 0000:fffee000       .debug$S                   10000000     MSVCRT:MSVCR120.dll
 0000:fffee000       .debug$S                   10000000     MSVCRT:MSVCR120.dll
 0000:fffee000       .debug$S                   10000000     U2Core:U2Core.dll
 0000:fffee000       .debug$S                   10000000     U2Core:U2Core.dll
 0000:fffee000       .debug$S                   10000000     U2Core:U2Core.dll
 0000:fffee000       .debug$S                   10000000     U2Core:U2Core.dll
 0000:fffee000       .debug$S                   10000000     MSVCRT:MSVCR120.dll
 0000:fffee000       .debug$S                   10000000     U2Core:U2Core.dll
 0000:fffee000       .debug$S                   10000000     MSVCRT:MSVCR120.dll
 0000:fffee000       .debug$S                   10000000     U2Core:U2Core.dll
 0000:fffee000       .debug$S                   10000000     MSVCRT:MSVCR120.dll
 0001:fffff000       __ehhandler$?_Copy@?$basic_string@DU?$char_traits@D@std@@V?$allocator@D@2@@std@@QAEXII@Z 10000000 f   moc_OpenCLSupportSettingsController.obj
 0000:fffee000       .debug$S                   10000000     U2Core:U2Core.dll
 0000:fffee000       .debug$S                   10000000     U2Core:U2Core.dll
 0000:fffee000       .debug$S                   10000000     U2Core:U2Core.dll
 0000:fffee000       .debug$S                   10000000     U2Core:U2Core.dll
 0000:fffee000       .debug$S                   10000000     U2Core:U2Core.dll
 0000:fffee000       .debug$S                   10000000     U2Core:U2Core.dll
 0002:ffff8000       __catchsym$?_Copy@?$basic_string@DU?$char_traits@D@std@@V?$allocator@D@2@@std@@QAEXII@Z$5 10000000     moc_OpenCLSupportSettingsController.obj
 0000:fffee000       .debug$S                   10000000     MSVCRT:MSVCR120.dll
 0000:fffee000       .debug$S                   10000000     MSVCRT:MSVCR120.dll
 0000:fffee000       .debug$S                   10000000     MSVCRT:MSVCR120.dll
 0000:fffee000       .debug$S                   10000000     MSVCRT:MSVCR120.dll
 0000:fffee000       .debug$S                   10000000     MSVCRT:MSVCR120.dll
 0000:fffee000       .debug$S                   10000000     MSVCRT:MSVCR120.dll
 0000:fffee000       .debug$S                   10000000     MSVCRT:MSVCR120.dll
 0002:ffff8000       ?_Generic_object$initializer$@?$_Error_objects@H@std@@2P6AXXZA 10000000     moc_OpenCLSupportSettingsController.obj
 0002:ffff8000       ?_Iostream_object$initializer$@?$_Error_objects@H@std@@2P6AXXZA 10000000     moc_OpenCLSupportSettingsController.obj
 0002:ffff8000       ?_System_object$initializer$@?$_Error_objects@H@std@@2P6AXXZA 10000000     moc_OpenCLSupportSettingsController.obj
 0000:fffee000       .debug$S                   10000000     MSVCRT:MSVCR120.dll
 0000:fffee000       .debug$S                   10000000     MSVCRT:MSVCR120.dll
 0000:fffee000       .debug$S                   10000000     U2Core:U2Core.dll
 0000:fffee000       .debug$S                   10000000     U2Core:U2Core.dll
 0000:fffee000       .debug$S                   10000000     MSVCRT:MSVCR120.dll
 0000:fffee000       .debug$S                   10000000     U2Core:U2Core.dll
 0000:fffee000       .debug$S                   10000000     MSVCRT:MSVCR120.dll
 0000:fffee000       .debug$S                   10000000     U2Core:U2Core.dll
 0000:fffee000       .debug$S                   10000000     MSVCRT:MSVCR120.dll
 0001:fffff000       __ehhandler$?_Copy@?$basic_string@DU?$char_traits@D@std@@V?$allocator@D@2@@std@@QAEXII@Z 10000000 f   moc_OpenCLSupportPlugin.obj
 0000:fffee000       .debug$S                   10000000     U2Core:U2Core.dll
 0000:fffee000       .debug$S                   10000000     U2Core:U2Core.dll
 0000:fffee000       .debug$S                   10000000     U2Core:U2Core.dll
 0000:fffee000       .debug$S                   10000000     U2Core:U2Core.dll
 0000:fffee000       .debug$S                   10000000     U2Core:U2Core.dll
 0000:fffee000       .debug$S                   10000000     U2Core:U2Core.dll
 0002:ffff8000       __catchsym$?_Copy@?$basic_string@DU?$char_traits@D@std@@V?$allocator@D@2@@std@@QAEXII@Z$5 10000000     moc_OpenCLSupportPlugin.obj
 0000:fffee000       .debug$S                   10000000     U2Core:U2Core.dll
 0000:fffee000       .debug$S                   10000000     U2Core:U2Core.dll
 0000:fffee000       .debug$S                   10000000     U2Algorithm:U2Algorithm.dll
 0000:fffee000       .debug$S                   10000000     U2Algorithm:U2Algorithm.dll
 0000:fffee000       .debug$S                   10000000     msvcprt:MSVCP120.dll
 0002:ffff8000       ?_Generic_object$initializer$@?$_Error_objects@H@std@@2P6AXXZA 10000000     moc_OpenCLSupportPlugin.obj
 0002:ffff8000       ?_Iostream_object$initializer$@?$_Error_objects@H@std@@2P6AXXZA 10000000     moc_OpenCLSupportPlugin.obj
 0002:ffff8000       ?_System_object$initializer$@?$_Error_objects@H@std@@2P6AXXZA 10000000     moc_OpenCLSupportPlugin.obj
 0000:fffee000       .debug$S                   10000000     msvcprt:MSVCP120.dll
 0000:fffee000       .debug$S                   10000000     msvcprt:MSVCP120.dll
 0000:fffee000       .debug$S                   10000000     U2Algorithm:U2Algorithm.dll
 0000:fffee000       .debug$S                   10000000     msvcprt:MSVCP120.dll
 0000:fffee000       .debug$S                   10000000     U2Algorithm:U2Algorithm.dll
 0000:fffee000       .debug$S                   10000000     msvcprt:MSVCP120.dll
 0000:fffee000       .debug$S                   10000000     U2Algorithm:U2Algorithm.dll
 0000:fffee000       .debug$S                   10000000     kernel32:KERNEL32.dll
 0000:fffee000       .debug$S                   10000000     U2Algorithm:U2Algorithm.dll
 0000:fffee000       .debug$S                   10000000     kernel32:KERNEL32.dll
 0000:fffee000       .debug$S                   10000000     U2Algorithm:U2Algorithm.dll
 0000:fffee000       .debug$S                   10000000     kernel32:KERNEL32.dll
 0000:fffee000       .debug$S                   10000000     U2Algorithm:U2Algorithm.dll
 0000:fffee000       .debug$S                   10000000     kernel32:KERNEL32.dll
 0000:fffee000       .debug$S                   10000000     U2Gui:U2Gui.dll
 0000:fffee000       .debug$S                   10000000     kernel32:KERNEL32.dll
 0000:fffee000       .debug$S                   10000000     U2Gui:U2Gui.dll
 0000:fffee000       .debug$S                   10000000     kernel32:KERNEL32.dll
 0000:fffee000       .debug$S                   10000000     U2Gui:U2Gui.dll
 0000:fffee000       .debug$S                   10000000     kernel32:KERNEL32.dll
 0000:fffee000       .debug$S                   10000000     U2Gui:U2Gui.dll
 0000:fffee000       .debug$S                   10000000     kernel32:KERNEL32.dll
 0000:fffee000       .debug$S                   10000000     U2Gui:U2Gui.dll
 0000:fffee000       .debug$S                   10000000     kernel32:KERNEL32.dll
 0000:fffee000       .debug$S                   10000000     U2Gui:U2Gui.dll
 0000:fffee000       .debug$S                   10000000     Qt5Core:Qt5Core.dll
 0000:fffee000       .debug$S                   10000000     U2Gui:U2Gui.dll
 0000:fffee000       .debug$S                   10000000     Qt5Core:Qt5Core.dll
 0001:fffff000       __ehhandler$?_Copy@?$basic_string@DU?$char_traits@D@std@@V?$allocator@D@2@@std@@QAEXII@Z 10000000 f   OpenCLSupportSettingsController.obj
 0000:fffee000       .debug$S                   10000000     U2Gui:U2Gui.dll
 0000:fffee000       .debug$S                   10000000     U2Gui:U2Gui.dll
 0000:fffee000       .debug$S                   10000000     U2Gui:U2Gui.dll
 0001:fffff000       __unwindfunclet$??H@YA?BVQString@@ABV0@0@Z$0 10000000 f   OpenCLSupportSettingsController.obj
 0000:fffee000       .debug$S                   10000000     U2Gui:U2Gui.dll
 0001:fffff000       __unwindfunclet$??H@YA?BVQString@@ABV0@PBD@Z$0 10000000 f   OpenCLSupportSettingsController.obj
 0000:fffee000       .debug$S                   10000000     U2Gui:U2Gui.dll
 0000:fffee000       .debug$S                   10000000     Qt5Core:Qt5Core.dll
 0000:fffee000       .debug$S                   10000000     Qt5Core:Qt5Core.dll
 0000:fffee000       .debug$S                   10000000     Qt5Core:Qt5Core.dll
 0000:fffee000       .debug$S                   10000000     Qt5Core:Qt5Core.dll
 0000:fffee000       .debug$S                   10000000     Qt5Core:Qt5Core.dll
 0000:fffee000       .debug$S                   10000000     Qt5Core:Qt5Core.dll
 0000:fffee000       .debug$S                   10000000     Qt5Core:Qt5Core.dll
 0000:fffee000       .debug$S                   10000000     Qt5Core:Qt5Core.dll
 0000:fffee000       .debug$S                   10000000     Qt5Core:Qt5Core.dll
 0000:fffee000       .debug$S                   10000000     Qt5Core:Qt5Core.dll
 0000:fffee000       .debug$S                   10000000     Qt5Core:Qt5Core.dll
 0000:fffee000       .debug$S                   10000000     Qt5Core:Qt5Core.dll
 0000:fffee000       .debug$S                   10000000     Qt5Core:Qt5Core.dll
 0000:fffee000       .debug$S                   10000000     Qt5Core:Qt5Core.dll
 0000:fffee000       .debug$S                   10000000     Qt5Core:Qt5Core.dll
 0000:fffee000       .debug$S                   10000000     Qt5Core:Qt5Core.dll
 0000:fffee000       .debug$S                   10000000     Qt5Core:Qt5Core.dll
 0000:fffee000       .debug$S                   10000000     Qt5Core:Qt5Core.dll
 0000:fffee000       .debug$S                   10000000     Qt5Core:Qt5Core.dll
 0000:fffee000       .debug$S                   10000000     Qt5Core:Qt5Core.dll
 0000:fffee000       .debug$S                   10000000     Qt5Core:Qt5Core.dll
 0000:fffee000       .debug$S                   10000000     Qt5Core:Qt5Core.dll
 0000:fffee000       .debug$S                   10000000     Qt5Core:Qt5Core.dll
 0000:fffee000       .debug$S                   10000000     Qt5Core:Qt5Core.dll
 0000:fffee000       .debug$S                   10000000     Qt5Core:Qt5Core.dll
 0000:fffee000       .debug$S                   10000000     Qt5Core:Qt5Core.dll
 0000:fffee000       .debug$S                   10000000     Qt5Core:Qt5Core.dll
 0000:fffee000       .debug$S                   10000000     Qt5Core:Qt5Core.dll
 0000:fffee000       .debug$S                   10000000     Qt5Core:Qt5Core.dll
 0000:fffee000       .debug$S                   10000000     Qt5Core:Qt5Core.dll
 0000:fffee000       .debug$S                   10000000     Qt5Core:Qt5Core.dll
 0000:fffee000       .debug$S                   10000000     Qt5Core:Qt5Core.dll
 0000:fffee000       .debug$S                   10000000     Qt5Core:Qt5Core.dll
 0000:fffee000       .debug$S                   10000000     Qt5Core:Qt5Core.dll
 0000:fffee000       .debug$S                   10000000     Qt5Core:Qt5Core.dll
 0000:fffee000       .debug$S                   10000000     Qt5Core:Qt5Core.dll
 0000:fffee000       .debug$S                   10000000     Qt5Core:Qt5Core.dll
 0000:fffee000       .debug$S                   10000000     U2Gui:U2Gui.dll
 0000:fffee000       .debug$S                   10000000     U2Gui:U2Gui.dll
 0000:fffee000       .debug$S                   10000000     Qt5Core:Qt5Core.dll
 0000:fffee000       .debug$S                   10000000     Qt5Core:Qt5Core.dll
 0000:fffee000       .debug$S                   10000000     Qt5Widgets:Qt5Widgets.dll
 0000:fffee000       .debug$S                   10000000     Qt5Widgets:Qt5Widgets.dll
 0000:fffee000       .debug$S                   10000000     Qt5Widgets:Qt5Widgets.dll
 0000:fffee000       .debug$S                   10000000     Qt5Widgets:Qt5Widgets.dll
 0000:fffee000       .debug$S                   10000000     Qt5Widgets:Qt5Widgets.dll
 0000:fffee000       .debug$S                   10000000     Qt5Widgets:Qt5Widgets.dll
 0000:fffee000       .debug$S                   10000000     Qt5Widgets:Qt5Widgets.dll
 0000:fffee000       .debug$S                   10000000     Qt5Widgets:Qt5Widgets.dll
 0000:fffee000       .debug$S                   10000000     Qt5Widgets:Qt5Widgets.dll
 0000:fffee000       .debug$S                   10000000     Qt5Widgets:Qt5Widgets.dll
 0000:fffee000       .debug$S                   10000000     Qt5Widgets:Qt5Widgets.dll
 0000:fffee000       .debug$S                   10000000     Qt5Widgets:Qt5Widgets.dll
 0000:fffee000       .debug$S                   10000000     Qt5Widgets:Qt5Widgets.dll
 0000:fffee000       .debug$S                   10000000     Qt5Widgets:Qt5Widgets.dll
 0000:fffee000       .debug$S                   10000000     Qt5Widgets:Qt5Widgets.dll
 0000:fffee000       .debug$S                   10000000     Qt5Widgets:Qt5Widgets.dll
 0000:fffee000       .debug$S                   10000000     Qt5Widgets:Qt5Widgets.dll
 0000:fffee000       .debug$S                   10000000     Qt5Widgets:Qt5Widgets.dll
 0000:fffee000       .debug$S                   10000000     Qt5Widgets:Qt5Widgets.dll
 0000:fffee000       .debug$S                   10000000     Qt5Widgets:Qt5Widgets.dll
 0000:fffee000       .debug$S                   10000000     Qt5Widgets:Qt5Widgets.dll
 0000:fffee000       .debug$S                   10000000     Qt5Widgets:Qt5Widgets.dll
 0000:fffee000       .debug$S                   10000000     Qt5Widgets:Qt5Widgets.dll
 0000:fffee000       .debug$S                   10000000     Qt5Widgets:Qt5Widgets.dll
 0000:fffee000       .debug$S                   10000000     Qt5Widgets:Qt5Widgets.dll
 0000:fffee000       .debug$S                   10000000     Qt5Widgets:Qt5Widgets.dll
 0000:fffee000       .debug$S                   10000000     Qt5Widgets:Qt5Widgets.dll
 0000:fffee000       .debug$S                   10000000     Qt5Widgets:Qt5Widgets.dll
 0000:fffee000       .debug$S                   10000000     Qt5Widgets:Qt5Widgets.dll
 0000:fffee000       .debug$S                   10000000     Qt5Widgets:Qt5Widgets.dll
 0000:fffee000       .debug$S                   10000000     Qt5Widgets:Qt5Widgets.dll
 0000:fffee000       .debug$S                   10000000     Qt5Widgets:Qt5Widgets.dll
 0000:fffee000       .debug$S                   10000000     Qt5Widgets:Qt5Widgets.dll
 0000:fffee000       .debug$S                   10000000     Qt5Widgets:Qt5Widgets.dll
 0000:fffee000       .debug$S                   10000000     Qt5Widgets:Qt5Widgets.dll
 0001:fffff000       __ehhandler$??0?$QList@PAVOpenCLGpuModel@U2@@@@QAE@ABV0@@Z 10000000 f   OpenCLSupportSettingsController.obj
 0000:fffee000       .debug$S                   10000000     Qt5Widgets:Qt5Widgets.dll
 0000:fffee000       .debug$S                   10000000     Qt5Widgets:Qt5Widgets.dll
 0000:fffee000       .debug$S                   10000000     Qt5Widgets:Qt5Widgets.dll
 0002:ffff8000       ?_System_object$initializer$@?$_Error_objects@H@std@@2P6AXXZA 10000000     OpenCLSupportSettingsController.obj
 0002:ffff8000       ?_Iostream_object$initializer$@?$_Error_objects@H@std@@2P6AXXZA 10000000     OpenCLSupportSettingsController.obj
 0002:ffff8000       ?_Generic_object$initializer$@?$_Error_objects@H@std@@2P6AXXZA 10000000     OpenCLSupportSettingsController.obj
 0000:fffee000       .debug$S                   10000000     Qt5Widgets:Qt5Widgets.dll
 0002:ffff8000       __catchsym$?_Copy@?$basic_string@DU?$char_traits@D@std@@V?$allocator@D@2@@std@@QAEXII@Z$5 10000000     OpenCLSupportSettingsController.obj
 0000:fffee000       .debug$S                   10000000     Qt5Widgets:Qt5Widgets.dll
 0002:ffff8000       __unwindtable$??H@YA?BVQString@@ABV0@0@Z 10000000     OpenCLSupportSettingsController.obj
 0000:fffee000       .debug$S                   10000000     Qt5Widgets:Qt5Widgets.dll
 0002:ffff8000       __unwindtable$??H@YA?BVQString@@ABV0@PBD@Z 10000000     OpenCLSupportSettingsController.obj
 0000:fffee000       .debug$S                   10000000     Qt5Widgets:Qt5Widgets.dll
 0000:fffee000       .debug$S                   10000000     Qt5Widgets:Qt5Widgets.dll
 0000:fffee000       .debug$S                   10000000     Qt5Widgets:Qt5Widgets.dll
 0000:fffee000       .debug$S                   10000000     Qt5Widgets:Qt5Widgets.dll
 0000:fffee000       .debug$S                   10000000     Qt5Widgets:Qt5Widgets.dll
 0000:fffee000       .debug$S                   10000000     Qt5Widgets:Qt5Widgets.dll
 0000:fffee000       .debug$S                   10000000     Qt5Widgets:Qt5Widgets.dll
 0000:fffee000       .debug$S                   10000000     Qt5Widgets:Qt5Widgets.dll
 0000:fffee000       .debug$S                   10000000     Qt5Widgets:Qt5Widgets.dll
 0000:fffee000       .debug$S                   10000000     Qt5Widgets:Qt5Widgets.dll
 0000:fffee000       .debug$S                   10000000     Qt5Widgets:Qt5Widgets.dll
 0000:fffee000       .debug$S                   10000000     Qt5Widgets:Qt5Widgets.dll
 0000:fffee000       .debug$S                   10000000     Qt5Widgets:Qt5Widgets.dll
 0000:fffee000       .debug$S                   10000000     Qt5Widgets:Qt5Widgets.dll
 0000:fffee000       .debug$S                   10000000     Qt5Widgets:Qt5Widgets.dll
 0000:fffee000       .debug$S                   10000000     Qt5Widgets:Qt5Widgets.dll
 0000:fffee000       .debug$S                   10000000     Qt5Widgets:Qt5Widgets.dll
 0000:fffee000       .debug$S                   10000000     Qt5Widgets:Qt5Widgets.dll
 0000:fffee000       .debug$S                   10000000     Qt5Widgets:Qt5Widgets.dll
 0000:fffee000       .debug$S                   10000000     Qt5Widgets:Qt5Widgets.dll
 0000:fffee000       .debug$S                   10000000     Qt5Widgets:Qt5Widgets.dll
 0000:fffee000       .debug$S                   10000000     Qt5Widgets:Qt5Widgets.dll
 0000:fffee000       .debug$S                   10000000     Qt5Widgets:Qt5Widgets.dll
 0000:fffee000       .debug$S                   10000000     Qt5Widgets:Qt5Widgets.dll
 0000:fffee000       .debug$S                   10000000     Qt5Widgets:Qt5Widgets.dll
 0000:fffee000       .debug$S                   10000000     Qt5Widgets:Qt5Widgets.dll
 0000:fffee000       .debug$S                   10000000     Qt5Widgets:Qt5Widgets.dll
 0000:fffee000       .debug$S                   10000000     Qt5Widgets:Qt5Widgets.dll
 0000:fffee000       .debug$S                   10000000     Qt5Widgets:Qt5Widgets.dll
 0000:fffee000       .debug$S                   10000000     Qt5Widgets:Qt5Widgets.dll
 0000:fffee000       .debug$S                   10000000     Qt5Widgets:Qt5Widgets.dll
 0000:fffee000       .debug$S                   10000000     Qt5Widgets:Qt5Widgets.dll
 0000:fffee000       .debug$S                   10000000     Qt5Widgets:Qt5Widgets.dll
 0000:fffee000       .debug$S                   10000000     Qt5Widgets:Qt5Widgets.dll
 0000:fffee000       .debug$S                   10000000     Qt5Widgets:Qt5Widgets.dll
 0000:fffee000       .debug$S                   10000000     Qt5Widgets:Qt5Widgets.dll
 0000:fffee000       .debug$S                   10000000     Qt5Widgets:Qt5Widgets.dll
 0000:fffee000       .debug$S                   10000000     Qt5Widgets:Qt5Widgets.dll
 0000:fffee000       .debug$S                   10000000     Qt5Widgets:Qt5Widgets.dll
 0000:fffee000       .debug$S                   10000000     Qt5Widgets:Qt5Widgets.dll
 0000:fffee000       .debug$S                   10000000     Qt5Widgets:Qt5Widgets.dll
 0000:fffee000       .debug$S                   10000000     Qt5Widgets:Qt5Widgets.dll
 0000:fffee000       .debug$S                   10000000     Qt5Widgets:Qt5Widgets.dll
 0000:fffee000       .debug$S                   10000000     Qt5Widgets:Qt5Widgets.dll
 0000:fffee000       .debug$S                   10000000     Qt5Widgets:Qt5Widgets.dll
 0000:fffee000       .debug$S                   10000000     Qt5Widgets:Qt5Widgets.dll
 0000:fffee000       .debug$S                   10000000     Qt5Widgets:Qt5Widgets.dll
 0000:fffee000       .debug$S                   10000000     Qt5Widgets:Qt5Widgets.dll
 0000:fffee000       .debug$S                   10000000     Qt5Widgets:Qt5Widgets.dll
 0000:fffee000       .debug$S                   10000000     Qt5Widgets:Qt5Widgets.dll
 0000:fffee000       .debug$S                   10000000     Qt5Widgets:Qt5Widgets.dll
 0000:fffee000       .debug$S                   10000000     Qt5Widgets:Qt5Widgets.dll
 0000:fffee000       .debug$S                   10000000     Qt5Widgets:Qt5Widgets.dll
 0000:fffee000       .debug$S                   10000000     Qt5Widgets:Qt5Widgets.dll
 0000:fffee000       .debug$S                   10000000     Qt5Widgets:Qt5Widgets.dll
 0000:fffee000       .debug$S                   10000000     Qt5Widgets:Qt5Widgets.dll
 0000:fffee000       .debug$S                   10000000     Qt5Widgets:Qt5Widgets.dll
 0000:fffee000       .debug$S                   10000000     Qt5Widgets:Qt5Widgets.dll
 0000:fffee000       .debug$S                   10000000     Qt5Widgets:Qt5Widgets.dll
 0000:fffee000       .debug$S                   10000000     Qt5Widgets:Qt5Widgets.dll
 0000:fffee000       .debug$S                   10000000     Qt5Widgets:Qt5Widgets.dll
 0002:ffff8000       __catchsym$??0?$QList@PAVOpenCLGpuModel@U2@@@@QAE@ABV0@@Z$2 10000000     OpenCLSupportSettingsController.obj
 0000:fffee000       .debug$S                   10000000     Qt5Widgets:Qt5Widgets.dll
 0000:fffee000       .debug$S                   10000000     Qt5Widgets:Qt5Widgets.dll
 0000:fffee000       .debug$S                   10000000     Qt5Widgets:Qt5Widgets.dll
 0000:fffee000       .debug$S                   10000000     Qt5Widgets:Qt5Widgets.dll
 0000:fffee000       .debug$S                   10000000     Qt5Widgets:Qt5Widgets.dll
 0000:fffee000       .debug$S                   10000000     Qt5Widgets:Qt5Widgets.dll
 0000:fffee000       .debug$S                   10000000     Qt5Widgets:Qt5Widgets.dll
 0000:fffee000       .debug$S                   10000000     Qt5Widgets:Qt5Widgets.dll
 0000:fffee000       .debug$S                   10000000     Qt5Widgets:Qt5Widgets.dll
 0000:fffee000       .debug$S                   10000000     Qt5Widgets:Qt5Widgets.dll
 0000:fffee000       .debug$S                   10000000     Qt5Widgets:Qt5Widgets.dll
 0000:fffee000       .debug$S                   10000000     Qt5Widgets:Qt5Widgets.dll
 0000:fffee000       .debug$S                   10000000     Qt5Widgets:Qt5Widgets.dll
 0000:fffee000       .debug$S                   10000000     Qt5Widgets:Qt5Widgets.dll
 0000:fffee000       .debug$S                   10000000     Qt5Widgets:Qt5Widgets.dll
 0000:fffee000       .debug$S                   10000000     Qt5Widgets:Qt5Widgets.dll
 0000:fffee000       .debug$S                   10000000     Qt5Widgets:Qt5Widgets.dll
 0000:fffee000       .debug$S                   10000000     Qt5Widgets:Qt5Widgets.dll
 0000:fffee000       .debug$S                   10000000     Qt5Widgets:Qt5Widgets.dll
 0000:fffee000       .debug$S                   10000000     Qt5Widgets:Qt5Widgets.dll
 0000:fffee000       .debug$S                   10000000     Qt5Widgets:Qt5Widgets.dll
 0000:fffee000       .debug$S                   10000000     U2Core:U2Core.dll
 0002:ffff8008       __ehfuncinfo$??H@YA?BVQString@@ABV0@0@Z 10000008     OpenCLSupportSettingsController.obj
 0002:ffff8010       __ehfuncinfo$??H@YA?BVQString@@ABV0@PBD@Z 10000010     OpenCLSupportSettingsController.obj
 0002:ffff8010       __catchsym$?_Copy@?$basic_string@DU?$char_traits@D@std@@V?$allocator@D@2@@std@@QAEXII@Z$4 10000010     moc_OpenCLSupportPlugin.obj
 0002:ffff8010       __unwindtable$??0?$QList@PAVOpenCLGpuModel@U2@@@@QAE@ABV0@@Z 10000010     OpenCLSupportSettingsController.obj
 0002:ffff8010       __catchsym$?_Copy@?$basic_string@DU?$char_traits@D@std@@V?$allocator@D@2@@std@@QAEXII@Z$4 10000010     OpenCLSupportSettingsController.obj
 0002:ffff8010       __catchsym$?_Copy@?$basic_string@DU?$char_traits@D@std@@V?$allocator@D@2@@std@@QAEXII@Z$4 10000010     moc_OpenCLSupportSettingsController.obj
 0001:fffff01a       __ehhandler$??H@YA?BVQString@@ABV0@0@Z 1000001a f   OpenCLSupportSettingsController.obj
 0001:fffff01a       __unwindfunclet$??H@YA?BVQString@@ABV0@PBD@Z$1 1000001a f   OpenCLSupportSettingsController.obj
 0002:ffff8020       __tryblocktable$??0?$QList@PAVOpenCLGpuModel@U2@@@@QAE@ABV0@@Z 10000020     OpenCLSupportSettingsController.obj
 0002:ffff8020       __unwindtable$?_Copy@?$basic_string@DU?$char_traits@D@std@@V?$allocator@D@2@@std@@QAEXII@Z 10000020     moc_OpenCLSupportSettingsController.obj
 0002:ffff8020       __unwindtable$?_Copy@?$basic_string@DU?$char_traits@D@std@@V?$allocator@D@2@@std@@QAEXII@Z 10000020     moc_OpenCLSupportPlugin.obj
 0002:ffff8020       __unwindtable$?_Copy@?$basic_string@DU?$char_traits@D@std@@V?$allocator@D@2@@std@@QAEXII@Z 10000020     OpenCLSupportSettingsController.obj
 0001:fffff023       __ehhandler$??H@YA?BVQString@@ABV0@PBD@Z 10000023 f   OpenCLSupportSettingsController.obj
 0002:ffff8034       __ehfuncinfo$??0?$QList@PAVOpenCLGpuModel@U2@@@@QAE@ABV0@@Z 10000034     OpenCLSupportSettingsController.obj
 0002:ffff8040       __ehfuncinfo$?_Copy@?$basic_string@DU?$char_traits@D@std@@V?$allocator@D@2@@std@@QAEXII@Z 10000040     moc_OpenCLSupportSettingsController.obj
 0002:ffff8040       __ehfuncinfo$?_Copy@?$basic_string@DU?$char_traits@D@std@@V?$allocator@D@2@@std@@QAEXII@Z 10000040     moc_OpenCLSupportPlugin.obj
 0002:ffff8040       __ehfuncinfo$?_Copy@?$basic_string@DU?$char_traits@D@std@@V?$allocator@D@2@@std@@QAEXII@Z 10000040     OpenCLSupportSettingsController.obj
 0002:ffff8064       __tryblocktable$?_Copy@?$basic_string@DU?$char_traits@D@std@@V?$allocator@D@2@@std@@QAEXII@Z 10000064     moc_OpenCLSupportSettingsController.obj
 0002:ffff8064       __tryblocktable$?_Copy@?$basic_string@DU?$char_traits@D@std@@V?$allocator@D@2@@std@@QAEXII@Z 10000064     moc_OpenCLSupportPlugin.obj
 0002:ffff8064       __tryblocktable$?_Copy@?$basic_string@DU?$char_traits@D@std@@V?$allocator@D@2@@std@@QAEXII@Z 10000064     OpenCLSupportSettingsController.obj
 0001:fffff096       __catch$?_Copy@?$basic_string@DU?$char_traits@D@std@@V?$allocator@D@2@@std@@QAEXII@Z$0 10000096 f   moc_OpenCLSupportPlugin.obj
 0001:fffff096       __catch$?_Copy@?$basic_string@DU?$char_traits@D@std@@V?$allocator@D@2@@std@@QAEXII@Z$0 10000096 f   moc_OpenCLSupportSettingsController.obj
 0001:fffff096       __catch$?_Copy@?$basic_string@DU?$char_traits@D@std@@V?$allocator@D@2@@std@@QAEXII@Z$0 10000096 f   OpenCLSupportSettingsController.obj
 0001:fffff09e       __catch$??0?$QList@PAVOpenCLGpuModel@U2@@@@QAE@ABV0@@Z$0 1000009e f   OpenCLSupportSettingsController.obj
 0001:fffff0d3       __catch$?_Copy@?$basic_string@DU?$char_traits@D@std@@V?$allocator@D@2@@std@@QAEXII@Z$1 100000d3 f   moc_OpenCLSupportSettingsController.obj
 0001:fffff0d3       __catch$?_Copy@?$basic_string@DU?$char_traits@D@std@@V?$allocator@D@2@@std@@QAEXII@Z$1 100000d3 f   moc_OpenCLSupportPlugin.obj
 0001:fffff0d3       __catch$?_Copy@?$basic_string@DU?$char_traits@D@std@@V?$allocator@D@2@@std@@QAEXII@Z$1 100000d3 f   OpenCLSupportSettingsController.obj
 0001:00000000       ??__E?_Generic_object@?$_Error_objects@H@std@@2V_Generic_error_category@2@A@@YAXXZ 10001000 f   OpenCLSupportPlugin.obj
 0001:00000010       ??__E?_Iostream_object@?$_Error_objects@H@std@@2V_Iostream_error_category@2@A@@YAXXZ 10001010 f   OpenCLSupportPlugin.obj
 0001:00000020       ??__E?_System_object@?$_Error_objects@H@std@@2V_System_error_category@2@A@@YAXXZ 10001020 f   OpenCLSupportPlugin.obj
 0001:00000030       ??__EalgoLog@U2@@YAXXZ     10001030 f   OpenCLSupportPlugin.obj
 0001:000000b0       ??__EcmdLog@U2@@YAXXZ      100010b0 f   OpenCLSupportPlugin.obj
 0001:00000130       ??__EcoreLog@U2@@YAXXZ     10001130 f   OpenCLSupportPlugin.obj
 0001:000001b0       ??__EioLog@U2@@YAXXZ       100011b0 f   OpenCLSupportPlugin.obj
 0001:00000230       ??__EperfLog@U2@@YAXXZ     10001230 f   OpenCLSupportPlugin.obj
 0001:000002b0       ??__EscriptLog@U2@@YAXXZ   100012b0 f   OpenCLSupportPlugin.obj
 0001:00000330       ??__EtaskLog@U2@@YAXXZ     10001330 f   OpenCLSupportPlugin.obj
 0001:000003b0       ??__EuiLog@U2@@YAXXZ       100013b0 f   OpenCLSupportPlugin.obj
 0001:00000430       ??__EuserActLog@U2@@YAXXZ  10001430 f   OpenCLSupportPlugin.obj
 0001:000004b0       ??__E?_Generic_object@?$_Error_objects@H@std@@2V_Generic_error_category@2@A@@YAXXZ 100014b0 f   OpenCLSupportSettingsController.obj
 0001:000004c0       ??__E?_Iostream_object@?$_Error_objects@H@std@@2V_Iostream_error_category@2@A@@YAXXZ 100014c0 f   OpenCLSupportSettingsController.obj
 0001:000004d0       ??__E?_System_object@?$_Error_objects@H@std@@2V_System_error_category@2@A@@YAXXZ 100014d0 f   OpenCLSupportSettingsController.obj
 0001:000004e0       ??__E?helpPageId@OpenCLSupportSettingsPageController@U2@@0VQString@@B@@YAXXZ 100014e0 f   OpenCLSupportSettingsController.obj
 0001:00000500       ??__EalgoLog@U2@@YAXXZ     10001500 f   OpenCLSupportSettingsController.obj
 0001:00000580       ??__EcmdLog@U2@@YAXXZ      10001580 f   OpenCLSupportSettingsController.obj
 0001:00000600       ??__EcoreLog@U2@@YAXXZ     10001600 f   OpenCLSupportSettingsController.obj
 0001:00000680       ??__EioLog@U2@@YAXXZ       10001680 f   OpenCLSupportSettingsController.obj
 0001:00000700       ??__EperfLog@U2@@YAXXZ     10001700 f   OpenCLSupportSettingsController.obj
 0001:00000780       ??__EscriptLog@U2@@YAXXZ   10001780 f   OpenCLSupportSettingsController.obj
 0001:00000800       ??__EtaskLog@U2@@YAXXZ     10001800 f   OpenCLSupportSettingsController.obj
 0001:00000880       ??__EuiLog@U2@@YAXXZ       10001880 f   OpenCLSupportSettingsController.obj
 0001:00000900       ??__EuserActLog@U2@@YAXXZ  10001900 f   OpenCLSupportSettingsController.obj
 0001:00000980       ??__E?_Generic_object@?$_Error_objects@H@std@@2V_Generic_error_category@2@A@@YAXXZ 10001980 f   moc_OpenCLSupportPlugin.obj
 0001:00000990       ??__E?_Iostream_object@?$_Error_objects@H@std@@2V_Iostream_error_category@2@A@@YAXXZ 10001990 f   moc_OpenCLSupportPlugin.obj
 0001:000009a0       ??__E?_System_object@?$_Error_objects@H@std@@2V_System_error_category@2@A@@YAXXZ 100019a0 f   moc_OpenCLSupportPlugin.obj
 0001:000009b0       ??__E?staticMetaObject@OpenCLSupportPlugin@U2@@2UQMetaObject@@B@@YAXXZ 100019b0 f   moc_OpenCLSupportPlugin.obj
 0001:000009c0       ??__E?_Generic_object@?$_Error_objects@H@std@@2V_Generic_error_category@2@A@@YAXXZ 100019c0 f   moc_OpenCLSupportSettingsController.obj
 0001:000009d0       ??__E?_Iostream_object@?$_Error_objects@H@std@@2V_Iostream_error_category@2@A@@YAXXZ 100019d0 f   moc_OpenCLSupportSettingsController.obj
 0001:000009e0       ??__E?_System_object@?$_Error_objects@H@std@@2V_System_error_category@2@A@@YAXXZ 100019e0 f   moc_OpenCLSupportSettingsController.obj
 0001:000009f0       ??__E?staticMetaObject@OpenCLSupportSettingsPageController@U2@@2UQMetaObject@@B@@YAXXZ 100019f0 f   moc_OpenCLSupportSettingsController.obj
 0001:00000a00       ??__E?staticMetaObject@OpenCLSupportSettingsPageState@U2@@2UQMetaObject@@B@@YAXXZ 10001a00 f   moc_OpenCLSupportSettingsController.obj
 0001:00000a10       ??__E?staticMetaObject@OpenCLSupportSettingsPageWidget@U2@@2UQMetaObject@@B@@YAXXZ 10001a10 f   moc_OpenCLSupportSettingsController.obj
 0001:00000c3e       __catch$??0?$QList@PAVOpenCLGpuModel@U2@@@@QAE@ABV0@@Z$0 10001c3e f i OpenCLSupportPlugin.obj
 0001:00001636       __catch$?_Copy@?$basic_string@DU?$char_traits@D@std@@V?$allocator@D@2@@std@@QAEXII@Z$0 10002636 f i OpenCLSupportPlugin.obj
 0001:00001673       __catch$?_Copy@?$basic_string@DU?$char_traits@D@std@@V?$allocator@D@2@@std@@QAEXII@Z$1 10002673 f i OpenCLSupportPlugin.obj
 0001:00001995       __catch$?append@?$QList@PAVOpenCLGpuModel@U2@@@@QAEXABQAVOpenCLGpuModel@U2@@@Z$4 10002995 f i OpenCLSupportPlugin.obj
 0001:00001e71       __catch$?detach_helper_grow@?$QList@PAVOpenCLGpuModel@U2@@@@AAEPAUNode@1@HH@Z$2 10002e71 f i OpenCLSupportPlugin.obj
 0001:00001e71       __catch$?detach_helper_grow@?$QList@PAVOpenCLGpuModel@U2@@@@AAEPAUNode@1@HH@Z$0 10002e71 f i OpenCLSupportPlugin.obj
 0001:000040a5       __catch$?append@?$QList@PAVQCheckBox@@@@QAEXABQAVQCheckBox@@@Z$4 100050a5 f i OpenCLSupportSettingsController.obj
 0001:000043fc       __catch$?detach_helper@?$QList@PAVOpenCLGpuModel@U2@@@@AAEXH@Z$0 100053fc f i OpenCLSupportSettingsController.obj
 0001:00004521       __catch$?detach_helper_grow@?$QList@PAVQCheckBox@@@@AAEPAUNode@1@HH@Z$0 10005521 f i OpenCLSupportSettingsController.obj
 0001:00004521       __catch$?detach_helper_grow@?$QList@PAVQCheckBox@@@@AAEPAUNode@1@HH@Z$2 10005521 f i OpenCLSupportSettingsController.obj
 0001:00004a63       __catch$?reallocData@?$QVector@_N@@AAEXHHV?$QFlags@W4AllocationOption@QArrayData@@@@@Z$0 10005a63 f i OpenCLSupportSettingsController.obj
 0001:00004a75       __catch$?reallocData@?$QVector@_N@@AAEXHHV?$QFlags@W4AllocationOption@QArrayData@@@@@Z$2 10005a75 f i OpenCLSupportSettingsController.obj
 0001:0000573c       _pre_c_init                1000673c f   MSVCRT:crtdll.obj
 0001:000059a9       ___DllMainCRTStartup       100069a9 f   MSVCRT:crtdll.obj
 0001:00005b00       $$000000                   10006b00     MSVCRT:sehprolg4.obj
 0001:00005f15       ?ArrayUnwindFilter@@YAHPAU_EXCEPTION_POINTERS@@@Z 10006f15 f   MSVCRT:ehvecdtr.obj
 0001:00006260       __ehhandler$??0?$QList@PAVOpenCLGpuModel@U2@@@@QAE@ABV0@@Z 10007260 f   OpenCLSupportPlugin.obj
 0001:00006280       __unwindfunclet$??0OpenCLSupportPlugin@U2@@QAE@XZ$0 10007280 f   OpenCLSupportPlugin.obj
 0001:00006289       __unwindfunclet$??0OpenCLSupportPlugin@U2@@QAE@XZ$1 10007289 f   OpenCLSupportPlugin.obj
 0001:00006292       __unwindfunclet$??0OpenCLSupportPlugin@U2@@QAE@XZ$2 10007292 f   OpenCLSupportPlugin.obj
 0001:0000629b       __unwindfunclet$??0OpenCLSupportPlugin@U2@@QAE@XZ$3 1000729b f   OpenCLSupportPlugin.obj
 0001:000062a6       __unwindfunclet$??0OpenCLSupportPlugin@U2@@QAE@XZ$4 100072a6 f   OpenCLSupportPlugin.obj
 0001:000062b2       __unwindfunclet$??0OpenCLSupportPlugin@U2@@QAE@XZ$5 100072b2 f   OpenCLSupportPlugin.obj
 0001:000062bb       __unwindfunclet$??0OpenCLSupportPlugin@U2@@QAE@XZ$6 100072bb f   OpenCLSupportPlugin.obj
 0001:000062c4       __unwindfunclet$??0OpenCLSupportPlugin@U2@@QAE@XZ$7 100072c4 f   OpenCLSupportPlugin.obj
 0001:000062cf       __unwindfunclet$??0OpenCLSupportPlugin@U2@@QAE@XZ$8 100072cf f   OpenCLSupportPlugin.obj
 0001:000062d8       __unwindfunclet$??0OpenCLSupportPlugin@U2@@QAE@XZ$9 100072d8 f   OpenCLSupportPlugin.obj
 0001:000062e3       __unwindfunclet$??0OpenCLSupportPlugin@U2@@QAE@XZ$10 100072e3 f   OpenCLSupportPlugin.obj
 0001:000062fd       __unwindfunclet$??0OpenCLSupportPlugin@U2@@QAE@XZ$11 100072fd f   OpenCLSupportPlugin.obj
 0001:00006317       __ehhandler$??0OpenCLSupportPlugin@U2@@QAE@XZ 10007317 f   OpenCLSupportPlugin.obj
 0001:00006340       __unwindfunclet$??1OpenCLSupportPlugin@U2@@UAE@XZ$0 10007340 f   OpenCLSupportPlugin.obj
 0001:00006349       __unwindfunclet$??1OpenCLSupportPlugin@U2@@UAE@XZ$1 10007349 f   OpenCLSupportPlugin.obj
 0001:00006354       __unwindfunclet$??1OpenCLSupportPlugin@U2@@UAE@XZ$2 10007354 f   OpenCLSupportPlugin.obj
 0001:00006360       __ehhandler$??1OpenCLSupportPlugin@U2@@UAE@XZ 10007360 f   OpenCLSupportPlugin.obj
 0001:00006380       __unwindfunclet$??H@YA?BVQString@@ABV0@0@Z$0 10007380 f   OpenCLSupportPlugin.obj
 0001:0000639a       __ehhandler$??H@YA?BVQString@@ABV0@0@Z 1000739a f   OpenCLSupportPlugin.obj
 0001:000063c0       __unwindfunclet$??H@YA?BVQString@@ABV0@PBD@Z$0 100073c0 f   OpenCLSupportPlugin.obj
 0001:000063da       __unwindfunclet$??H@YA?BVQString@@ABV0@PBD@Z$1 100073da f   OpenCLSupportPlugin.obj
 0001:000063e3       __ehhandler$??H@YA?BVQString@@ABV0@PBD@Z 100073e3 f   OpenCLSupportPlugin.obj
 0001:00006400       __unwindfunclet$??H@YA?BVQString@@PBDABV0@@Z$0 10007400 f   OpenCLSupportPlugin.obj
 0001:0000641a       __ehhandler$??H@YA?BVQString@@PBDABV0@@Z 1000741a f   OpenCLSupportPlugin.obj
 0001:00006440       __unwindfunclet$??__EalgoLog@U2@@YAXXZ$0 10007440 f   OpenCLSupportPlugin.obj
 0001:00006449       __ehhandler$??__EalgoLog@U2@@YAXXZ 10007449 f   OpenCLSupportPlugin.obj
 0001:00006470       __unwindfunclet$??__EcmdLog@U2@@YAXXZ$0 10007470 f   OpenCLSupportPlugin.obj
 0001:00006479       __ehhandler$??__EcmdLog@U2@@YAXXZ 10007479 f   OpenCLSupportPlugin.obj
 0001:000064a0       __unwindfunclet$??__EcoreLog@U2@@YAXXZ$0 100074a0 f   OpenCLSupportPlugin.obj
 0001:000064a9       __ehhandler$??__EcoreLog@U2@@YAXXZ 100074a9 f   OpenCLSupportPlugin.obj
 0001:000064d0       __unwindfunclet$??__EioLog@U2@@YAXXZ$0 100074d0 f   OpenCLSupportPlugin.obj
 0001:000064d9       __ehhandler$??__EioLog@U2@@YAXXZ 100074d9 f   OpenCLSupportPlugin.obj
 0001:00006500       __unwindfunclet$??__EperfLog@U2@@YAXXZ$0 10007500 f   OpenCLSupportPlugin.obj
 0001:00006509       __ehhandler$??__EperfLog@U2@@YAXXZ 10007509 f   OpenCLSupportPlugin.obj
 0001:00006530       __unwindfunclet$??__EscriptLog@U2@@YAXXZ$0 10007530 f   OpenCLSupportPlugin.obj
 0001:00006539       __ehhandler$??__EscriptLog@U2@@YAXXZ 10007539 f   OpenCLSupportPlugin.obj
 0001:00006560       __unwindfunclet$??__EtaskLog@U2@@YAXXZ$0 10007560 f   OpenCLSupportPlugin.obj
 0001:00006569       __ehhandler$??__EtaskLog@U2@@YAXXZ 10007569 f   OpenCLSupportPlugin.obj
 0001:00006590       __unwindfunclet$??__EuiLog@U2@@YAXXZ$0 10007590 f   OpenCLSupportPlugin.obj
 0001:00006599       __ehhandler$??__EuiLog@U2@@YAXXZ 10007599 f   OpenCLSupportPlugin.obj
 0001:000065c0       __unwindfunclet$??__EuserActLog@U2@@YAXXZ$0 100075c0 f   OpenCLSupportPlugin.obj
 0001:000065c9       __ehhandler$??__EuserActLog@U2@@YAXXZ 100075c9 f   OpenCLSupportPlugin.obj
 0001:000065f0       __ehhandler$?_Copy@?$basic_string@DU?$char_traits@D@std@@V?$allocator@D@2@@std@@QAEXII@Z 100075f0 f   OpenCLSupportPlugin.obj
 0001:00006610       __ehhandler$?append@?$QList@PAVOpenCLGpuModel@U2@@@@QAEXABQAVOpenCLGpuModel@U2@@@Z 10007610 f   OpenCLSupportPlugin.obj
 0001:00006630       __ehhandler$?detach_helper_grow@?$QList@PAVOpenCLGpuModel@U2@@@@AAEPAUNode@1@HH@Z 10007630 f   OpenCLSupportPlugin.obj
 0001:00006650       __unwindfunclet$?hasOPENCLError@OpenCLSupportPlugin@U2@@AAE_NHAAVQString@@@Z$0 10007650 f   OpenCLSupportPlugin.obj
 0001:00006659       __unwindfunclet$?hasOPENCLError@OpenCLSupportPlugin@U2@@AAE_NHAAVQString@@@Z$1 10007659 f   OpenCLSupportPlugin.obj
 0001:00006662       __ehhandler$?hasOPENCLError@OpenCLSupportPlugin@U2@@AAE_NHAAVQString@@@Z 10007662 f   OpenCLSupportPlugin.obj
 0001:00006680       __unwindfunclet$?loadGpusSettings@OpenCLSupportPlugin@U2@@AAEXXZ$0 10007680 f   OpenCLSupportPlugin.obj
 0001:00006688       __unwindfunclet$?loadGpusSettings@OpenCLSupportPlugin@U2@@AAEXXZ$1 10007688 f   OpenCLSupportPlugin.obj
 0001:00006691       __unwindfunclet$?loadGpusSettings@OpenCLSupportPlugin@U2@@AAEXXZ$2 10007691 f   OpenCLSupportPlugin.obj
 0001:0000669a       __unwindfunclet$?loadGpusSettings@OpenCLSupportPlugin@U2@@AAEXXZ$3 1000769a f   OpenCLSupportPlugin.obj
 0001:000066a3       __unwindfunclet$?loadGpusSettings@OpenCLSupportPlugin@U2@@AAEXXZ$4 100076a3 f   OpenCLSupportPlugin.obj
 0001:000066ac       __unwindfunclet$?loadGpusSettings@OpenCLSupportPlugin@U2@@AAEXXZ$5 100076ac f   OpenCLSupportPlugin.obj
 0001:000066b5       __ehhandler$?loadGpusSettings@OpenCLSupportPlugin@U2@@AAEXXZ 100076b5 f   OpenCLSupportPlugin.obj
 0001:000066d0       __unwindfunclet$?obtainGpusInfo@OpenCLSupportPlugin@U2@@AAE?AW4OpenCLSupportError@12@AAVQString@@@Z$0 100076d0 f   OpenCLSupportPlugin.obj
 0001:000066d9       __unwindfunclet$?obtainGpusInfo@OpenCLSupportPlugin@U2@@AAE?AW4OpenCLSupportError@12@AAVQString@@@Z$1 100076d9 f   OpenCLSupportPlugin.obj
 0001:000066e2       __unwindfunclet$?obtainGpusInfo@OpenCLSupportPlugin@U2@@AAE?AW4OpenCLSupportError@12@AAVQString@@@Z$2 100076e2 f   OpenCLSupportPlugin.obj
 0001:000066ea       __unwindfunclet$?obtainGpusInfo@OpenCLSupportPlugin@U2@@AAE?AW4OpenCLSupportError@12@AAVQString@@@Z$3 100076ea f   OpenCLSupportPlugin.obj
 0001:000066f3       __unwindfunclet$?obtainGpusInfo@OpenCLSupportPlugin@U2@@AAE?AW4OpenCLSupportError@12@AAVQString@@@Z$4 100076f3 f   OpenCLSupportPlugin.obj
 0001:000066fc       __unwindfunclet$?obtainGpusInfo@OpenCLSupportPlugin@U2@@AAE?AW4OpenCLSupportError@12@AAVQString@@@Z$5 100076fc f   OpenCLSupportPlugin.obj
 0001:00006704       __unwindfunclet$?obtainGpusInfo@OpenCLSupportPlugin@U2@@AAE?AW4OpenCLSupportError@12@AAVQString@@@Z$6 10007704 f   OpenCLSupportPlugin.obj
 0001:00006710       __unwindfunclet$?obtainGpusInfo@OpenCLSupportPlugin@U2@@AAE?AW4OpenCLSupportError@12@AAVQString@@@Z$7 10007710 f   OpenCLSupportPlugin.obj
 0001:00006719       __unwindfunclet$?obtainGpusInfo@OpenCLSupportPlugin@U2@@AAE?AW4OpenCLSupportError@12@AAVQString@@@Z$8 10007719 f   OpenCLSupportPlugin.obj
 0001:00006724       __unwindfunclet$?obtainGpusInfo@OpenCLSupportPlugin@U2@@AAE?AW4OpenCLSupportError@12@AAVQString@@@Z$9 10007724 f   OpenCLSupportPlugin.obj
 0001:0000672f       __unwindfunclet$?obtainGpusInfo@OpenCLSupportPlugin@U2@@AAE?AW4OpenCLSupportError@12@AAVQString@@@Z$10 1000772f f   OpenCLSupportPlugin.obj
 0001:00006738       __unwindfunclet$?obtainGpusInfo@OpenCLSupportPlugin@U2@@AAE?AW4OpenCLSupportError@12@AAVQString@@@Z$11 10007738 f   OpenCLSupportPlugin.obj
 0001:00006743       __unwindfunclet$?obtainGpusInfo@OpenCLSupportPlugin@U2@@AAE?AW4OpenCLSupportError@12@AAVQString@@@Z$12 10007743 f   OpenCLSupportPlugin.obj
 0001:0000674c       __unwindfunclet$?obtainGpusInfo@OpenCLSupportPlugin@U2@@AAE?AW4OpenCLSupportError@12@AAVQString@@@Z$13 1000774c f   OpenCLSupportPlugin.obj
 0001:00006757       __unwindfunclet$?obtainGpusInfo@OpenCLSupportPlugin@U2@@AAE?AW4OpenCLSupportError@12@AAVQString@@@Z$14 10007757 f   OpenCLSupportPlugin.obj
 0001:00006774       __unwindfunclet$?obtainGpusInfo@OpenCLSupportPlugin@U2@@AAE?AW4OpenCLSupportError@12@AAVQString@@@Z$15 10007774 f   OpenCLSupportPlugin.obj
 0001:0000678e       __unwindfunclet$?obtainGpusInfo@OpenCLSupportPlugin@U2@@AAE?AW4OpenCLSupportError@12@AAVQString@@@Z$16 1000778e f   OpenCLSupportPlugin.obj
 0001:00006797       __unwindfunclet$?obtainGpusInfo@OpenCLSupportPlugin@U2@@AAE?AW4OpenCLSupportError@12@AAVQString@@@Z$17 10007797 f   OpenCLSupportPlugin.obj
 0001:000067a3       __unwindfunclet$?obtainGpusInfo@OpenCLSupportPlugin@U2@@AAE?AW4OpenCLSupportError@12@AAVQString@@@Z$18 100077a3 f   OpenCLSupportPlugin.obj
 0001:000067af       __unwindfunclet$?obtainGpusInfo@OpenCLSupportPlugin@U2@@AAE?AW4OpenCLSupportError@12@AAVQString@@@Z$19 100077af f   OpenCLSupportPlugin.obj
 0001:000067bb       __unwindfunclet$?obtainGpusInfo@OpenCLSupportPlugin@U2@@AAE?AW4OpenCLSupportError@12@AAVQString@@@Z$20 100077bb f   OpenCLSupportPlugin.obj
 0001:000067c4       __unwindfunclet$?obtainGpusInfo@OpenCLSupportPlugin@U2@@AAE?AW4OpenCLSupportError@12@AAVQString@@@Z$21 100077c4 f   OpenCLSupportPlugin.obj
 0001:000067cd       __unwindfunclet$?obtainGpusInfo@OpenCLSupportPlugin@U2@@AAE?AW4OpenCLSupportError@12@AAVQString@@@Z$22 100077cd f   OpenCLSupportPlugin.obj
 0001:000067d6       __unwindfunclet$?obtainGpusInfo@OpenCLSupportPlugin@U2@@AAE?AW4OpenCLSupportError@12@AAVQString@@@Z$23 100077d6 f   OpenCLSupportPlugin.obj
 0001:000067e2       __ehhandler$?obtainGpusInfo@OpenCLSupportPlugin@U2@@AAE?AW4OpenCLSupportError@12@AAVQString@@@Z 100077e2 f   OpenCLSupportPlugin.obj
 0001:00006800       __unwindfunclet$?registerAvailableGpus@OpenCLSupportPlugin@U2@@AAEXXZ$0 10007800 f   OpenCLSupportPlugin.obj
 0001:00006808       __ehhandler$?registerAvailableGpus@OpenCLSupportPlugin@U2@@AAEXXZ 10007808 f   OpenCLSupportPlugin.obj
 0001:00006830       __unwindfunclet$?unregisterAvailableGpus@OpenCLSupportPlugin@U2@@AAEXXZ$0 10007830 f   OpenCLSupportPlugin.obj
 0001:00006838       __ehhandler$?unregisterAvailableGpus@OpenCLSupportPlugin@U2@@AAEXXZ 10007838 f   OpenCLSupportPlugin.obj
 0001:00006860       __unwindfunclet$??0OpenCLSupportSettingsPageController@U2@@QAE@ABVQString@@PAVQObject@@@Z$0 10007860 f   OpenCLSupportSettingsController.obj
 0001:00006869       __unwindfunclet$??0OpenCLSupportSettingsPageController@U2@@QAE@ABVQString@@PAVQObject@@@Z$1 10007869 f   OpenCLSupportSettingsController.obj
 0001:00006872       __unwindfunclet$??0OpenCLSupportSettingsPageController@U2@@QAE@ABVQString@@PAVQObject@@@Z$2 10007872 f   OpenCLSupportSettingsController.obj
 0001:0000687b       __ehhandler$??0OpenCLSupportSettingsPageController@U2@@QAE@ABVQString@@PAVQObject@@@Z 1000787b f   OpenCLSupportSettingsController.obj
 0001:000068a0       __unwindfunclet$??0OpenCLSupportSettingsPageState@U2@@QAE@H@Z$0 100078a0 f   OpenCLSupportSettingsController.obj
 0001:000068a9       __unwindfunclet$??0OpenCLSupportSettingsPageState@U2@@QAE@H@Z$1 100078a9 f   OpenCLSupportSettingsController.obj
 0001:000068b4       __ehhandler$??0OpenCLSupportSettingsPageState@U2@@QAE@H@Z 100078b4 f   OpenCLSupportSettingsController.obj
 0001:000068d0       __unwindfunclet$??0OpenCLSupportSettingsPageWidget@U2@@QAE@ABVQString@@PAVOpenCLSupportSettingsPageController@1@@Z$0 100078d0 f   OpenCLSupportSettingsController.obj
 0001:000068d9       __unwindfunclet$??0OpenCLSupportSettingsPageWidget@U2@@QAE@ABVQString@@PAVOpenCLSupportSettingsPageController@1@@Z$1 100078d9 f   OpenCLSupportSettingsController.obj
 0001:000068e5       __unwindfunclet$??0OpenCLSupportSettingsPageWidget@U2@@QAE@ABVQString@@PAVOpenCLSupportSettingsPageController@1@@Z$2 100078e5 f   OpenCLSupportSettingsController.obj
 0001:000068f0       __unwindfunclet$??0OpenCLSupportSettingsPageWidget@U2@@QAE@ABVQString@@PAVOpenCLSupportSettingsPageController@1@@Z$3 100078f0 f   OpenCLSupportSettingsController.obj
 0001:000068fb       __unwindfunclet$??0OpenCLSupportSettingsPageWidget@U2@@QAE@ABVQString@@PAVOpenCLSupportSettingsPageController@1@@Z$4 100078fb f   OpenCLSupportSettingsController.obj
 0001:00006906       __unwindfunclet$??0OpenCLSupportSettingsPageWidget@U2@@QAE@ABVQString@@PAVOpenCLSupportSettingsPageController@1@@Z$5 10007906 f   OpenCLSupportSettingsController.obj
 0001:00006911       __unwindfunclet$??0OpenCLSupportSettingsPageWidget@U2@@QAE@ABVQString@@PAVOpenCLSupportSettingsPageController@1@@Z$6 10007911 f   OpenCLSupportSettingsController.obj
 0001:00006919       __unwindfunclet$??0OpenCLSupportSettingsPageWidget@U2@@QAE@ABVQString@@PAVOpenCLSupportSettingsPageController@1@@Z$7 10007919 f   OpenCLSupportSettingsController.obj
 0001:00006933       __unwindfunclet$??0OpenCLSupportSettingsPageWidget@U2@@QAE@ABVQString@@PAVOpenCLSupportSettingsPageController@1@@Z$8 10007933 f   OpenCLSupportSettingsController.obj
 0001:0000694d       __unwindfunclet$??0OpenCLSupportSettingsPageWidget@U2@@QAE@ABVQString@@PAVOpenCLSupportSettingsPageController@1@@Z$9 1000794d f   OpenCLSupportSettingsController.obj
 0001:00006956       __unwindfunclet$??0OpenCLSupportSettingsPageWidget@U2@@QAE@ABVQString@@PAVOpenCLSupportSettingsPageController@1@@Z$10 10007956 f   OpenCLSupportSettingsController.obj
 0001:00006961       __unwindfunclet$??0OpenCLSupportSettingsPageWidget@U2@@QAE@ABVQString@@PAVOpenCLSupportSettingsPageController@1@@Z$11 10007961 f   OpenCLSupportSettingsController.obj
 0001:00006969       __unwindfunclet$??0OpenCLSupportSettingsPageWidget@U2@@QAE@ABVQString@@PAVOpenCLSupportSettingsPageController@1@@Z$12 10007969 f   OpenCLSupportSettingsController.obj
 0001:00006974       __unwindfunclet$??0OpenCLSupportSettingsPageWidget@U2@@QAE@ABVQString@@PAVOpenCLSupportSettingsPageController@1@@Z$13 10007974 f   OpenCLSupportSettingsController.obj
 0001:0000697d       __unwindfunclet$??0OpenCLSupportSettingsPageWidget@U2@@QAE@ABVQString@@PAVOpenCLSupportSettingsPageController@1@@Z$14 1000797d f   OpenCLSupportSettingsController.obj
 0001:00006986       __unwindfunclet$??0OpenCLSupportSettingsPageWidget@U2@@QAE@ABVQString@@PAVOpenCLSupportSettingsPageController@1@@Z$15 10007986 f   OpenCLSupportSettingsController.obj
 0001:0000698f       __unwindfunclet$??0OpenCLSupportSettingsPageWidget@U2@@QAE@ABVQString@@PAVOpenCLSupportSettingsPageController@1@@Z$16 1000798f f   OpenCLSupportSettingsController.obj
 0001:00006998       __unwindfunclet$??0OpenCLSupportSettingsPageWidget@U2@@QAE@ABVQString@@PAVOpenCLSupportSettingsPageController@1@@Z$17 10007998 f   OpenCLSupportSettingsController.obj
 0001:000069a1       __unwindfunclet$??0OpenCLSupportSettingsPageWidget@U2@@QAE@ABVQString@@PAVOpenCLSupportSettingsPageController@1@@Z$18 100079a1 f   OpenCLSupportSettingsController.obj
 0001:000069ac       __ehhandler$??0OpenCLSupportSettingsPageWidget@U2@@QAE@ABVQString@@PAVOpenCLSupportSettingsPageController@1@@Z 100079ac f   OpenCLSupportSettingsController.obj
 0001:000069d0       __unwindfunclet$??1OpenCLSupportSettingsPageController@U2@@UAE@XZ$0 100079d0 f   OpenCLSupportSettingsController.obj
 0001:000069d9       __ehhandler$??1OpenCLSupportSettingsPageController@U2@@UAE@XZ 100079d9 f   OpenCLSupportSettingsController.obj
 0001:00006a00       __unwindfunclet$??1OpenCLSupportSettingsPageState@U2@@UAE@XZ$0 10007a00 f   OpenCLSupportSettingsController.obj
 0001:00006a09       __ehhandler$??1OpenCLSupportSettingsPageState@U2@@UAE@XZ 10007a09 f   OpenCLSupportSettingsController.obj
 0001:00006a30       __unwindfunclet$??1OpenCLSupportSettingsPageWidget@U2@@UAE@XZ$0 10007a30 f   OpenCLSupportSettingsController.obj
 0001:00006a39       __unwindfunclet$??1OpenCLSupportSettingsPageWidget@U2@@UAE@XZ$1 10007a39 f   OpenCLSupportSettingsController.obj
 0001:00006a45       __ehhandler$??1OpenCLSupportSettingsPageWidget@U2@@UAE@XZ 10007a45 f   OpenCLSupportSettingsController.obj
 0001:00006a60       __unwindfunclet$??_GOpenCLSupportSettingsPageController@U2@@UAEPAXI@Z$0 10007a60 f   OpenCLSupportSettingsController.obj
 0001:00006a69       __ehhandler$??_GOpenCLSupportSettingsPageController@U2@@UAEPAXI@Z 10007a69 f   OpenCLSupportSettingsController.obj
 0001:00006a90       __unwindfunclet$??_GOpenCLSupportSettingsPageState@U2@@UAEPAXI@Z$0 10007a90 f   OpenCLSupportSettingsController.obj
 0001:00006a99       __ehhandler$??_GOpenCLSupportSettingsPageState@U2@@UAEPAXI@Z 10007a99 f   OpenCLSupportSettingsController.obj
 0001:00006ac0       __unwindfunclet$??_GOpenCLSupportSettingsPageWidget@U2@@UAEPAXI@Z$0 10007ac0 f   OpenCLSupportSettingsController.obj
 0001:00006ac9       __unwindfunclet$??_GOpenCLSupportSettingsPageWidget@U2@@UAEPAXI@Z$1 10007ac9 f   OpenCLSupportSettingsController.obj
 0001:00006ad5       __ehhandler$??_GOpenCLSupportSettingsPageWidget@U2@@UAEPAXI@Z 10007ad5 f   OpenCLSupportSettingsController.obj
 0001:00006af0       __unwindfunclet$??__EalgoLog@U2@@YAXXZ$0 10007af0 f   OpenCLSupportSettingsController.obj
 0001:00006af9       __ehhandler$??__EalgoLog@U2@@YAXXZ 10007af9 f   OpenCLSupportSettingsController.obj
 0001:00006b20       __unwindfunclet$??__EcmdLog@U2@@YAXXZ$0 10007b20 f   OpenCLSupportSettingsController.obj
 0001:00006b29       __ehhandler$??__EcmdLog@U2@@YAXXZ 10007b29 f   OpenCLSupportSettingsController.obj
 0001:00006b50       __unwindfunclet$??__EcoreLog@U2@@YAXXZ$0 10007b50 f   OpenCLSupportSettingsController.obj
 0001:00006b59       __ehhandler$??__EcoreLog@U2@@YAXXZ 10007b59 f   OpenCLSupportSettingsController.obj
 0001:00006b80       __unwindfunclet$??__EioLog@U2@@YAXXZ$0 10007b80 f   OpenCLSupportSettingsController.obj
 0001:00006b89       __ehhandler$??__EioLog@U2@@YAXXZ 10007b89 f   OpenCLSupportSettingsController.obj
 0001:00006bb0       __unwindfunclet$??__EperfLog@U2@@YAXXZ$0 10007bb0 f   OpenCLSupportSettingsController.obj
 0001:00006bb9       __ehhandler$??__EperfLog@U2@@YAXXZ 10007bb9 f   OpenCLSupportSettingsController.obj
 0001:00006be0       __unwindfunclet$??__EscriptLog@U2@@YAXXZ$0 10007be0 f   OpenCLSupportSettingsController.obj
 0001:00006be9       __ehhandler$??__EscriptLog@U2@@YAXXZ 10007be9 f   OpenCLSupportSettingsController.obj
 0001:00006c10       __unwindfunclet$??__EtaskLog@U2@@YAXXZ$0 10007c10 f   OpenCLSupportSettingsController.obj
 0001:00006c19       __ehhandler$??__EtaskLog@U2@@YAXXZ 10007c19 f   OpenCLSupportSettingsController.obj
 0001:00006c40       __unwindfunclet$??__EuiLog@U2@@YAXXZ$0 10007c40 f   OpenCLSupportSettingsController.obj
 0001:00006c49       __ehhandler$??__EuiLog@U2@@YAXXZ 10007c49 f   OpenCLSupportSettingsController.obj
 0001:00006c70       __unwindfunclet$??__EuserActLog@U2@@YAXXZ$0 10007c70 f   OpenCLSupportSettingsController.obj
 0001:00006c79       __ehhandler$??__EuserActLog@U2@@YAXXZ 10007c79 f   OpenCLSupportSettingsController.obj
 0001:00006ca0       __ehhandler$?append@?$QList@PAVQCheckBox@@@@QAEXABQAVQCheckBox@@@Z 10007ca0 f   OpenCLSupportSettingsController.obj
 0001:00006cc0       __unwindfunclet$?createWidget@OpenCLSupportSettingsPageController@U2@@UAEPAVAppSettingsGUIPageWidget@2@PAVAppSettingsGUIPageState@2@@Z$0 10007cc0 f   OpenCLSupportSettingsController.obj
 0001:00006ccb       __ehhandler$?createWidget@OpenCLSupportSettingsPageController@U2@@UAEPAVAppSettingsGUIPageWidget@2@PAVAppSettingsGUIPageState@2@@Z 10007ccb f   OpenCLSupportSettingsController.obj
 0001:00006cf0       __ehhandler$?detach_helper@?$QList@PAVOpenCLGpuModel@U2@@@@AAEXH@Z 10007cf0 f   OpenCLSupportSettingsController.obj
 0001:00006d10       __ehhandler$?detach_helper_grow@?$QList@PAVQCheckBox@@@@AAEPAUNode@1@HH@Z 10007d10 f   OpenCLSupportSettingsController.obj
 0001:00006d30       __unwindfunclet$?getSavedState@OpenCLSupportSettingsPageController@U2@@UAEPAVAppSettingsGUIPageState@2@XZ$0 10007d30 f   OpenCLSupportSettingsController.obj
 0001:00006d38       __unwindfunclet$?getSavedState@OpenCLSupportSettingsPageController@U2@@UAEPAVAppSettingsGUIPageState@2@XZ$1 10007d38 f   OpenCLSupportSettingsController.obj
 0001:00006d43       __ehhandler$?getSavedState@OpenCLSupportSettingsPageController@U2@@UAEPAVAppSettingsGUIPageState@2@XZ 10007d43 f   OpenCLSupportSettingsController.obj
 0001:00006d60       __unwindfunclet$?getState@OpenCLSupportSettingsPageWidget@U2@@UBEPAVAppSettingsGUIPageState@2@AAVQString@@@Z$0 10007d60 f   OpenCLSupportSettingsController.obj
 0001:00006d6b       __ehhandler$?getState@OpenCLSupportSettingsPageWidget@U2@@UBEPAVAppSettingsGUIPageState@2@AAVQString@@@Z 10007d6b f   OpenCLSupportSettingsController.obj
 0001:00006d90       __ehhandler$?reallocData@?$QVector@_N@@AAEXHHV?$QFlags@W4AllocationOption@QArrayData@@@@@Z 10007d90 f   OpenCLSupportSettingsController.obj
 0001:00006db0       __unwindfunclet$?saveState@OpenCLSupportSettingsPageController@U2@@UAEXPAVAppSettingsGUIPageState@2@@Z$0 10007db0 f   OpenCLSupportSettingsController.obj
 0001:00006db8       __ehhandler$?saveState@OpenCLSupportSettingsPageController@U2@@UAEXPAVAppSettingsGUIPageState@2@@Z 10007db8 f   OpenCLSupportSettingsController.obj
 0001:00006de0       ??__F?_Generic_object@?$_Error_objects@H@std@@2V_Generic_error_category@2@A@@YAXXZ 10007de0 f   OpenCLSupportPlugin.obj
 0001:00006df0       ??__F?_Iostream_object@?$_Error_objects@H@std@@2V_Iostream_error_category@2@A@@YAXXZ 10007df0 f   OpenCLSupportPlugin.obj
 0001:00006e00       ??__F?_System_object@?$_Error_objects@H@std@@2V_System_error_category@2@A@@YAXXZ 10007e00 f   OpenCLSupportPlugin.obj
 0001:00006e10       ??__FalgoLog@U2@@YAXXZ     10007e10 f   OpenCLSupportPlugin.obj
 0001:00006e20       ??__FcmdLog@U2@@YAXXZ      10007e20 f   OpenCLSupportPlugin.obj
 0001:00006e30       ??__FcoreLog@U2@@YAXXZ     10007e30 f   OpenCLSupportPlugin.obj
 0001:00006e40       ??__FioLog@U2@@YAXXZ       10007e40 f   OpenCLSupportPlugin.obj
 0001:00006e50       ??__FperfLog@U2@@YAXXZ     10007e50 f   OpenCLSupportPlugin.obj
 0001:00006e60       ??__FscriptLog@U2@@YAXXZ   10007e60 f   OpenCLSupportPlugin.obj
 0001:00006e70       ??__FtaskLog@U2@@YAXXZ     10007e70 f   OpenCLSupportPlugin.obj
 0001:00006e80       ??__FuiLog@U2@@YAXXZ       10007e80 f   OpenCLSupportPlugin.obj
 0001:00006e90       ??__FuserActLog@U2@@YAXXZ  10007e90 f   OpenCLSupportPlugin.obj
 0001:00006ea0       ??__F?_Generic_object@?$_Error_objects@H@std@@2V_Generic_error_category@2@A@@YAXXZ 10007ea0 f   OpenCLSupportSettingsController.obj
 0001:00006eb0       ??__F?_Iostream_object@?$_Error_objects@H@std@@2V_Iostream_error_category@2@A@@YAXXZ 10007eb0 f   OpenCLSupportSettingsController.obj
 0001:00006ec0       ??__F?_System_object@?$_Error_objects@H@std@@2V_System_error_category@2@A@@YAXXZ 10007ec0 f   OpenCLSupportSettingsController.obj
 0001:00006ed0       ??__F?helpPageId@OpenCLSupportSettingsPageController@U2@@0VQString@@B@@YAXXZ 10007ed0 f   OpenCLSupportSettingsController.obj
 0001:00006ee0       ??__FalgoLog@U2@@YAXXZ     10007ee0 f   OpenCLSupportSettingsController.obj
 0001:00006ef0       ??__FcmdLog@U2@@YAXXZ      10007ef0 f   OpenCLSupportSettingsController.obj
 0001:00006f00       ??__FcoreLog@U2@@YAXXZ     10007f00 f   OpenCLSupportSettingsController.obj
 0001:00006f10       ??__FioLog@U2@@YAXXZ       10007f10 f   OpenCLSupportSettingsController.obj
 0001:00006f20       ??__FperfLog@U2@@YAXXZ     10007f20 f   OpenCLSupportSettingsController.obj
 0001:00006f30       ??__FscriptLog@U2@@YAXXZ   10007f30 f   OpenCLSupportSettingsController.obj
 0001:00006f40       ??__FtaskLog@U2@@YAXXZ     10007f40 f   OpenCLSupportSettingsController.obj
 0001:00006f50       ??__FuiLog@U2@@YAXXZ       10007f50 f   OpenCLSupportSettingsController.obj
 0001:00006f60       ??__FuserActLog@U2@@YAXXZ  10007f60 f   OpenCLSupportSettingsController.obj
 0001:00006f70       ??__F?_Generic_object@?$_Error_objects@H@std@@2V_Generic_error_category@2@A@@YAXXZ 10007f70 f   moc_OpenCLSupportPlugin.obj
 0001:00006f80       ??__F?_Iostream_object@?$_Error_objects@H@std@@2V_Iostream_error_category@2@A@@YAXXZ 10007f80 f   moc_OpenCLSupportPlugin.obj
 0001:00006f90       ??__F?_System_object@?$_Error_objects@H@std@@2V_System_error_category@2@A@@YAXXZ 10007f90 f   moc_OpenCLSupportPlugin.obj
 0001:00006fa0       ??__F?_Generic_object@?$_Error_objects@H@std@@2V_Generic_error_category@2@A@@YAXXZ 10007fa0 f   moc_OpenCLSupportSettingsController.obj
 0001:00006fb0       ??__F?_Iostream_object@?$_Error_objects@H@std@@2V_Iostream_error_category@2@A@@YAXXZ 10007fb0 f   moc_OpenCLSupportSettingsController.obj
 0001:00006fc0       ??__F?_System_object@?$_Error_objects@H@std@@2V_System_error_category@2@A@@YAXXZ 10007fc0 f   moc_OpenCLSupportSettingsController.obj
 0002:00000420       _algoLog$initializer$      10008420     OpenCLSupportPlugin.obj
 0002:00000424       _cmdLog$initializer$       10008424     OpenCLSupportPlugin.obj
 0002:00000428       _coreLog$initializer$      10008428     OpenCLSupportPlugin.obj
 0002:0000042c       _ioLog$initializer$        1000842c     OpenCLSupportPlugin.obj
 0002:00000430       _perfLog$initializer$      10008430     OpenCLSupportPlugin.obj
 0002:00000434       _scriptLog$initializer$    10008434     OpenCLSupportPlugin.obj
 0002:00000438       _taskLog$initializer$      10008438     OpenCLSupportPlugin.obj
 0002:0000043c       _uiLog$initializer$        1000843c     OpenCLSupportPlugin.obj
 0002:00000440       _userActLog$initializer$   10008440     OpenCLSupportPlugin.obj
 0002:00000444       ?_Generic_object$initializer$@?$_Error_objects@H@std@@2P6AXXZA 10008444     OpenCLSupportPlugin.obj
 0002:00000448       ?_Iostream_object$initializer$@?$_Error_objects@H@std@@2P6AXXZA 10008448     OpenCLSupportPlugin.obj
 0002:0000044c       ?_System_object$initializer$@?$_Error_objects@H@std@@2P6AXXZA 1000844c     OpenCLSupportPlugin.obj
 0002:00000450       _algoLog$initializer$      10008450     OpenCLSupportSettingsController.obj
 0002:00000454       _cmdLog$initializer$       10008454     OpenCLSupportSettingsController.obj
 0002:00000458       _coreLog$initializer$      10008458     OpenCLSupportSettingsController.obj
 0002:0000045c       _ioLog$initializer$        1000845c     OpenCLSupportSettingsController.obj
 0002:00000460       _perfLog$initializer$      10008460     OpenCLSupportSettingsController.obj
 0002:00000464       _scriptLog$initializer$    10008464     OpenCLSupportSettingsController.obj
 0002:00000468       _taskLog$initializer$      10008468     OpenCLSupportSettingsController.obj
 0002:0000046c       _uiLog$initializer$        1000846c     OpenCLSupportSettingsController.obj
 0002:00000470       _userActLog$initializer$   10008470     OpenCLSupportSettingsController.obj
 0002:00000474       ?helpPageId$initializer$@OpenCLSupportSettingsPageController@U2@@0P6AXXZA 10008474     OpenCLSupportSettingsController.obj
 0002:00000478       ?staticMetaObject$initializer$@OpenCLSupportPlugin@U2@@2P6AXXZA 10008478     moc_OpenCLSupportPlugin.obj
 0002:0000047c       ?staticMetaObject$initializer$@OpenCLSupportSettingsPageController@U2@@2P6AXXZA 1000847c     moc_OpenCLSupportSettingsController.obj
 0002:00000480       ?staticMetaObject$initializer$@OpenCLSupportSettingsPageState@U2@@2P6AXXZA 10008480     moc_OpenCLSupportSettingsController.obj
 0002:00000484       ?staticMetaObject$initializer$@OpenCLSupportSettingsPageWidget@U2@@2P6AXXZA 10008484     moc_OpenCLSupportSettingsController.obj
 0002:00000490       _pcinit                    10008490     MSVCRT:crtdll.obj
 0002:00000494       _pinit                     10008494     MSVCRT:atonexit.obj
 0002:00000f8c       _qt_meta_stringdata_U2__OpenCLSupportPlugin 10008f8c     moc_OpenCLSupportPlugin.obj
 0002:00000fb4       _qt_meta_data_U2__OpenCLSupportPlugin 10008fb4     moc_OpenCLSupportPlugin.obj
 0002:00000ff0       _qt_meta_stringdata_U2__OpenCLSupportSettingsPageController 10008ff0     moc_OpenCLSupportSettingsController.obj
 0002:00001028       _qt_meta_data_U2__OpenCLSupportSettingsPageController 10009028     moc_OpenCLSupportSettingsController.obj
 0002:00001064       _qt_meta_stringdata_U2__OpenCLSupportSettingsPageState 10009064     moc_OpenCLSupportSettingsController.obj
 0002:00001098       _qt_meta_data_U2__OpenCLSupportSettingsPageState 10009098     moc_OpenCLSupportSettingsController.obj
 0002:000010d4       _qt_meta_stringdata_U2__OpenCLSupportSettingsPageWidget 100090d4     moc_OpenCLSupportSettingsController.obj
 0002:00001108       _qt_meta_data_U2__OpenCLSupportSettingsPageWidget 10009108     moc_OpenCLSupportSettingsController.obj
 0002:00001154       _GS_ExceptionPointers      10009154     MSVCRT:gs_report.obj
 0002:00001b08       __catchsym$?_Copy@?$basic_string@DU?$char_traits@D@std@@V?$allocator@D@2@@std@@QAEXII@Z$5 10009b08     OpenCLSupportPlugin.obj
 0002:00001b18       __catchsym$?_Copy@?$basic_string@DU?$char_traits@D@std@@V?$allocator@D@2@@std@@QAEXII@Z$4 10009b18     OpenCLSupportPlugin.obj
 0002:00001b28       __unwindtable$?_Copy@?$basic_string@DU?$char_traits@D@std@@V?$allocator@D@2@@std@@QAEXII@Z 10009b28     OpenCLSupportPlugin.obj
 0002:00001b48       __ehfuncinfo$?_Copy@?$basic_string@DU?$char_traits@D@std@@V?$allocator@D@2@@std@@QAEXII@Z 10009b48     OpenCLSupportPlugin.obj
 0002:00001b6c       __tryblocktable$?_Copy@?$basic_string@DU?$char_traits@D@std@@V?$allocator@D@2@@std@@QAEXII@Z 10009b6c     OpenCLSupportPlugin.obj
 0002:00001b94       __unwindtable$??H@YA?BVQString@@ABV0@0@Z 10009b94     OpenCLSupportPlugin.obj
 0002:00001b9c       __ehfuncinfo$??H@YA?BVQString@@ABV0@0@Z 10009b9c     OpenCLSupportPlugin.obj
 0002:00001bc0       __unwindtable$??H@YA?BVQString@@ABV0@PBD@Z 10009bc0     OpenCLSupportPlugin.obj
 0002:00001bd0       __ehfuncinfo$??H@YA?BVQString@@ABV0@PBD@Z 10009bd0     OpenCLSupportPlugin.obj
 0002:00001bf4       __unwindtable$??H@YA?BVQString@@PBDABV0@@Z 10009bf4     OpenCLSupportPlugin.obj
 0002:00001bfc       __ehfuncinfo$??H@YA?BVQString@@PBDABV0@@Z 10009bfc     OpenCLSupportPlugin.obj
 0002:00001c20       __unwindtable$??__EalgoLog@U2@@YAXXZ 10009c20     OpenCLSupportPlugin.obj
 0002:00001c28       __ehfuncinfo$??__EalgoLog@U2@@YAXXZ 10009c28     OpenCLSupportPlugin.obj
 0002:00001c4c       __unwindtable$??__EcmdLog@U2@@YAXXZ 10009c4c     OpenCLSupportPlugin.obj
 0002:00001c54       __ehfuncinfo$??__EcmdLog@U2@@YAXXZ 10009c54     OpenCLSupportPlugin.obj
 0002:00001c78       __unwindtable$??__EcoreLog@U2@@YAXXZ 10009c78     OpenCLSupportPlugin.obj
 0002:00001c80       __ehfuncinfo$??__EcoreLog@U2@@YAXXZ 10009c80     OpenCLSupportPlugin.obj
 0002:00001ca4       __unwindtable$??__EioLog@U2@@YAXXZ 10009ca4     OpenCLSupportPlugin.obj
 0002:00001cac       __ehfuncinfo$??__EioLog@U2@@YAXXZ 10009cac     OpenCLSupportPlugin.obj
 0002:00001cd0       __unwindtable$??__EperfLog@U2@@YAXXZ 10009cd0     OpenCLSupportPlugin.obj
 0002:00001cd8       __ehfuncinfo$??__EperfLog@U2@@YAXXZ 10009cd8     OpenCLSupportPlugin.obj
 0002:00001cfc       __unwindtable$??__EscriptLog@U2@@YAXXZ 10009cfc     OpenCLSupportPlugin.obj
 0002:00001d04       __ehfuncinfo$??__EscriptLog@U2@@YAXXZ 10009d04     OpenCLSupportPlugin.obj
 0002:00001d28       __unwindtable$??__EtaskLog@U2@@YAXXZ 10009d28     OpenCLSupportPlugin.obj
 0002:00001d30       __ehfuncinfo$??__EtaskLog@U2@@YAXXZ 10009d30     OpenCLSupportPlugin.obj
 0002:00001d54       __unwindtable$??__EuiLog@U2@@YAXXZ 10009d54     OpenCLSupportPlugin.obj
 0002:00001d5c       __ehfuncinfo$??__EuiLog@U2@@YAXXZ 10009d5c     OpenCLSupportPlugin.obj
 0002:00001d80       __unwindtable$??__EuserActLog@U2@@YAXXZ 10009d80     OpenCLSupportPlugin.obj
 0002:00001d88       __ehfuncinfo$??__EuserActLog@U2@@YAXXZ 10009d88     OpenCLSupportPlugin.obj
 0002:00001dac       __ehfuncinfo$??0OpenCLSupportPlugin@U2@@QAE@XZ 10009dac     OpenCLSupportPlugin.obj
 0002:00001dd0       __unwindtable$??0OpenCLSupportPlugin@U2@@QAE@XZ 10009dd0     OpenCLSupportPlugin.obj
 0002:00001e50       __unwindtable$??1OpenCLSupportPlugin@U2@@UAE@XZ 10009e50     OpenCLSupportPlugin.obj
 0002:00001e68       __ehfuncinfo$??1OpenCLSupportPlugin@U2@@UAE@XZ 10009e68     OpenCLSupportPlugin.obj
 0002:00001e8c       __ehfuncinfo$?obtainGpusInfo@OpenCLSupportPlugin@U2@@AAE?AW4OpenCLSupportError@12@AAVQString@@@Z 10009e8c     OpenCLSupportPlugin.obj
 0002:00001eb0       __unwindtable$?obtainGpusInfo@OpenCLSupportPlugin@U2@@AAE?AW4OpenCLSupportError@12@AAVQString@@@Z 10009eb0     OpenCLSupportPlugin.obj
 0002:00001f80       __ehfuncinfo$?loadGpusSettings@OpenCLSupportPlugin@U2@@AAEXXZ 10009f80     OpenCLSupportPlugin.obj
 0002:00001fa4       __unwindtable$?loadGpusSettings@OpenCLSupportPlugin@U2@@AAEXXZ 10009fa4     OpenCLSupportPlugin.obj
 0002:00001fec       __unwindtable$?registerAvailableGpus@OpenCLSupportPlugin@U2@@AAEXXZ 10009fec     OpenCLSupportPlugin.obj
 0002:00001ff4       __ehfuncinfo$?registerAvailableGpus@OpenCLSupportPlugin@U2@@AAEXXZ 10009ff4     OpenCLSupportPlugin.obj
 0002:00002018       __unwindtable$?unregisterAvailableGpus@OpenCLSupportPlugin@U2@@AAEXXZ 1000a018     OpenCLSupportPlugin.obj
 0002:00002020       __ehfuncinfo$?unregisterAvailableGpus@OpenCLSupportPlugin@U2@@AAEXXZ 1000a020     OpenCLSupportPlugin.obj
 0002:00002044       __unwindtable$?hasOPENCLError@OpenCLSupportPlugin@U2@@AAE_NHAAVQString@@@Z 1000a044     OpenCLSupportPlugin.obj
 0002:00002054       __ehfuncinfo$?hasOPENCLError@OpenCLSupportPlugin@U2@@AAE_NHAAVQString@@@Z 1000a054     OpenCLSupportPlugin.obj
 0002:00002078       __catchsym$??0?$QList@PAVOpenCLGpuModel@U2@@@@QAE@ABV0@@Z$2 1000a078     OpenCLSupportPlugin.obj
 0002:00002088       __unwindtable$??0?$QList@PAVOpenCLGpuModel@U2@@@@QAE@ABV0@@Z 1000a088     OpenCLSupportPlugin.obj
 0002:00002098       __tryblocktable$??0?$QList@PAVOpenCLGpuModel@U2@@@@QAE@ABV0@@Z 1000a098     OpenCLSupportPlugin.obj
 0002:000020ac       __ehfuncinfo$??0?$QList@PAVOpenCLGpuModel@U2@@@@QAE@ABV0@@Z 1000a0ac     OpenCLSupportPlugin.obj
 0002:000020d0       __catchsym$?append@?$QList@PAVOpenCLGpuModel@U2@@@@QAEXABQAVOpenCLGpuModel@U2@@@Z$6 1000a0d0     OpenCLSupportPlugin.obj
 0002:000020e0       __tryblocktable$?append@?$QList@PAVOpenCLGpuModel@U2@@@@QAEXABQAVOpenCLGpuModel@U2@@@Z 1000a0e0     OpenCLSupportPlugin.obj
 0002:000020f4       __ehfuncinfo$?append@?$QList@PAVOpenCLGpuModel@U2@@@@QAEXABQAVOpenCLGpuModel@U2@@@Z 1000a0f4     OpenCLSupportPlugin.obj
 0002:00002118       __unwindtable$?append@?$QList@PAVOpenCLGpuModel@U2@@@@QAEXABQAVOpenCLGpuModel@U2@@@Z 1000a118     OpenCLSupportPlugin.obj
 0002:00002148       __catchsym$?detach_helper_grow@?$QList@PAVOpenCLGpuModel@U2@@@@AAEPAUNode@1@HH@Z$5 1000a148     OpenCLSupportPlugin.obj
 0002:00002158       __catchsym$?detach_helper_grow@?$QList@PAVOpenCLGpuModel@U2@@@@AAEPAUNode@1@HH@Z$4 1000a158     OpenCLSupportPlugin.obj
 0002:00002168       __unwindtable$?detach_helper_grow@?$QList@PAVOpenCLGpuModel@U2@@@@AAEPAUNode@1@HH@Z 1000a168     OpenCLSupportPlugin.obj
 0002:00002188       __ehfuncinfo$?detach_helper_grow@?$QList@PAVOpenCLGpuModel@U2@@@@AAEPAUNode@1@HH@Z 1000a188     OpenCLSupportPlugin.obj
 0002:000021ac       __tryblocktable$?detach_helper_grow@?$QList@PAVOpenCLGpuModel@U2@@@@AAEPAUNode@1@HH@Z 1000a1ac     OpenCLSupportPlugin.obj
 0002:000021d4       __unwindtable$??__EalgoLog@U2@@YAXXZ 1000a1d4     OpenCLSupportSettingsController.obj
 0002:000021dc       __ehfuncinfo$??__EalgoLog@U2@@YAXXZ 1000a1dc     OpenCLSupportSettingsController.obj
 0002:00002200       __unwindtable$??__EcmdLog@U2@@YAXXZ 1000a200     OpenCLSupportSettingsController.obj
 0002:00002208       __ehfuncinfo$??__EcmdLog@U2@@YAXXZ 1000a208     OpenCLSupportSettingsController.obj
 0002:0000222c       __unwindtable$??__EcoreLog@U2@@YAXXZ 1000a22c     OpenCLSupportSettingsController.obj
 0002:00002234       __ehfuncinfo$??__EcoreLog@U2@@YAXXZ 1000a234     OpenCLSupportSettingsController.obj
 0002:00002258       __unwindtable$??__EioLog@U2@@YAXXZ 1000a258     OpenCLSupportSettingsController.obj
 0002:00002260       __ehfuncinfo$??__EioLog@U2@@YAXXZ 1000a260     OpenCLSupportSettingsController.obj
 0002:00002284       __unwindtable$??__EperfLog@U2@@YAXXZ 1000a284     OpenCLSupportSettingsController.obj
 0002:0000228c       __ehfuncinfo$??__EperfLog@U2@@YAXXZ 1000a28c     OpenCLSupportSettingsController.obj
 0002:000022b0       __unwindtable$??__EscriptLog@U2@@YAXXZ 1000a2b0     OpenCLSupportSettingsController.obj
 0002:000022b8       __ehfuncinfo$??__EscriptLog@U2@@YAXXZ 1000a2b8     OpenCLSupportSettingsController.obj
 0002:000022dc       __unwindtable$??__EtaskLog@U2@@YAXXZ 1000a2dc     OpenCLSupportSettingsController.obj
 0002:000022e4       __ehfuncinfo$??__EtaskLog@U2@@YAXXZ 1000a2e4     OpenCLSupportSettingsController.obj
 0002:00002308       __unwindtable$??__EuiLog@U2@@YAXXZ 1000a308     OpenCLSupportSettingsController.obj
 0002:00002310       __ehfuncinfo$??__EuiLog@U2@@YAXXZ 1000a310     OpenCLSupportSettingsController.obj
 0002:00002334       __unwindtable$??__EuserActLog@U2@@YAXXZ 1000a334     OpenCLSupportSettingsController.obj
 0002:0000233c       __ehfuncinfo$??__EuserActLog@U2@@YAXXZ 1000a33c     OpenCLSupportSettingsController.obj
 0002:00002360       __ehfuncinfo$??0OpenCLSupportSettingsPageController@U2@@QAE@ABVQString@@PAVQObject@@@Z 1000a360     OpenCLSupportSettingsController.obj
 0002:00002384       __unwindtable$??0OpenCLSupportSettingsPageController@U2@@QAE@ABVQString@@PAVQObject@@@Z 1000a384     OpenCLSupportSettingsController.obj
 0002:000023ac       __unwindtable$?getSavedState@OpenCLSupportSettingsPageController@U2@@UAEPAVAppSettingsGUIPageState@2@XZ 1000a3ac     OpenCLSupportSettingsController.obj
 0002:000023bc       __ehfuncinfo$?getSavedState@OpenCLSupportSettingsPageController@U2@@UAEPAVAppSettingsGUIPageState@2@XZ 1000a3bc     OpenCLSupportSettingsController.obj
 0002:000023e0       __unwindtable$?saveState@OpenCLSupportSettingsPageController@U2@@UAEXPAVAppSettingsGUIPageState@2@@Z 1000a3e0     OpenCLSupportSettingsController.obj
 0002:000023e8       __ehfuncinfo$?saveState@OpenCLSupportSettingsPageController@U2@@UAEXPAVAppSettingsGUIPageState@2@@Z 1000a3e8     OpenCLSupportSettingsController.obj
 0002:0000240c       __unwindtable$?createWidget@OpenCLSupportSettingsPageController@U2@@UAEPAVAppSettingsGUIPageWidget@2@PAVAppSettingsGUIPageState@2@@Z 1000a40c     OpenCLSupportSettingsController.obj
 0002:00002414       __ehfuncinfo$?createWidget@OpenCLSupportSettingsPageController@U2@@UAEPAVAppSettingsGUIPageWidget@2@PAVAppSettingsGUIPageState@2@@Z 1000a414     OpenCLSupportSettingsController.obj
 0002:00002438       __unwindtable$??1OpenCLSupportSettingsPageController@U2@@UAE@XZ 1000a438     OpenCLSupportSettingsController.obj
 0002:00002440       __ehfuncinfo$??1OpenCLSupportSettingsPageController@U2@@UAE@XZ 1000a440     OpenCLSupportSettingsController.obj
 0002:00002464       __unwindtable$??_GOpenCLSupportSettingsPageController@U2@@UAEPAXI@Z 1000a464     OpenCLSupportSettingsController.obj
 0002:0000246c       __ehfuncinfo$??_GOpenCLSupportSettingsPageController@U2@@UAEPAXI@Z 1000a46c     OpenCLSupportSettingsController.obj
 0002:00002490       __unwindtable$??0OpenCLSupportSettingsPageState@U2@@QAE@H@Z 1000a490     OpenCLSupportSettingsController.obj
 0002:000024a0       __ehfuncinfo$??0OpenCLSupportSettingsPageState@U2@@QAE@H@Z 1000a4a0     OpenCLSupportSettingsController.obj
 0002:000024c4       __catchsym$?reallocData@?$QVector@_N@@AAEXHHV?$QFlags@W4AllocationOption@QArrayData@@@@@Z$5 1000a4c4     OpenCLSupportSettingsController.obj
 0002:000024d4       __catchsym$?reallocData@?$QVector@_N@@AAEXHHV?$QFlags@W4AllocationOption@QArrayData@@@@@Z$4 1000a4d4     OpenCLSupportSettingsController.obj
 0002:000024e4       __unwindtable$?reallocData@?$QVector@_N@@AAEXHHV?$QFlags@W4AllocationOption@QArrayData@@@@@Z 1000a4e4     OpenCLSupportSettingsController.obj
 0002:00002504       __ehfuncinfo$?reallocData@?$QVector@_N@@AAEXHHV?$QFlags@W4AllocationOption@QArrayData@@@@@Z 1000a504     OpenCLSupportSettingsController.obj
 0002:00002528       __tryblocktable$?reallocData@?$QVector@_N@@AAEXHHV?$QFlags@W4AllocationOption@QArrayData@@@@@Z 1000a528     OpenCLSupportSettingsController.obj
 0002:00002550       __unwindtable$??1OpenCLSupportSettingsPageState@U2@@UAE@XZ 1000a550     OpenCLSupportSettingsController.obj
 0002:00002558       __ehfuncinfo$??1OpenCLSupportSettingsPageState@U2@@UAE@XZ 1000a558     OpenCLSupportSettingsController.obj
 0002:0000257c       __unwindtable$??_GOpenCLSupportSettingsPageState@U2@@UAEPAXI@Z 1000a57c     OpenCLSupportSettingsController.obj
 0002:00002584       __ehfuncinfo$??_GOpenCLSupportSettingsPageState@U2@@UAEPAXI@Z 1000a584     OpenCLSupportSettingsController.obj
 0002:000025a8       __ehfuncinfo$??0OpenCLSupportSettingsPageWidget@U2@@QAE@ABVQString@@PAVOpenCLSupportSettingsPageController@1@@Z 1000a5a8     OpenCLSupportSettingsController.obj
 0002:000025cc       __unwindtable$??0OpenCLSupportSettingsPageWidget@U2@@QAE@ABVQString@@PAVOpenCLSupportSettingsPageController@1@@Z 1000a5cc     OpenCLSupportSettingsController.obj
 0002:00002694       __unwindtable$?getState@OpenCLSupportSettingsPageWidget@U2@@UBEPAVAppSettingsGUIPageState@2@AAVQString@@@Z 1000a694     OpenCLSupportSettingsController.obj
 0002:0000269c       __ehfuncinfo$?getState@OpenCLSupportSettingsPageWidget@U2@@UBEPAVAppSettingsGUIPageState@2@AAVQString@@@Z 1000a69c     OpenCLSupportSettingsController.obj
 0002:000026c0       __catchsym$?append@?$QList@PAVQCheckBox@@@@QAEXABQAVQCheckBox@@@Z$6 1000a6c0     OpenCLSupportSettingsController.obj
 0002:000026d0       __tryblocktable$?append@?$QList@PAVQCheckBox@@@@QAEXABQAVQCheckBox@@@Z 1000a6d0     OpenCLSupportSettingsController.obj
 0002:000026e4       __ehfuncinfo$?append@?$QList@PAVQCheckBox@@@@QAEXABQAVQCheckBox@@@Z 1000a6e4     OpenCLSupportSettingsController.obj
 0002:00002708       __unwindtable$?append@?$QList@PAVQCheckBox@@@@QAEXABQAVQCheckBox@@@Z 1000a708     OpenCLSupportSettingsController.obj
 0002:00002738       __catchsym$?detach_helper_grow@?$QList@PAVQCheckBox@@@@AAEPAUNode@1@HH@Z$5 1000a738     OpenCLSupportSettingsController.obj
 0002:00002748       __catchsym$?detach_helper_grow@?$QList@PAVQCheckBox@@@@AAEPAUNode@1@HH@Z$4 1000a748     OpenCLSupportSettingsController.obj
 0002:00002758       __unwindtable$?detach_helper_grow@?$QList@PAVQCheckBox@@@@AAEPAUNode@1@HH@Z 1000a758     OpenCLSupportSettingsController.obj
 0002:00002778       __ehfuncinfo$?detach_helper_grow@?$QList@PAVQCheckBox@@@@AAEPAUNode@1@HH@Z 1000a778     OpenCLSupportSettingsController.obj
 0002:0000279c       __tryblocktable$?detach_helper_grow@?$QList@PAVQCheckBox@@@@AAEPAUNode@1@HH@Z 1000a79c     OpenCLSupportSettingsController.obj
 0002:000027c4       __unwindtable$??1OpenCLSupportSettingsPageWidget@U2@@UAE@XZ 1000a7c4     OpenCLSupportSettingsController.obj
 0002:000027d4       __ehfuncinfo$??1OpenCLSupportSettingsPageWidget@U2@@UAE@XZ 1000a7d4     OpenCLSupportSettingsController.obj
 0002:000027f8       __unwindtable$??_GOpenCLSupportSettingsPageWidget@U2@@UAEPAXI@Z 1000a7f8     OpenCLSupportSettingsController.obj
 0002:00002808       __ehfuncinfo$??_GOpenCLSupportSettingsPageWidget@U2@@UAEPAXI@Z 1000a808     OpenCLSupportSettingsController.obj
 0002:0000282c       __catchsym$?detach_helper@?$QList@PAVOpenCLGpuModel@U2@@@@AAEXH@Z$2 1000a82c     OpenCLSupportSettingsController.obj
 0002:0000283c       __unwindtable$?detach_helper@?$QList@PAVOpenCLGpuModel@U2@@@@AAEXH@Z 1000a83c     OpenCLSupportSettingsController.obj
 0002:0000284c       __tryblocktable$?detach_helper@?$QList@PAVOpenCLGpuModel@U2@@@@AAEXH@Z 1000a84c     OpenCLSupportSettingsController.obj
 0002:00002860       __ehfuncinfo$?detach_helper@?$QList@PAVOpenCLGpuModel@U2@@@@AAEXH@Z 1000a860     OpenCLSupportSettingsController.obj
 0002:00002888       __sehtable$__onexit        1000a888     MSVCRT:atonexit.obj
 0002:000028a8       __sehtable$___DllMainCRTStartup 1000a8a8     MSVCRT:crtdll.obj
 0002:000028d0       __sehtable$??_M@YGXPAXIHP6EX0@Z@Z 1000a8d0     MSVCRT:ehvecdtr.obj
 0002:000028f0       __sehtable$?__ArrayUnwind@@YGXPAXIHP6EX0@Z@Z 1000a8f0     MSVCRT:ehvecdtr.obj
 0002:00002910       __sehtable$__IsNonwritableInCurrentImage 1000a910     MSVCRT:pesect.obj
 0002:00002930       .edata                     1000a930     opencl_support.exp
 0002:00002958       rgpv                       1000a958     opencl_support.exp
 0002:00002964       rgszName                   1000a964     opencl_support.exp
 0002:00002970       rgwOrd                     1000a970     opencl_support.exp
 0002:00002976       szName                     1000a976     opencl_support.exp
 0002:00002989       $N00001                    1000a989     opencl_support.exp
 0002:000029a3       $N00002                    1000a9a3     opencl_support.exp
 0002:000029b5       $N00003                    1000a9b5     opencl_support.exp
 0002:000033ba       .idata$6                   1000b3ba     U2Core:U2Core.dll
 0002:00003584       .idata$6                   1000b584     U2Algorithm:U2Algorithm.dll
 0002:000038f2       .idata$6                   1000b8f2     U2Gui:U2Gui.dll
 0002:00004f46       .idata$6                   1000cf46     Qt5Widgets:Qt5Widgets.dll
 0002:00005550       .idata$6                   1000d550     Qt5Core:Qt5Core.dll
 0002:000055f6       .idata$6                   1000d5f6     msvcprt:MSVCP120.dll
 0002:000056b0       .idata$6                   1000d6b0     MSVCRT:MSVCR120.dll
 0002:000058c4       .idata$6                   1000d8c4     kernel32:KERNEL32.dll
 0003:00000000       _RESOURCE_OPENCL_GPU_NAME  1000e000     OpenCLSupportPlugin.obj
 0003:00000010       _gpusDiscoveredText        1000e010     OpenCLSupportSettingsController.obj
 0003:00000014       _noGpusDiscoveredText      1000e014     OpenCLSupportSettingsController.obj
 0003:00000430       __Tuple_alloc              1000e430     OpenCLSupportPlugin.obj
 0003:00000431       _ignore                    1000e431     OpenCLSupportPlugin.obj
 0003:00000432       _allocator_arg             1000e432     OpenCLSupportPlugin.obj
 0003:00000433       _piecewise_construct       1000e433     OpenCLSupportPlugin.obj
 0003:00000434       _taskLog                   1000e434     OpenCLSupportPlugin.obj
 0003:0000043c       _algoLog                   1000e43c     OpenCLSupportPlugin.obj
 0003:00000444       _userActLog                1000e444     OpenCLSupportPlugin.obj
 0003:0000044c       _ioLog                     1000e44c     OpenCLSupportPlugin.obj
 0003:00000454       _coreLog                   1000e454     OpenCLSupportPlugin.obj
 0003:0000045c       _uiLog                     1000e45c     OpenCLSupportPlugin.obj
 0003:00000464       _scriptLog                 1000e464     OpenCLSupportPlugin.obj
 0003:0000046c       _perfLog                   1000e46c     OpenCLSupportPlugin.obj
 0003:00000474       _cmdLog                    1000e474     OpenCLSupportPlugin.obj
 0003:00000484       __Tuple_alloc              1000e484     OpenCLSupportSettingsController.obj
 0003:00000485       _ignore                    1000e485     OpenCLSupportSettingsController.obj
 0003:00000486       _allocator_arg             1000e486     OpenCLSupportSettingsController.obj
 0003:00000487       _piecewise_construct       1000e487     OpenCLSupportSettingsController.obj
 0003:00000488       _taskLog                   1000e488     OpenCLSupportSettingsController.obj
 0003:00000490       _algoLog                   1000e490     OpenCLSupportSettingsController.obj
 0003:00000498       _userActLog                1000e498     OpenCLSupportSettingsController.obj
 0003:000004a0       _ioLog                     1000e4a0     OpenCLSupportSettingsController.obj
 0003:000004a8       _coreLog                   1000e4a8     OpenCLSupportSettingsController.obj
 0003:000004b0       _uiLog                     1000e4b0     OpenCLSupportSettingsController.obj
 0003:000004b8       _scriptLog                 1000e4b8     OpenCLSupportSettingsController.obj
 0003:000004c0       _perfLog                   1000e4c0     OpenCLSupportSettingsController.obj
 0003:000004c8       _cmdLog                    1000e4c8     OpenCLSupportSettingsController.obj
 0003:000004d4       __Tuple_alloc              1000e4d4     moc_OpenCLSupportPlugin.obj
 0003:000004d5       _ignore                    1000e4d5     moc_OpenCLSupportPlugin.obj
 0003:000004d6       _allocator_arg             1000e4d6     moc_OpenCLSupportPlugin.obj
 0003:000004d7       _piecewise_construct       1000e4d7     moc_OpenCLSupportPlugin.obj
 0003:000004d8       __Tuple_alloc              1000e4d8     moc_OpenCLSupportSettingsController.obj
 0003:000004d9       _ignore                    1000e4d9     moc_OpenCLSupportSettingsController.obj
 0003:000004da       _allocator_arg             1000e4da     moc_OpenCLSupportSettingsController.obj
 0003:000004db       _piecewise_construct       1000e4db     moc_OpenCLSupportSettingsController.obj
 0003:000004dc       ___proc_attached           1000e4dc     MSVCRT:crtdll.obj
 0003:000004e0       _GS_ExceptionRecord        1000e4e0     MSVCRT:gs_report.obj
 0003:00000530       _GS_ContextRecord          1000e530     MSVCRT:gs_report.obj
 0003:000007fc       _DebuggerWasPresent        1000e7fc     MSVCRT:gs_report.obj
 0004:00000060       $R000000                   1000f060     * linker generated manifest res *

 Exports

  ordinal    name

        1    _ugene_plugin_fail_message
               exported name: ugene_plugin_fail_message
        2    _ugene_plugin_init
               exported name: ugene_plugin_init
        3    _ugene_plugin_verify
               exported name: ugene_plugin_verify
